 csp_serial

 Timestamp is 4da2a518 (Mon Apr 11 18:52:08 2011)

 Preferred load address is 10000000

 Start         Length     Name                   Class
 0001:00000000 00000004H .CRT$XCA                CODE
 0001:00000004 00000004H .CRT$XCZ                CODE
 0001:00000008 00000004H .CRT$XIA                CODE
 0001:0000000c 00000004H .CRT$XIZ                CODE
 0001:00000010 00000004H .CRT$XPA                CODE
 0001:00000014 00000004H .CRT$XPZ                CODE
 0001:00000018 00000004H .CRT$XTA                CODE
 0001:0000001c 00000004H .CRT$XTZ                CODE
 0001:00000020 00006298H .rdata                  CODE
 0001:000062b8 00000027H .rdata$debug            CODE
 0001:000062e0 00011840H .text                   CODE
 0001:00017b20 00000220H .xdata                  CODE
 0001:00017d40 0000003cH .idata$2                CODE
 0001:00017d7c 00000014H .idata$3                CODE
 0001:00017d90 00000128H .idata$4                CODE
 0001:00017eb8 0000014eH .idata$6                CODE
 0001:00018010 00000136H .edata                  CODE
 0002:00000000 00000128H .idata$5                DATA
 0002:00000128 0000044cH .data                   DATA
 0002:00000574 00000018H .bss                    DATA
 0003:00000000 000004b0H .pdata                  DATA

  Address         Publics by Value              Rva+Base       Lib:Object

 0000:00000000       ___safe_se_handler_table   00000000     <absolute>
 0000:00000000       ___safe_se_handler_count   00000000     <absolute>
 0001:00000000       __xc_a                     10001000     corelib0:crt0init.obj
 0001:00000004       __xc_z                     10001004     corelib0:crt0init.obj
 0001:00000008       __xi_a                     10001008     corelib0:crt0init.obj
 0001:0000000c       __xi_z                     1000100c     corelib0:crt0init.obj
 0001:00000010       __xp_a                     10001010     corelib0:crt0init.obj
 0001:00000014       __xp_z                     10001014     corelib0:crt0init.obj
 0001:00000018       __xt_a                     10001018     corelib0:crt0init.obj
 0001:0000001c       __xt_z                     1000101c     corelib0:crt0init.obj
 0001:0000003c       ??_C@_1DA@LGJDGOIM@?$AAp?$AAr?$AAo?$AAc?$AAe?$AAs?$AAs?$AA?5?$AAd?$AAe?$AAt?$AAa?$AAc?$AAh?$AA?5?$AAc?$AAa?$AAl?$AAl?$AAe?$AAd?$AA?$AN?$AA?6?$AA?$AA@ 1000103c     com_mdd2:mdd.obj
 0001:0000006c       ??_C@_1DK@BHNGFHBN@?$AAs?$AAe?$AAr?$AAi?$AAa?$AAl?$AA?5?$AAp?$AAo?$AAr?$AAt?$AA?5?$AAp?$AAr?$AAo?$AAc?$AAe?$AAs?$AAs?$AA?5?$AAa?$AAt?$AAt?$AAa?$AAc?$AAh?$AA?$AN?$AA?6?$AA?$AA@ 1000106c     com_mdd2:mdd.obj
 0001:000000a8       ??_C@_1EG@PNOECNFM@?$AAD?$AAo?$AAP?$AAu?$AAt?$AAB?$AAy?$AAt?$AAe?$AAs?$AA?5?$AAr?$AAe?$AAl?$AAe?$AAa?$AAs?$AAe?$AAd?$AA?5?$AAC?$AAr?$AAi?$AAt?$AAS?$AAe?$AAc?$AA?3?$AA?5?$AA?$CF?$AAx?$AA?4@ 100010a8     com_mdd2:mdd.obj
 0001:000000f0       ??_C@_1EO@IFEAHMMF@?$AAT?$AAr?$AAa?$AAn?$AAs?$AAm?$AAi?$AAs?$AAs?$AAi?$AAo?$AAn?$AA?5?$AAc?$AAo?$AAm?$AAp?$AAl?$AAe?$AAt?$AAe?$AA?0?$AA?5?$AA?$CF?$AAd?$AA?5?$AAb?$AAy?$AAt?$AAe?$AAs?$AA?5@ 100010f0     com_mdd2:mdd.obj
 0001:00000140       ??_C@_1DI@GGPGJBLB@?$AA?$CF?$AAd?$AA?5?$AAb?$AAy?$AAt?$AAe?$AAs?$AA?5?$AAa?$AAc?$AAt?$AAu?$AAa?$AAl?$AAl?$AAy?$AA?5?$AAc?$AAo?$AAp?$AAi?$AAe?$AAd?$AA?4?$AA?$AN?$AA?6?$AA?$AA@ 10001140     com_mdd2:mdd.obj
 0001:00000178       ??_C@_1DC@FONCMGND@?$AAA?$AAb?$AAo?$AAu?$AAt?$AA?5?$AAt?$AAo?$AA?5?$AAc?$AAo?$AAp?$AAy?$AA?5?$AA?$CF?$AAd?$AA?5?$AAb?$AAy?$AAt?$AAe?$AAs?$AA?$AN?$AA?6?$AA?$AA@ 10001178     com_mdd2:mdd.obj
 0001:000001b0       ??_C@_1GC@MPMHAODJ@?$AAT?$AAx?$AAR?$AAe?$AAa?$AAd?$AA?5?$AA?$DN?$AA?5?$AA?$CF?$AAd?$AA?0?$AA?5?$AAT?$AAx?$AAL?$AAe?$AAn?$AAg?$AAt?$AAh?$AA?5?$AA?$DN?$AA?5?$AA?$CF?$AAd?$AA?0?$AA?5?$AAT?$AAx?$AAB?$AAy@ 100011b0     com_mdd2:mdd.obj
 0001:00000214       ??_C@_1DC@KIHGPOMJ@?$AAX?$AAO?$AAF?$AAF?$AA?8?$AAe?$AAd?$AA?0?$AA?5?$AAs?$AAe?$AAn?$AAd?$AA?5?$AAn?$AAo?$AAt?$AAh?$AAi?$AAn?$AAg?$AA?4?$AA?$AN?$AA?6?$AA?$AA@ 10001214     com_mdd2:mdd.obj
 0001:00000248       ??_C@_1BG@OPJKPKO@?$AAR?$AAT?$AAS?$AA?5?$AAs?$AAe?$AAt?$AA?4?$AA?$AN?$AA?6?$AA?$AA@ 10001248     com_mdd2:mdd.obj
 0001:00000260       ??_C@_1FC@IBKKBMKO@?$AAS?$AAe?$AAr?$AAi?$AAa?$AAl?$AAE?$AAv?$AAe?$AAn?$AAt?$AAH?$AAa?$AAn?$AAd?$AAl?$AAe?$AAr?$AA?3?$AA?5?$AA?$CF?$AAd?$AA?5?$AAs?$AAe?$AAn?$AAt?$AA?5?$AAu?$AAp?$AA?9?$AAt@ 10001260     com_mdd2:mdd.obj
 0001:000002b8       ??_C@_1EI@PHLIHGKN@?$AAD?$AAe?$AAv?$AAi?$AAc?$AAe?$AA?5?$AAc?$AAl?$AAo?$AAs?$AAe?$AAd?$AA?$CB?$AA?5?$AAQ?$AAu?$AAi?$AAt?$AA?5?$AAt?$AAr?$AAa?$AAn?$AAs?$AAm?$AAi?$AAs?$AAs?$AAi?$AAo?$AAn@ 100012b8     com_mdd2:mdd.obj
 0001:00000300       ??_C@_1DK@JKMHGAMG@?$AAD?$AAo?$AAP?$AAu?$AAt?$AAB?$AAy?$AAt?$AAe?$AAs?$AA?5?$AAg?$AAo?$AAt?$AA?5?$AAC?$AAr?$AAi?$AAt?$AAS?$AAe?$AAc?$AA?5?$AA?$CF?$AAx?$AA?4?$AA?$AN?$AA?6?$AA?$AA@ 10001300     com_mdd2:mdd.obj
 0001:00000340       ??_C@_1EE@GKGAJBJP@?$AAD?$AAo?$AAP?$AAu?$AAt?$AAB?$AAy?$AAt?$AAe?$AAs?$AA?5?$AAw?$AAa?$AAi?$AAt?$AA?5?$AAf?$AAo?$AAr?$AA?5?$AAC?$AAr?$AAi?$AAt?$AAS?$AAe?$AAc?$AA?5?$AA?$CF?$AAx?$AA?4?$AA?$AN@ 10001340     com_mdd2:mdd.obj
 0001:00000388       ??_C@_1FI@GGFBGELP@?$AA?9?$AAS?$AAe?$AAr?$AAi?$AAa?$AAl?$AAE?$AAv?$AAe?$AAn?$AAt?$AAH?$AAa?$AAn?$AAd?$AAl?$AAe?$AAr?$AA?0?$AA?5?$AAF?$AAi?$AAf?$AAo?$AA?$CI?$AAR?$AA?$DN?$AA?$CF?$AAd?$AA?0?$AAW@ 10001388     com_mdd2:mdd.obj
 0001:000003e0       ??_C@_1CI@EJHAPNLK@?$AAL?$AAi?$AAn?$AAe?$AA?5?$AAE?$AAv?$AAe?$AAn?$AAt?$AA?0?$AA?5?$AAi?$AAt?$AA?3?$AA?$CF?$AAx?$AA?$AN?$AA?6?$AA?$AA@ 100013e0     com_mdd2:mdd.obj
 0001:00000408       ??_C@_1CK@CPCFPBFI@?$AAO?$AAt?$AAh?$AAe?$AAr?$AA?5?$AAE?$AAv?$AAe?$AAn?$AAt?$AA?0?$AA?5?$AAi?$AAt?$AA?3?$AA?$CF?$AAx?$AA?$AN?$AA?6?$AA?$AA@ 10001408     com_mdd2:mdd.obj
 0001:00000434       ??_C@_1BG@KFPNBBDH@?$AAT?$AAx?$AA?5?$AAE?$AAv?$AAe?$AAn?$AAt?$AA?$AN?$AA?6?$AA?$AA@ 10001434     com_mdd2:mdd.obj
 0001:0000044c       ??_C@_1BO@CNGNDNHF@?$AAS?$AAe?$AAn?$AAd?$AAi?$AAn?$AAg?$AA?5?$AAX?$AAO?$AAF?$AAF?$AA?$AN?$AA?6?$AA?$AA@ 1000144c     com_mdd2:mdd.obj
 0001:00000470       ??_C@_1EK@LMCHJDFJ@?$AAR?$AAT?$AAS?$AA_?$AAC?$AAO?$AAN?$AAT?$AAR?$AAO?$AAL?$AA_?$AAH?$AAA?$AAN?$AAD?$AAS?$AAH?$AAA?$AAK?$AAE?$AA?5?$AAC?$AAl?$AAe?$AAa?$AAr?$AAi?$AAn?$AAg?$AA?5?$AAR@ 10001470     com_mdd2:mdd.obj
 0001:000004c0       ??_C@_1EK@FLILIJBB@?$AAD?$AAT?$AAR?$AA_?$AAC?$AAO?$AAN?$AAT?$AAR?$AAO?$AAL?$AA_?$AAH?$AAA?$AAN?$AAD?$AAS?$AAH?$AAA?$AAK?$AAE?$AA?5?$AAC?$AAl?$AAe?$AAa?$AAr?$AAi?$AAn?$AAg?$AA?5?$AAD@ 100014c0     com_mdd2:mdd.obj
 0001:0000050c       ??_C@_1BO@EEIJDLJ@?$AAR?$AAe?$AAc?$AAe?$AAi?$AAv?$AAe?$AAd?$AA?5?$AAX?$AAO?$AAN?$AA?$AN?$AA?6?$AA?$AA@ 1000150c     com_mdd2:mdd.obj
 0001:0000052c       ??_C@_1CA@EJJJJNNE@?$AAR?$AAe?$AAc?$AAe?$AAi?$AAv?$AAe?$AAd?$AA?5?$AAX?$AAO?$AAF?$AAF?$AA?$AN?$AA?6?$AA?$AA@ 1000152c     com_mdd2:mdd.obj
 0001:00000550       ??_C@_1HG@EGFFDKNF@?$AAA?$AAf?$AAt?$AAe?$AAr?$AA?5?$AAH?$AAW?$AAG?$AAe?$AAt?$AAB?$AAy?$AAt?$AAe?$AAs?$AA?0?$AA?5?$AAF?$AAi?$AAf?$AAo?$AA?$CI?$AAR?$AA?$DN?$AA?$CF?$AAd?$AA?0?$AAW?$AA?$DN?$AA?$CF?$AAd@ 10001550     com_mdd2:mdd.obj
 0001:000005c8       ??_C@_1CE@NDNCGIIC@?$AAT?$AAo?$AAs?$AAs?$AAe?$AAd?$AA?5?$AA?$CF?$AAd?$AA?5?$AAb?$AAy?$AAt?$AAe?$AAs?$AA?$AN?$AA?6?$AA?$AA@ 100015c8     com_mdd2:mdd.obj
 0001:000005ec       ??_C@_1BG@NHAMELLH@?$AAR?$AAx?$AA?5?$AAE?$AAv?$AAe?$AAn?$AAt?$AA?$AN?$AA?6?$AA?$AA@ 100015ec     com_mdd2:mdd.obj
 0001:00000608       ??_C@_1EM@PPCKGCIP@?$AAS?$AAe?$AAr?$AAi?$AAa?$AAl?$AAE?$AAv?$AAe?$AAn?$AAt?$AAH?$AAa?$AAn?$AAd?$AAl?$AAe?$AAr?$AA?0?$AA?5?$AAI?$AAn?$AAt?$AAe?$AAr?$AAr?$AAu?$AAp?$AAt?$AAs?$AA?5?$AA0@ 10001608     com_mdd2:mdd.obj
 0001:00000658       ??_C@_1EI@MHGBBLDA@?$AAS?$AAe?$AAr?$AAi?$AAa?$AAl?$AAE?$AAv?$AAe?$AAn?$AAt?$AAH?$AAa?$AAn?$AAd?$AAl?$AAe?$AAr?$AA?0?$AA?5?$AAN?$AAo?$AA?5?$AAI?$AAn?$AAt?$AAe?$AAr?$AAr?$AAu?$AAp?$AAt@ 10001658     com_mdd2:mdd.obj
 0001:000006a0       ??_C@_1CE@JLPIMJPF@?$AAE?$AAx?$AAi?$AAt?$AAt?$AAi?$AAn?$AAg?$AA?5?$AAt?$AAh?$AAr?$AAe?$AAa?$AAd?$AA?$AN?$AA?6?$AA?$AA@ 100016a0     com_mdd2:mdd.obj
 0001:000006c8       ??_C@_1EE@PGFICLOP@?$AA?$CL?$AAS?$AAe?$AAr?$AAi?$AAa?$AAl?$AAE?$AAv?$AAe?$AAn?$AAt?$AAH?$AAa?$AAn?$AAd?$AAl?$AAe?$AAr?$AA?0?$AA?5?$AAp?$AAH?$AAe?$AAa?$AAd?$AA?5?$AA0?$AAx?$AA?$CF?$AAX?$AA?$AN@ 100016c8     com_mdd2:mdd.obj
 0001:0000070c       ??_C@_1DI@KMMMNJHO@?$AAC?$AAr?$AAe?$AAa?$AAt?$AAe?$AAd?$AA?5?$AAr?$AAe?$AAc?$AAe?$AAi?$AAv?$AAe?$AA?5?$AAt?$AAh?$AAr?$AAe?$AAa?$AAd?$AA?5?$AA?$CF?$AAX?$AA?$AN?$AA?6?$AA?$AA@ 1000170c     com_mdd2:mdd.obj
 0001:00000748       ??_C@_1EM@FFMAHOCG@?$AAE?$AAr?$AAr?$AAo?$AAr?$AA?5?$AAc?$AAr?$AAe?$AAa?$AAt?$AAi?$AAn?$AAg?$AA?5?$AAd?$AAi?$AAs?$AAp?$AAa?$AAt?$AAc?$AAh?$AA?5?$AAt?$AAh?$AAr?$AAe?$AAa?$AAd?$AA?5?$AA?$CI@ 10001748     com_mdd2:mdd.obj
 0001:00000794       ??_C@_1CI@MPKANNOJ@?$AAS?$AAp?$AAi?$AAn?$AAn?$AAi?$AAn?$AAg?$AA?5?$AAt?$AAh?$AAr?$AAe?$AAa?$AAd?$AA?$CF?$AAX?$AA?6?$AA?$AN?$AA?$AA@ 10001794     com_mdd2:mdd.obj
 0001:000007bc       ??_C@_1DO@GDLJAKBF@?$AAE?$AAr?$AAr?$AAo?$AAr?$AA?5?$AAi?$AAn?$AAi?$AAt?$AAi?$AAa?$AAl?$AAi?$AAz?$AAi?$AAn?$AAg?$AA?5?$AAi?$AAn?$AAt?$AAe?$AAr?$AAr?$AAu?$AAp?$AAt?$AA?6?$AA?$AN?$AA?$AA@ 100017bc     com_mdd2:mdd.obj
 0001:00000800       ??_C@_1EI@EFCKMID@?$AAI?$AAn?$AAi?$AAt?$AAi?$AAa?$AAl?$AAi?$AAz?$AAi?$AAn?$AAg?$AA?5?$AAi?$AAn?$AAt?$AAe?$AAr?$AAr?$AAu?$AAp?$AAt?$AA?5?$AA0?$AAx?$AA?$CF?$AAX?$AA?0?$AA?5?$AA0?$AAx?$AA?$CF@ 10001800     com_mdd2:mdd.obj
 0001:00000848       ??_C@_1EE@NKOOKCAI@?$AAS?$AAe?$AAr?$AAi?$AAa?$AAl?$AAD?$AAi?$AAs?$AAp?$AAa?$AAt?$AAc?$AAh?$AAT?$AAh?$AAr?$AAe?$AAa?$AAd?$AA?5?$AA?$CF?$AAx?$AA?5?$AAe?$AAx?$AAi?$AAt?$AAi?$AAn?$AAg?$AA?$AN@ 10001848     com_mdd2:mdd.obj
 0001:0000088c       ??_C@_1BO@CNJNPPHP@?$AAE?$AAv?$AAe?$AAn?$AAt?$AA?5?$AA?$CF?$AAX?$AA?0?$AA?5?$AA?$CF?$AAd?$AA?$AN?$AA?6?$AA?$AA@ 1000188c     com_mdd2:mdd.obj
 0001:000008b0       ??_C@_1EI@IJEBFPL@?$AAS?$AAp?$AAi?$AAn?$AAn?$AAi?$AAn?$AAg?$AA?5?$AAi?$AAn?$AA?5?$AAd?$AAi?$AAs?$AAp?$AAa?$AAt?$AAc?$AAh?$AA?5?$AAt?$AAh?$AAr?$AAe?$AAa?$AAd?$AA?5?$AA?$CF?$AAX?$AA?5?$AA?$CF@ 100018b0     com_mdd2:mdd.obj
 0001:000008f8       ??_C@_1EE@JPBAFGIH@?$AAE?$AAn?$AAt?$AAe?$AAr?$AAe?$AAd?$AA?5?$AAS?$AAe?$AAr?$AAi?$AAa?$AAl?$AAD?$AAi?$AAs?$AAp?$AAa?$AAt?$AAc?$AAh?$AAT?$AAh?$AAr?$AAe?$AAa?$AAd?$AA?5?$AA?$CF?$AAX?$AA?$AN@ 100018f8     com_mdd2:mdd.obj
 0001:0000093c       ??_C@_1DM@NEFLPBFN@?$AA?$AN?$AA?6?$AAR?$AAe?$AAt?$AAu?$AAr?$AAn?$AAe?$AAd?$AA?5?$AAf?$AAr?$AAo?$AAm?$AA?5?$AAC?$AAl?$AAo?$AAs?$AAe?$AAH?$AAa?$AAn?$AAd?$AAl?$AAe?$AA?$AN?$AA?6?$AA?$AA@ 1000193c     com_mdd2:mdd.obj
 0001:00000978       ??_C@_1DO@BPPHAKCP@?$AA?$AN?$AA?6?$AAT?$AAr?$AAy?$AAi?$AAn?$AAg?$AA?5?$AAt?$AAo?$AA?5?$AAc?$AAa?$AAl?$AAl?$AA?5?$AAC?$AAl?$AAo?$AAs?$AAe?$AAH?$AAa?$AAn?$AAd?$AAl?$AAe?$AA?$AN?$AA?6?$AA?$AA@ 10001978     com_mdd2:mdd.obj
 0001:000009b8       ??_C@_1EI@FHNFOMPC@?$AA?$AN?$AA?6?$AAT?$AAr?$AAy?$AAi?$AAn?$AAg?$AA?5?$AAt?$AAo?$AA?5?$AAs?$AAi?$AAg?$AAn?$AAa?$AAl?$AA?5?$AAs?$AAe?$AAr?$AAi?$AAa?$AAl?$AA?5?$AAt?$AAh?$AAr?$AAe?$AAa?$AAd@ 100019b8     com_mdd2:mdd.obj
 0001:00000a00       ??_C@_1EI@JFKDHKHE@?$AA?$AN?$AA?6?$AAT?$AAr?$AAy?$AAi?$AAn?$AAg?$AA?5?$AAt?$AAo?$AA?5?$AAc?$AAl?$AAo?$AAs?$AAe?$AA?5?$AAd?$AAi?$AAs?$AAp?$AAa?$AAt?$AAc?$AAh?$AA?5?$AAt?$AAh?$AAr?$AAe?$AAa@ 10001a00     com_mdd2:mdd.obj
 0001:00000a48       ??_C@_1FE@DAKNODMA@?$AAI?$AAO?$AAC?$AAT?$AAL?$AA?3?$AAR?$AAT?$AAS?$AA_?$AAC?$AAO?$AAN?$AAT?$AAR?$AAO?$AAL?$AA_?$AAH?$AAA?$AAN?$AAD?$AAS?$AAH?$AAA?$AAK?$AAE?$AA?5?$AAS?$AAe?$AAt?$AAt@ 10001a48     com_mdd2:mdd.obj
 0001:00000aa0       ??_C@_1FG@IDPAINNF@?$AAI?$AAO?$AAC?$AAT?$AAL?$AA?3?$AAR?$AAT?$AAS?$AA_?$AAC?$AAO?$AAN?$AAT?$AAR?$AAO?$AAL?$AA_?$AAH?$AAA?$AAN?$AAD?$AAS?$AAH?$AAA?$AAK?$AAE?$AA?5?$AAC?$AAl?$AAe?$AAa@ 10001aa0     com_mdd2:mdd.obj
 0001:00000af8       ??_C@_1FE@MINNMIFE@?$AAI?$AAO?$AAC?$AAT?$AAL?$AA?3?$AAD?$AAT?$AAR?$AA_?$AAC?$AAO?$AAN?$AAT?$AAR?$AAO?$AAL?$AA_?$AAH?$AAA?$AAN?$AAD?$AAS?$AAH?$AAA?$AAK?$AAE?$AA?5?$AAS?$AAe?$AAt?$AAt@ 10001af8     com_mdd2:mdd.obj
 0001:00000b50       ??_C@_1FG@GEFMJHJN@?$AAI?$AAO?$AAC?$AAT?$AAL?$AA?3?$AAD?$AAT?$AAR?$AA_?$AAC?$AAO?$AAN?$AAT?$AAR?$AAO?$AAL?$AA_?$AAH?$AAA?$AAN?$AAD?$AAS?$AAH?$AAA?$AAK?$AAE?$AA?5?$AAC?$AAl?$AAe?$AAa@ 10001b50     com_mdd2:mdd.obj
 0001:00000ba8       ??_C@_1BI@NFEFLGML@?$AA?9?$AAC?$AAO?$AAM?$AA_?$AAI?$AAn?$AAi?$AAt?$AA?$AN?$AA?6?$AA?$AA@ 10001ba8     com_mdd2:mdd.obj
 0001:00000bc0       ??_C@_1EI@FNCKFJMM@?$AAR?$AAx?$AAB?$AAu?$AAf?$AAf?$AAe?$AAr?$AA?5?$AAi?$AAn?$AAi?$AAt?$AA?8?$AAe?$AAd?$AA?5?$AAw?$AAi?$AAt?$AAh?$AA?5?$AAs?$AAt?$AAa?$AAr?$AAt?$AA?5?$AAa?$AAt?$AA?5?$AA?$CF@ 10001bc0     com_mdd2:mdd.obj
 0001:00000c08       ??_C@_1CC@POKINGEF@?$AAR?$AAx?$AAH?$AAe?$AAa?$AAd?$AA?5?$AAi?$AAn?$AAi?$AAt?$AA?8?$AAe?$AAd?$AA?$AN?$AA?6?$AA?$AA@ 10001c08     com_mdd2:mdd.obj
 0001:00000c30       ??_C@_1GG@FCOIFIDD@?$AAE?$AAr?$AAr?$AAo?$AAr?$AA?5?$AAa?$AAl?$AAl?$AAo?$AAc?$AAa?$AAt?$AAi?$AAn?$AAg?$AA?5?$AAr?$AAe?$AAc?$AAe?$AAi?$AAv?$AAe?$AA?5?$AAb?$AAu?$AAf?$AAf?$AAe?$AAr?$AA?0@ 10001c30     com_mdd2:mdd.obj
 0001:00000c98       ??_C@_1DE@CLLKJMN@?$AAB?$AAa?$AAc?$AAk?$AA?5?$AAf?$AAr?$AAo?$AAm?$AA?5?$AAh?$AAa?$AAr?$AAd?$AAw?$AAa?$AAr?$AAe?$AA?5?$AAi?$AAn?$AAi?$AAt?$AA?$AN?$AA?6?$AA?$AA@ 10001c98     com_mdd2:mdd.obj
 0001:00000cd0       ??_C@_1GG@LFOFGOL@?$AAH?$AAa?$AAr?$AAd?$AAw?$AAa?$AAr?$AAe?$AA?5?$AAd?$AAo?$AAe?$AAs?$AAn?$AA?8?$AAt?$AA?5?$AAi?$AAn?$AAi?$AAt?$AA?5?$AAc?$AAo?$AAr?$AAr?$AAe?$AAc?$AAt?$AAl?$AAy?$AA?0@ 10001cd0     com_mdd2:mdd.obj
 0001:00000d38       ??_C@_1EA@DFMKFADA@?$AAA?$AAb?$AAo?$AAu?$AAt?$AA?5?$AAt?$AAo?$AA?5?$AAc?$AAa?$AAl?$AAl?$AA?5?$AAH?$AAW?$AAI?$AAn?$AAi?$AAt?$AA?$CI?$AA?$CF?$AAs?$AA?0?$AA0?$AAx?$AA?$CF?$AAX?$AA?$CJ?$AA?$AN?$AA?6?$AA?$AA@ 10001d38     com_mdd2:mdd.obj
 0001:00000d78       ??_C@_1FI@OHFMJBNJ@?$AAE?$AAr?$AAr?$AAo?$AAr?$AA?5?$AAi?$AAn?$AA?5?$AAG?$AAe?$AAt?$AAS?$AAe?$AAr?$AAi?$AAa?$AAl?$AAO?$AAb?$AAj?$AAe?$AAc?$AAt?$AA?0?$AA?5?$AAC?$AAO?$AAM?$AA_?$AAI?$AAn@ 10001d78     com_mdd2:mdd.obj
 0001:00000dd0       ??_C@_1BM@EFMMMFDH@?$AAD?$AAe?$AAv?$AAI?$AAn?$AAd?$AAe?$AAx?$AA?5?$AA?$CF?$AAX?$AA?$AN?$AA?6?$AA?$AA@ 10001dd0     com_mdd2:mdd.obj
 0001:00000df0       ??_C@_1GI@IGAGBKDE@?$AAF?$AAa?$AAi?$AAl?$AAe?$AAd?$AA?5?$AAt?$AAo?$AA?5?$AAg?$AAe?$AAt?$AA?5?$AAP?$AAr?$AAi?$AAo?$AAr?$AAi?$AAt?$AAy?$AA2?$AA5?$AA6?$AA?5?$AAv?$AAa?$AAl?$AAu?$AAe?$AA?0@ 10001df0     com_mdd2:mdd.obj
 0001:00000e58       ??_C@_1BI@BHLBGEOK@?$AAP?$AAr?$AAi?$AAo?$AAr?$AAi?$AAt?$AAy?$AA2?$AA5?$AA6?$AA?$AA@ 10001e58     com_mdd2:mdd.obj
 0001:00000e70       ??_C@_1HA@FDKKDCHL@?$AAF?$AAa?$AAi?$AAl?$AAe?$AAd?$AA?5?$AAt?$AAo?$AA?5?$AAg?$AAe?$AAt?$AA?5?$AAD?$AAe?$AAv?$AAi?$AAc?$AAe?$AAA?$AAr?$AAr?$AAa?$AAy?$AAI?$AAn?$AAd?$AAe?$AAx?$AA?5?$AAv@ 10001e70     com_mdd2:mdd.obj
 0001:00000ee0       ??_C@_1CC@KMPFMANC@?$AAD?$AAe?$AAv?$AAi?$AAc?$AAe?$AAA?$AAr?$AAr?$AAa?$AAy?$AAI?$AAn?$AAd?$AAe?$AAx?$AA?$AA@ 10001ee0     com_mdd2:mdd.obj
 0001:00000f08       ??_C@_1FK@GNPHIAEF@?$AAF?$AAa?$AAi?$AAl?$AAe?$AAd?$AA?5?$AAt?$AAo?$AA?5?$AAo?$AAp?$AAe?$AAn?$AA?5?$AAd?$AAe?$AAv?$AAk?$AAe?$AAy?$AAp?$AAa?$AAt?$AAh?$AA?0?$AA?5?$AAC?$AAO?$AAM?$AA_?$AAI@ 10001f08     com_mdd2:mdd.obj
 0001:00000f64       ??_C@_1CC@OIKDCOFG@?$AAT?$AAr?$AAy?$AA?5?$AAt?$AAo?$AA?5?$AAo?$AAp?$AAe?$AAn?$AA?5?$AA?$CF?$AAs?$AA?$AN?$AA?6?$AA?$AA@ 10001f64     com_mdd2:mdd.obj
 0001:00000f88       ??_C@_1FA@BECDDKGM@?$AAE?$AAr?$AAr?$AAo?$AAr?$AA?5?$AAc?$AAr?$AAe?$AAa?$AAt?$AAi?$AAn?$AAg?$AA?5?$AAe?$AAv?$AAe?$AAn?$AAt?$AA?0?$AA?5?$AAC?$AAO?$AAM?$AA_?$AAI?$AAn?$AAi?$AAt?$AA?5?$AAf@ 10001f88     com_mdd2:mdd.obj
 0001:00000fd8       ??_C@_1HG@FCOJGPAE@?$AAE?$AAr?$AAr?$AAo?$AAr?$AA?5?$AAa?$AAl?$AAl?$AAo?$AAc?$AAa?$AAt?$AAi?$AAn?$AAg?$AA?5?$AAm?$AAe?$AAm?$AAo?$AAr?$AAy?$AA?5?$AAf?$AAo?$AAr?$AA?5?$AAp?$AAS?$AAe?$AAr@ 10001fd8     com_mdd2:mdd.obj
 0001:00001050       ??_C@_1EK@DLAABGLF@?$AAI?$AAn?$AAv?$AAa?$AAl?$AAi?$AAd?$AA?5?$AAP?$AAa?$AAr?$AAa?$AAm?$AAe?$AAt?$AAe?$AAr?$AA?0?$AA?5?$AAC?$AAO?$AAM?$AA_?$AAI?$AAn?$AAi?$AAt?$AA?5?$AAf?$AAa?$AAi?$AAl@ 10002050     com_mdd2:mdd.obj
 0001:0000109c       ??_C@_1BI@GFHIOEJL@?$AA?$CL?$AAC?$AAO?$AAM?$AA_?$AAI?$AAn?$AAi?$AAt?$AA?$AN?$AA?6?$AA?$AA@ 1000209c     com_mdd2:mdd.obj
 0001:000010b4       ??_C@_1CE@HHPKLFBI@?$AAH?$AAW?$AA?5?$AAO?$AAp?$AAe?$AAn?$AA?5?$AAf?$AAa?$AAi?$AAl?$AAe?$AAd?$AA?4?$AA?$AN?$AA?6?$AA?$AA@ 100020b4     com_mdd2:mdd.obj
 0001:000010d8       ??_C@_1FG@FDKJAEDJ@?$AAC?$AAO?$AAM?$AA_?$AAO?$AAp?$AAe?$AAn?$AA?3?$AA?5?$AAF?$AAa?$AAi?$AAl?$AAe?$AAd?$AA?5?$AAS?$AAt?$AAa?$AAr?$AAt?$AAD?$AAi?$AAs?$AAp?$AAa?$AAt?$AAc?$AAh?$AAT?$AAh@ 100020d8     com_mdd2:mdd.obj
 0001:00001130       ??_C@_1FA@GFAOJBEN@?$AAC?$AAO?$AAM?$AA_?$AAO?$AAp?$AAe?$AAn?$AA?3?$AA?5?$AAS?$AAt?$AAa?$AAr?$AAt?$AAi?$AAn?$AAg?$AA?5?$AAD?$AAi?$AAs?$AAp?$AAa?$AAt?$AAc?$AAh?$AAT?$AAh?$AAr?$AAe?$AAa@ 10002130     com_mdd2:mdd.obj
 0001:00001180       ??_C@_1EK@MCEDHMPN@?$AAC?$AAO?$AAM?$AA_?$AAO?$AAp?$AAe?$AAn?$AA?3?$AA?5?$AAF?$AAi?$AAr?$AAs?$AAt?$AA?5?$AAo?$AAp?$AAe?$AAn?$AA?5?$AA?3?$AA?5?$AAD?$AAo?$AA?5?$AAI?$AAn?$AAi?$AAt?$AA?5?$AAx@ 10002180     com_mdd2:mdd.obj
 0001:000011d0       ??_C@_1EK@MFLOMJPC@?$AA?9?$AAC?$AAO?$AAM?$AA_?$AAO?$AAp?$AAe?$AAn?$AA?5?$AAh?$AAa?$AAn?$AAd?$AAl?$AAe?$AA?5?$AAx?$AA?$CF?$AAX?$AA?0?$AA?5?$AAx?$AA?$CF?$AAX?$AA?0?$AA?5?$AAR?$AAe?$AAf?$AA?5?$AAx@ 100021d0     com_mdd2:mdd.obj
 0001:00001220       ??_C@_1GC@CLBBDJNN@?$AAC?$AAO?$AAM?$AA_?$AAO?$AAp?$AAe?$AAn?$AA?3?$AA?5?$AAA?$AAc?$AAc?$AAe?$AAs?$AAs?$AA?5?$AAp?$AAe?$AAr?$AAm?$AAi?$AAs?$AAs?$AAi?$AAo?$AAn?$AA?5?$AAh?$AAa?$AAn?$AAd@ 10002220     com_mdd2:mdd.obj
 0001:00001288       ??_C@_1HC@GGJLMGKF@?$AAE?$AAr?$AAr?$AAo?$AAr?$AA?5?$AAa?$AAl?$AAl?$AAo?$AAc?$AAa?$AAt?$AAi?$AAn?$AAg?$AA?5?$AAm?$AAe?$AAm?$AAo?$AAr?$AAy?$AA?5?$AAf?$AAo?$AAr?$AA?5?$AAp?$AAO?$AAp?$AAe@ 10002288     com_mdd2:mdd.obj
 0001:00001300       ??_C@_1HA@GJBLLAJC@?$AAO?$AAp?$AAe?$AAn?$AA?5?$AAr?$AAe?$AAq?$AAu?$AAe?$AAs?$AAt?$AAe?$AAd?$AA?5?$AAa?$AAc?$AAc?$AAe?$AAs?$AAs?$AA?5?$AA?$CF?$AAx?$AA?0?$AA?5?$AAh?$AAa?$AAn?$AAd?$AAl?$AAe@ 10002300     com_mdd2:mdd.obj
 0001:00001370       ??_C@_1EK@IHGIHNNE@?$AAO?$AAp?$AAe?$AAn?$AA?5?$AAa?$AAt?$AAt?$AAe?$AAm?$AAp?$AAt?$AAe?$AAd?$AA?5?$AAo?$AAn?$AA?5?$AAu?$AAn?$AAi?$AAn?$AAi?$AAt?$AAe?$AAd?$AA?5?$AAd?$AAe?$AAv?$AAi?$AAc@ 10002370     com_mdd2:mdd.obj
 0001:000013c0       ??_C@_1FM@OGLFDPL@?$AA?$CL?$AAC?$AAO?$AAM?$AA_?$AAO?$AAp?$AAe?$AAn?$AA?5?$AAh?$AAa?$AAn?$AAd?$AAl?$AAe?$AA?5?$AAx?$AA?$CF?$AAX?$AA?0?$AA?5?$AAa?$AAc?$AAc?$AAe?$AAs?$AAs?$AA?5?$AAx?$AA?$CF?$AAX@ 100023c0     com_mdd2:mdd.obj
 0001:00001420       ??_C@_1FK@FNONLNGN@?$AA?$CF?$AAs?$AA?3?$AA?5?$AAD?$AAE?$AAB?$AAU?$AAG?$AAC?$AAH?$AAK?$AA?5?$AAf?$AAa?$AAi?$AAl?$AAe?$AAd?$AA?5?$AAi?$AAn?$AA?5?$AAf?$AAi?$AAl?$AAe?$AA?5?$AA?$CF?$AAs?$AA?5?$AAa@ 10002420     com_mdd2:mdd.obj
 0001:0000147c       ??_C@_1BA@LEPJIIOK@?$AAU?$AAn?$AAk?$AAn?$AAo?$AAw?$AAn?$AA?$AA@ 1000247c     com_mdd2:mdd.obj
 0001:00001490       ??_C@_1FO@FLGHDMHK@?$AAd?$AA?3?$AA?2?$AAc?$AAh?$AAe?$AAl?$AAa?$AAn?$AAr?$AAt?$AAm?$AA2?$AA?2?$AAp?$AAu?$AAb?$AAl?$AAi?$AAc?$AA?2?$AAc?$AAo?$AAm?$AAm?$AAo?$AAn?$AA?2?$AAs?$AAd?$AAk?$AA?2@ 10002490     com_mdd2:mdd.obj
 0001:000014f0       ??_C@_1CA@KJOIAGGH@?$AA?9?$AAC?$AAO?$AAM?$AA_?$AAP?$AAr?$AAe?$AAC?$AAl?$AAo?$AAs?$AAe?$AA?$AN?$AA?6?$AA?$AA@ 100024f0     com_mdd2:mdd.obj
 0001:00001510       ??_C@_1EK@NAJGEFLJ@?$AA?$CB?$AA?$CB?$AAP?$AAr?$AAe?$AAC?$AAl?$AAo?$AAs?$AAe?$AA?5?$AAo?$AAf?$AA?5?$AAn?$AAo?$AAn?$AA?9?$AAo?$AAp?$AAe?$AAn?$AA?5?$AAs?$AAe?$AAr?$AAi?$AAa?$AAl?$AA?5?$AAp?$AAo@ 10002510     com_mdd2:mdd.obj
 0001:00001560       ??_C@_1FM@KBMCIDEH@?$AAC?$AAO?$AAM?$AA_?$AAP?$AAr?$AAe?$AAC?$AAl?$AAo?$AAs?$AAe?$AA?3?$AA?5?$AAs?$AAe?$AAr?$AAi?$AAa?$AAl?$AA?5?$AAu?$AAs?$AAe?$AAr?$AAs?$AA?5?$AAt?$AAo?$AA?5?$AAe?$AAx@ 10002560     com_mdd2:mdd.obj
 0001:000015c0       ??_C@_1FE@NPNGHGCB@?$AAC?$AAO?$AAM?$AA_?$AAP?$AAr?$AAe?$AAC?$AAl?$AAo?$AAs?$AAe?$AA?3?$AA?5?$AA?$CF?$AAd?$AA?5?$AAu?$AAs?$AAe?$AAr?$AAs?$AA?5?$AAi?$AAn?$AA?5?$AAM?$AAD?$AAD?$AA?5?$AAf?$AAu@ 100025c0     com_mdd2:mdd.obj
 0001:00001618       ??_C@_1FA@EDDADDPP@?$AA?$CB?$AA?$CB?$AAC?$AAO?$AAM?$AA_?$AAP?$AAr?$AAe?$AAC?$AAl?$AAo?$AAs?$AAe?$AA?3?$AA?5?$AAp?$AAS?$AAe?$AAr?$AAi?$AAa?$AAl?$AAH?$AAe?$AAa?$AAd?$AA?5?$AA?$DN?$AA?$DN?$AA?5?$AAN@ 10002618     com_mdd2:mdd.obj
 0001:00001668       ??_C@_1BK@GDIGGGLD@?$AA?9?$AAC?$AAO?$AAM?$AA_?$AAC?$AAl?$AAo?$AAs?$AAe?$AA?$AN?$AA?6?$AA?$AA@ 10002668     com_mdd2:mdd.obj
 0001:00001688       ??_C@_1EE@HJGCIAAB@?$AA?$CB?$AA?$CB?$AAC?$AAl?$AAo?$AAs?$AAe?$AA?5?$AAo?$AAf?$AA?5?$AAn?$AAo?$AAn?$AA?9?$AAo?$AAp?$AAe?$AAn?$AA?5?$AAs?$AAe?$AAr?$AAi?$AAa?$AAl?$AA?5?$AAp?$AAo?$AAr?$AAt?$AA?$AN@ 10002688     com_mdd2:mdd.obj
 0001:000016d0       ??_C@_1FA@FDHIAIFB@?$AAC?$AAO?$AAM?$AA_?$AAC?$AAl?$AAo?$AAs?$AAe?$AA?3?$AA?5?$AAC?$AAl?$AAo?$AAs?$AAe?$AAd?$AA?5?$AAa?$AAc?$AAc?$AAe?$AAs?$AAs?$AA?5?$AAo?$AAw?$AAn?$AAe?$AAr?$AA?5?$AAh@ 100026d0     com_mdd2:mdd.obj
 0001:00001720       ??_C@_1EO@KHAJIML@?$AAC?$AAO?$AAM?$AA_?$AAC?$AAl?$AAo?$AAs?$AAe?$AA?5?$AA?3?$AA?5?$AAS?$AAt?$AAo?$AAp?$AAp?$AAi?$AAn?$AAg?$AA?5?$AAD?$AAi?$AAs?$AAp?$AAa?$AAt?$AAc?$AAh?$AA?5?$AAT?$AAh@ 10002720     com_mdd2:mdd.obj
 0001:00001770       ??_C@_1DA@HIJABIAN@?$AAR?$AAe?$AAt?$AAu?$AAr?$AAn?$AAe?$AAd?$AA?5?$AAf?$AAr?$AAo?$AAm?$AA?5?$AAH?$AAW?$AAC?$AAl?$AAo?$AAs?$AAe?$AA?$AN?$AA?6?$AA?$AA@ 10002770     com_mdd2:mdd.obj
 0001:000017a0       ??_C@_1DA@EPLPIONK@?$AAA?$AAb?$AAo?$AAu?$AAt?$AA?5?$AAt?$AAo?$AA?5?$AAc?$AAa?$AAl?$AAl?$AA?5?$AAH?$AAW?$AAC?$AAl?$AAo?$AAs?$AAe?$AA?$AN?$AA?6?$AA?$AA@ 100027a0     com_mdd2:mdd.obj
 0001:000017d0       ??_C@_1JK@JHJOGNCH@?$AAC?$AAO?$AAM?$AA_?$AAC?$AAl?$AAo?$AAs?$AAe?$AA?3?$AA?5?$AA?$CI?$AA?$CF?$AAd?$AA?5?$AAh?$AAa?$AAn?$AAd?$AAl?$AAe?$AAs?$AA?$CJ?$AA?5?$AAt?$AAo?$AAt?$AAa?$AAl?$AA?5?$AAR?$AAX@ 100027d0     com_mdd2:mdd.obj
 0001:00001870       ??_C@_1EK@JBKGBIGA@?$AA?$CB?$AA?$CB?$AAC?$AAO?$AAM?$AA_?$AAC?$AAl?$AAo?$AAs?$AAe?$AA?3?$AA?5?$AAp?$AAS?$AAe?$AAr?$AAi?$AAa?$AAl?$AAH?$AAe?$AAa?$AAd?$AA?5?$AA?$DN?$AA?$DN?$AA?5?$AAN?$AAU?$AAL?$AAL@ 10002870     com_mdd2:mdd.obj
 0001:000018bc       ??_C@_1BK@FMFILLAC@?$AA?$CL?$AAC?$AAO?$AAM?$AA_?$AAC?$AAl?$AAo?$AAs?$AAe?$AA?$AN?$AA?6?$AA?$AA@ 100028bc     com_mdd2:mdd.obj
 0001:000018d8       ??_C@_1CE@KKIBLMOF@?$AA?9?$AAP?$AAr?$AAo?$AAc?$AAe?$AAs?$AAs?$AAE?$AAx?$AAi?$AAt?$AAi?$AAn?$AAg?$AA?$AN?$AA?6?$AA?$AA@ 100028d8     com_mdd2:mdd.obj
 0001:00001900       ??_C@_1FE@DFEILEFJ@?$AA?$CB?$AA?$CB?$AAP?$AAr?$AAo?$AAc?$AAe?$AAs?$AAs?$AAE?$AAx?$AAi?$AAt?$AAi?$AAn?$AAg?$AA?3?$AA?5?$AAp?$AAS?$AAe?$AAr?$AAi?$AAa?$AAl?$AAH?$AAe?$AAa?$AAd?$AA?5?$AA?$DN?$AA?$DN@ 10002900     com_mdd2:mdd.obj
 0001:00001954       ??_C@_1CE@GDEBELBJ@?$AA?$CL?$AAP?$AAr?$AAo?$AAc?$AAe?$AAs?$AAs?$AAE?$AAx?$AAi?$AAt?$AAi?$AAn?$AAg?$AA?$AN?$AA?6?$AA?$AA@ 10002954     com_mdd2:mdd.obj
 0001:00001978       ??_C@_1CC@EOGEOIEK@?$AA?9?$AAC?$AAO?$AAM?$AA_?$AAP?$AAr?$AAe?$AAD?$AAe?$AAi?$AAn?$AAi?$AAt?$AA?$AN?$AA?6?$AA?$AA@ 10002978     com_mdd2:mdd.obj
 0001:0000199c       ??_C@_1DI@PDPAMALM@?$AAR?$AAe?$AAt?$AAu?$AAr?$AAn?$AAe?$AAd?$AA?5?$AAf?$AAr?$AAo?$AAm?$AA?5?$AAH?$AAW?$AAP?$AAr?$AAe?$AAD?$AAe?$AAi?$AAn?$AAi?$AAt?$AA?$AN?$AA?6?$AA?$AA@ 1000299c     com_mdd2:mdd.obj
 0001:000019d4       ??_C@_1DI@JGMLCPMK@?$AAA?$AAb?$AAo?$AAu?$AAt?$AA?5?$AAt?$AAo?$AA?5?$AAc?$AAa?$AAl?$AAl?$AA?5?$AAH?$AAW?$AAP?$AAr?$AAe?$AAD?$AAe?$AAi?$AAn?$AAi?$AAt?$AA?$AN?$AA?6?$AA?$AA@ 100029d4     com_mdd2:mdd.obj
 0001:00001a10       ??_C@_1EM@KLLBGOIP@?$AA?5?$AAP?$AAr?$AAe?$AAD?$AAe?$AAi?$AAn?$AAi?$AAt?$AA?5?$AA?9?$AAP?$AAr?$AAe?$AA?5?$AAC?$AAl?$AAo?$AAs?$AAi?$AAn?$AAg?$AA?5?$AAH?$AAa?$AAn?$AAd?$AAl?$AAe?$AA?5?$AA0@ 10002a10     com_mdd2:mdd.obj
 0001:00001a60       ??_C@_1EO@HNCGHLKP@?$AAC?$AAO?$AAM?$AA_?$AAP?$AAr?$AAe?$AAD?$AAe?$AAi?$AAn?$AAi?$AAt?$AA?5?$AAc?$AAa?$AAn?$AA?8?$AAt?$AA?5?$AAf?$AAi?$AAn?$AAd?$AA?5?$AAp?$AAS?$AAe?$AAr?$AAi?$AAa?$AAl@ 10002a60     com_mdd2:mdd.obj
 0001:00001ab0       ??_C@_1CC@JFGJAOPO@?$AA?$CL?$AAC?$AAO?$AAM?$AA_?$AAP?$AAr?$AAe?$AAD?$AAe?$AAi?$AAn?$AAi?$AAt?$AA?$AN?$AA?6?$AA?$AA@ 10002ab0     com_mdd2:mdd.obj
 0001:00001ad4       ??_C@_1BM@OGICEDGH@?$AA?9?$AAC?$AAO?$AAM?$AA_?$AAD?$AAe?$AAi?$AAn?$AAi?$AAt?$AA?$AN?$AA?6?$AA?$AA@ 10002ad4     com_mdd2:mdd.obj
 0001:00001af0       ??_C@_1DC@CLHJIHHM@?$AAR?$AAe?$AAt?$AAu?$AAr?$AAn?$AAe?$AAd?$AA?5?$AAf?$AAr?$AAo?$AAm?$AA?5?$AAH?$AAW?$AAD?$AAe?$AAi?$AAn?$AAi?$AAt?$AA?$AN?$AA?6?$AA?$AA@ 10002af0     com_mdd2:mdd.obj
 0001:00001b24       ??_C@_1DC@PMGMNFPK@?$AAA?$AAb?$AAo?$AAu?$AAt?$AA?5?$AAt?$AAo?$AA?5?$AAc?$AAa?$AAl?$AAl?$AA?5?$AAH?$AAW?$AAD?$AAe?$AAi?$AAn?$AAi?$AAt?$AA?$AN?$AA?6?$AA?$AA@ 10002b24     com_mdd2:mdd.obj
 0001:00001b58       ??_C@_1EA@JDMAPCPA@?$AA?5?$AAD?$AAe?$AAi?$AAn?$AAi?$AAt?$AA?5?$AA?9?$AA?5?$AAC?$AAl?$AAo?$AAs?$AAi?$AAn?$AAg?$AA?5?$AAH?$AAa?$AAn?$AAd?$AAl?$AAe?$AA?5?$AA0?$AAx?$AA?$CF?$AAX?$AA?$AN?$AA?6?$AA?$AA@ 10002b58     com_mdd2:mdd.obj
 0001:00001b98       ??_C@_1EI@FADDJAGG@?$AAC?$AAO?$AAM?$AA_?$AAD?$AAe?$AAi?$AAn?$AAi?$AAt?$AA?5?$AAc?$AAa?$AAn?$AA?8?$AAt?$AA?5?$AAf?$AAi?$AAn?$AAd?$AA?5?$AAp?$AAS?$AAe?$AAr?$AAi?$AAa?$AAl?$AAH?$AAe?$AAa@ 10002b98     com_mdd2:mdd.obj
 0001:00001be0       ??_C@_1BM@ODDOENCJ@?$AA?$CL?$AAC?$AAO?$AAM?$AA_?$AAD?$AAe?$AAi?$AAn?$AAi?$AAt?$AA?$AN?$AA?6?$AA?$AA@ 10002be0     com_mdd2:mdd.obj
 0001:00001c00       ??_C@_1GI@KJLFCJIJ@?$AA?9?$AAC?$AAO?$AAM?$AA_?$AAR?$AAE?$AAA?$AAD?$AA?3?$AA?5?$AAr?$AAe?$AAt?$AAu?$AAr?$AAn?$AAi?$AAn?$AAg?$AA?5?$AA?$CF?$AAd?$AA?5?$AA?$CI?$AAt?$AAo?$AAt?$AAa?$AAl?$AA?5?$AA?$CF@ 10002c00     com_mdd2:mdd.obj
 0001:00001c68       ??_C@_1CO@BMKNIMFL@?$AAR?$AAe?$AAc?$AAe?$AAi?$AAv?$AAe?$AAB?$AAy?$AAt?$AAe?$AAs?$AA?5?$AAe?$AAx?$AAi?$AAt?$AAi?$AAn?$AAg?$AA?$AN?$AA?6?$AA?$AA@ 10002c68     com_mdd2:mdd.obj
 0001:00001c98       ??_C@_1EI@NJBLBAI@?$AAD?$AAT?$AAR?$AA_?$AAC?$AAO?$AAN?$AAT?$AAR?$AAO?$AAL?$AA_?$AAH?$AAA?$AAN?$AAD?$AAS?$AAH?$AAA?$AAK?$AAE?$AA?5?$AAS?$AAe?$AAt?$AAt?$AAi?$AAn?$AAg?$AA?5?$AAD?$AAT@ 10002c98     com_mdd2:mdd.obj
 0001:00001ce0       ??_C@_1EI@PFOBJKJM@?$AAR?$AAT?$AAS?$AA_?$AAC?$AAO?$AAN?$AAT?$AAR?$AAO?$AAL?$AA_?$AAH?$AAA?$AAN?$AAD?$AAS?$AAH?$AAA?$AAK?$AAE?$AA?5?$AAS?$AAe?$AAt?$AAt?$AAi?$AAn?$AAg?$AA?5?$AAR?$AAT@ 10002ce0     com_mdd2:mdd.obj
 0001:00001d28       ??_C@_1BM@LDMNCPPP@?$AAS?$AAe?$AAn?$AAd?$AAi?$AAn?$AAg?$AA?5?$AAX?$AAO?$AAN?$AA?$AN?$AA?6?$AA?$AA@ 10002d28     com_mdd2:mdd.obj
 0001:00001d44       ??_C@_1DO@LAJCOFEP@?$AAC?$AAO?$AAM?$AA_?$AAR?$AAe?$AAa?$AAd?$AA?5?$AA?9?$AA?5?$AAd?$AAe?$AAv?$AAi?$AAc?$AAe?$AA?5?$AAw?$AAa?$AAs?$AA?5?$AAc?$AAl?$AAo?$AAs?$AAe?$AAd?$AA?6?$AA?$AN?$AA?$AA@ 10002d44     com_mdd2:mdd.obj
 0001:00001d84       ??_C@_1DG@NGGANINM@?$AAC?$AAO?$AAM?$AA_?$AAR?$AAe?$AAa?$AAd?$AA?5?$AA?9?$AA?5?$AAA?$AAb?$AAo?$AAr?$AAt?$AAi?$AAn?$AAg?$AA?5?$AAr?$AAe?$AAa?$AAd?$AA?$AN?$AA?6?$AA?$AA@ 10002d84     com_mdd2:mdd.obj
 0001:00001dbc       ??_C@_1CK@GLIEOMOP@?$AAA?$AAb?$AAo?$AAu?$AAt?$AA?5?$AAt?$AAo?$AA?5?$AAw?$AAa?$AAi?$AAt?$AA?5?$AA?$CF?$AAd?$AAm?$AAs?$AA?$AN?$AA?6?$AA?$AA@ 10002dbc     com_mdd2:mdd.obj
 0001:00001de8       ??_C@_1FC@CGIHBGNN@?$AAT?$AAo?$AAp?$AA?5?$AAo?$AAf?$AA?5?$AAL?$AAo?$AAo?$AAp?$AA?5?$AAF?$AAi?$AAf?$AAo?$AA?$CI?$AAR?$AA?$DN?$AA?$CF?$AAd?$AA?0?$AAW?$AA?$DN?$AA?$CF?$AAd?$AA?0?$AAL?$AA?$DN?$AA?$CF?$AAd?$AA?0@ 10002de8     com_mdd2:mdd.obj
 0001:00001e3c       ??_C@_1CE@PICJNKFA@?$AAT?$AAo?$AAt?$AAa?$AAl?$AAT?$AAi?$AAm?$AAe?$AAo?$AAu?$AAt?$AA?3?$AA?$CF?$AAd?$AA?$AN?$AA?6?$AA?$AA@ 10002e3c     com_mdd2:mdd.obj
 0001:00001e60       ??_C@_1FO@KCNFPNI@?$AAC?$AAO?$AAM?$AA_?$AAR?$AAE?$AAA?$AAD?$AA?0?$AA?5?$AAb?$AAa?$AAd?$AA?5?$AA?5?$AAp?$AAo?$AAi?$AAn?$AAt?$AAe?$AAr?$AA?$CI?$AA0?$AAx?$AA?$CF?$AAx?$AA?$CJ?$AA?5?$AAo?$AAr?$AA?5@ 10002e60     com_mdd2:mdd.obj
 0001:00001ec0       ??_C@_1FE@BNFDNPPG@?$AAC?$AAO?$AAM?$AA_?$AAR?$AAe?$AAa?$AAd?$AA?3?$AA?5?$AAA?$AAc?$AAc?$AAe?$AAs?$AAs?$AA?5?$AAp?$AAe?$AAr?$AAm?$AAi?$AAs?$AAs?$AAi?$AAo?$AAn?$AA?5?$AAf?$AAa?$AAi?$AAl@ 10002ec0     com_mdd2:mdd.obj
 0001:00001f14       ??_C@_1DI@CKPKPEIH@?$AAC?$AAO?$AAM?$AA_?$AAR?$AAE?$AAA?$AAD?$AA?0?$AA?5?$AAd?$AAe?$AAv?$AAi?$AAc?$AAe?$AA?5?$AAn?$AAo?$AAt?$AA?5?$AAo?$AAp?$AAe?$AAn?$AA?$AN?$AA?6?$AA?$AA@ 10002f14     com_mdd2:mdd.obj
 0001:00001f4c       ??_C@_1DC@DDENEIPK@?$AAC?$AAO?$AAM?$AA_?$AAR?$AAE?$AAA?$AAD?$AA?0?$AA?5?$AAW?$AAr?$AAo?$AAn?$AAg?$AA?5?$AAH?$AAa?$AAn?$AAd?$AAl?$AAe?$AA?$AN?$AA?6?$AA?$AA@ 10002f4c     com_mdd2:mdd.obj
 0001:00001f80       ??_C@_1DE@HFOANDEN@?$AA?$CL?$AAC?$AAO?$AAM?$AA_?$AAR?$AAE?$AAA?$AAD?$AA?$CI?$AA0?$AAx?$AA?$CF?$AAX?$AA?0?$AA0?$AAx?$AA?$CF?$AAX?$AA?0?$AA?$CF?$AAd?$AA?$CJ?$AA?$AN?$AA?6?$AA?$AA@ 10002f80     com_mdd2:mdd.obj
 0001:00001fb4       ??_C@_1DG@PKENKCNO@?$AA?9?$AAC?$AAO?$AAM?$AA_?$AAW?$AAR?$AAI?$AAT?$AAE?$AA?0?$AA?5?$AAr?$AAe?$AAt?$AAu?$AAr?$AAn?$AAi?$AAn?$AAg?$AA?5?$AA?$CF?$AAd?$AA?6?$AA?$AN?$AA?$AA@ 10002fb4     com_mdd2:mdd.obj
 0001:00001ff0       ??_C@_1FE@LGJDMHNB@?$AAC?$AAO?$AAM?$AA_?$AAW?$AAr?$AAi?$AAt?$AAe?$AA?5?$AAr?$AAe?$AAl?$AAe?$AAa?$AAs?$AAe?$AAd?$AA?5?$AAC?$AAr?$AAi?$AAt?$AAS?$AAe?$AAc?$AA?3?$AA?5?$AA?$CF?$AAx?$AA?4?$AA?5@ 10002ff0     com_mdd2:mdd.obj
 0001:00002048       ??_C@_1EA@JFKAOONE@?$AAC?$AAO?$AAM?$AA_?$AAW?$AAr?$AAi?$AAt?$AAe?$AA?5?$AAc?$AAo?$AAm?$AAp?$AAl?$AAe?$AAt?$AAe?$AAd?$AA?5?$AAn?$AAo?$AAr?$AAm?$AAa?$AAl?$AAl?$AAy?$AA?4?$AA?$AN?$AA?6?$AA?$AA@ 10003048     com_mdd2:mdd.obj
 0001:00002088       ??_C@_1CO@GMIGOOP@?$AAW?$AAr?$AAi?$AAt?$AAe?$AA?5?$AAt?$AAi?$AAm?$AAe?$AAo?$AAu?$AAt?$AA?5?$AA?$CF?$AAd?$AA?0?$AA?5?$AA?$CF?$AAd?$AA?$AN?$AA?6?$AA?$AA@ 10003088     com_mdd2:mdd.obj
 0001:000020b8       ??_C@_1EA@JJCCGAEK@?$AAC?$AAO?$AAM?$AA_?$AAW?$AAr?$AAi?$AAt?$AAe?$AA?5?$AA?9?$AA?5?$AAd?$AAe?$AAv?$AAi?$AAc?$AAe?$AA?5?$AAw?$AAa?$AAs?$AA?5?$AAc?$AAl?$AAo?$AAs?$AAe?$AAd?$AA?6?$AA?$AN?$AA?$AA@ 100030b8     com_mdd2:mdd.obj
 0001:000020f8       ??_C@_1DK@IBJJCGOP@?$AAC?$AAO?$AAM?$AA_?$AAW?$AAr?$AAi?$AAt?$AAe?$AA?5?$AA?9?$AA?5?$AAA?$AAb?$AAo?$AAr?$AAt?$AAi?$AAn?$AAg?$AA?5?$AAw?$AAr?$AAi?$AAt?$AAe?$AA?$AN?$AA?6?$AA?$AA@ 100030f8     com_mdd2:mdd.obj
 0001:00002138       ??_C@_1GK@PCKMKKFI@?$AAC?$AAO?$AAM?$AA_?$AAW?$AAr?$AAi?$AAt?$AAe?$AA?5?$AAw?$AAa?$AAi?$AAt?$AA?5?$AAf?$AAo?$AAr?$AA?5?$AAt?$AAr?$AAa?$AAn?$AAs?$AAm?$AAi?$AAs?$AAs?$AAi?$AAo?$AAn?$AA?5@ 10003138     com_mdd2:mdd.obj
 0001:000021a8       ??_C@_1EE@GAMOAJJK@?$AAC?$AAO?$AAM?$AA_?$AAW?$AAr?$AAi?$AAt?$AAe?$AA?5?$AAr?$AAe?$AAl?$AAe?$AAa?$AAs?$AAe?$AAd?$AA?5?$AAC?$AAr?$AAi?$AAt?$AAS?$AAe?$AAc?$AA?3?$AA?5?$AA?$CF?$AAx?$AA?4?$AA?$AN@ 100031a8     com_mdd2:mdd.obj
 0001:000021ec       ??_C@_1DI@DJLNOFJH@?$AAC?$AAO?$AAM?$AA_?$AAW?$AAr?$AAi?$AAt?$AAe?$AA?5?$AAg?$AAo?$AAt?$AA?5?$AAC?$AAr?$AAi?$AAt?$AAS?$AAe?$AAc?$AA?5?$AA?$CF?$AAx?$AA?4?$AA?$AN?$AA?6?$AA?$AA@ 100031ec     com_mdd2:mdd.obj
 0001:00002224       ??_C@_1DI@CAEOCHGO@?$AAC?$AAO?$AAM?$AA_?$AAW?$AAr?$AAi?$AAt?$AAe?$AA?5?$AAG?$AAo?$AAt?$AA?5?$AAC?$AAr?$AAi?$AAt?$AAS?$AAe?$AAc?$AA?5?$AA?$CF?$AAx?$AA?4?$AA?$AN?$AA?6?$AA?$AA@ 10003224     com_mdd2:mdd.obj
 0001:00002260       ??_C@_1EC@FLKHHNEC@?$AAC?$AAO?$AAM?$AA_?$AAW?$AAr?$AAi?$AAt?$AAe?$AA?5?$AAw?$AAa?$AAi?$AAt?$AA?5?$AAf?$AAo?$AAr?$AA?5?$AAC?$AAr?$AAi?$AAt?$AAS?$AAe?$AAc?$AA?5?$AA?$CF?$AAx?$AA?4?$AA?$AN?$AA?6@ 10003260     com_mdd2:mdd.obj
 0001:000022a8       ??_C@_1HM@LBPBKPM@?$AAd?$AA?3?$AA?2?$AAc?$AAh?$AAe?$AAl?$AAa?$AAn?$AAr?$AAt?$AAm?$AA2?$AA?2?$AAp?$AAu?$AAb?$AAl?$AAi?$AAc?$AA?2?$AAc?$AAo?$AAm?$AAm?$AAo?$AAn?$AA?2?$AAo?$AAa?$AAk?$AA?2@ 100032a8     com_mdd2:mdd.obj
 0001:00002328       ??_C@_1GC@BNCJFOA@?$AAC?$AAO?$AAM?$AA_?$AAW?$AAr?$AAi?$AAt?$AAe?$AA?5?$AAC?$AAe?$AAA?$AAl?$AAl?$AAo?$AAc?$AAA?$AAs?$AAy?$AAn?$AAc?$AAh?$AAr?$AAo?$AAn?$AAo?$AAu?$AAs?$AAB?$AAu?$AAf@ 10003328     com_mdd2:mdd.obj
 0001:00002390       ??_C@_1GA@CAKHMJEI@?$AAC?$AAO?$AAM?$AA_?$AAW?$AAR?$AAI?$AAT?$AAE?$AA?0?$AA?5?$AAb?$AAa?$AAd?$AA?5?$AA?5?$AAp?$AAo?$AAi?$AAn?$AAt?$AAe?$AAr?$AA?$CI?$AA0?$AAx?$AA?$CF?$AAx?$AA?$CJ?$AA?5?$AAo?$AAr@ 10003390     com_mdd2:mdd.obj
 0001:000023f0       ??_C@_1FG@IAEGGCHL@?$AAC?$AAO?$AAM?$AA_?$AAW?$AAr?$AAi?$AAt?$AAe?$AA?3?$AA?5?$AAA?$AAc?$AAc?$AAe?$AAs?$AAs?$AA?5?$AAp?$AAe?$AAr?$AAm?$AAi?$AAs?$AAs?$AAi?$AAo?$AAn?$AA?5?$AAf?$AAa?$AAi@ 100033f0     com_mdd2:mdd.obj
 0001:00002448       ??_C@_1DK@PMCNIBAH@?$AAC?$AAO?$AAM?$AA_?$AAW?$AAR?$AAI?$AAT?$AAE?$AA?0?$AA?5?$AAd?$AAe?$AAv?$AAi?$AAc?$AAe?$AA?5?$AAn?$AAo?$AAt?$AA?5?$AAo?$AAp?$AAe?$AAn?$AA?$AN?$AA?6?$AA?$AA@ 10003448     com_mdd2:mdd.obj
 0001:00002484       ??_C@_1DK@NPDDAOLJ@?$AA?$CL?$AAC?$AAO?$AAM?$AA_?$AAW?$AAR?$AAI?$AAT?$AAE?$AA?$CI?$AA0?$AAx?$AA?$CF?$AAX?$AA?0?$AA?5?$AA0?$AAx?$AA?$CF?$AAX?$AA?0?$AA?5?$AA?$CF?$AAd?$AA?$CJ?$AA?$AN?$AA?6?$AA?$AA@ 10003484     com_mdd2:mdd.obj
 0001:000024c0       ??_C@_1EO@HJMBEPIE@?$AA?9?$AAW?$AAa?$AAi?$AAt?$AAC?$AAo?$AAm?$AAm?$AAE?$AAv?$AAe?$AAn?$AAt?$AA?5?$AA?9?$AA?5?$AA?$CK?$AAp?$AAf?$AAd?$AAw?$AAE?$AAv?$AAe?$AAn?$AAt?$AAM?$AAa?$AAs?$AAk?$AA?5@ 100034c0     com_mdd2:mdd.obj
 0001:00002510       ??_C@_1EK@BIALANPL@?$AA?9?$AAW?$AAa?$AAi?$AAt?$AAC?$AAo?$AAm?$AAm?$AAE?$AAv?$AAe?$AAn?$AAt?$AA?5?$AA?9?$AA?5?$AAd?$AAe?$AAv?$AAi?$AAc?$AAe?$AA?5?$AAw?$AAa?$AAs?$AA?5?$AAc?$AAl?$AAo?$AAs@ 10003510     com_mdd2:mdd.obj
 0001:00002560       ??_C@_1EI@FGBADKHH@?$AA?5?$AAW?$AAa?$AAi?$AAt?$AAC?$AAo?$AAm?$AAm?$AAE?$AAv?$AAe?$AAn?$AAt?$AA?5?$AA?9?$AA?5?$AAM?$AAa?$AAs?$AAk?$AA?5?$AAw?$AAa?$AAs?$AA?5?$AAc?$AAl?$AAe?$AAa?$AAr?$AAe@ 10003560     com_mdd2:mdd.obj
 0001:000025a8       ??_C@_1GI@MFJIILJA@?$AA?5?$AAW?$AAa?$AAi?$AAt?$AAC?$AAo?$AAm?$AAm?$AAE?$AAv?$AAe?$AAn?$AAt?$AA?5?$AA?9?$AA?5?$AAE?$AAv?$AAe?$AAn?$AAt?$AAs?$AA?5?$AA0?$AAx?$AA?$CF?$AAX?$AA?0?$AA?5?$AAM?$AAa@ 100035a8     com_mdd2:mdd.obj
 0001:00002610       ??_C@_1EM@NBPFGEAJ@?$AA?9?$AAW?$AAa?$AAi?$AAt?$AAC?$AAo?$AAm?$AAm?$AAE?$AAv?$AAe?$AAn?$AAt?$AA?5?$AA?9?$AA?5?$AAM?$AAa?$AAs?$AAk?$AA?5?$AAa?$AAl?$AAr?$AAe?$AAa?$AAd?$AAy?$AA?5?$AAc?$AAl@ 10003610     com_mdd2:mdd.obj
 0001:00002660       ??_C@_1FM@MENBDCNM@?$AA?9?$AAW?$AAa?$AAi?$AAt?$AAC?$AAo?$AAm?$AAm?$AAE?$AAv?$AAe?$AAn?$AAt?$AA?5?$AA?9?$AA?5?$AAd?$AAe?$AAv?$AAi?$AAc?$AAe?$AA?5?$AAn?$AAo?$AAt?$AA?5?$AAo?$AAp?$AAe?$AAn@ 10003660     com_mdd2:mdd.obj
 0001:000026c0       ??_C@_1EI@CENKJDJK@?$AA?$CL?$AAW?$AAa?$AAi?$AAt?$AAC?$AAo?$AAm?$AAm?$AAE?$AAv?$AAe?$AAn?$AAt?$AA?5?$AAx?$AA?$CF?$AAX?$AA?5?$AAx?$AA?$CF?$AAX?$AA?0?$AA?5?$AAp?$AAM?$AAa?$AAs?$AAk?$AA?5?$AAx?$AA?$CF@ 100036c0     com_mdd2:mdd.obj
 0001:00002708       ??_C@_1GM@NOKKMADJ@?$AA?5?$AAC?$AAo?$AAm?$AAm?$AAE?$AAv?$AAe?$AAn?$AAt?$AA?5?$AA?9?$AA?5?$AAE?$AAv?$AAe?$AAn?$AAt?$AA?5?$AA0?$AAx?$AA?$CF?$AAX?$AA?0?$AA?5?$AAH?$AAa?$AAn?$AAd?$AAl?$AAe?$AA?5@ 10003708     com_mdd2:mdd.obj
 0001:00002778       ??_C@_1FI@GNEBOJFH@?$AA?5?$AAC?$AAo?$AAm?$AAm?$AAE?$AAv?$AAe?$AAn?$AAt?$AA?5?$AA?9?$AA?5?$AAE?$AAv?$AAe?$AAn?$AAt?$AA?5?$AA0?$AAx?$AA?$CF?$AAX?$AA?0?$AA?5?$AAG?$AAl?$AAo?$AAb?$AAa?$AAl?$AA?5@ 10003778     com_mdd2:mdd.obj
 0001:000027d0       ??_C@_1HI@JMOKNKMM@?$AA?5?$AAE?$AAv?$AAa?$AAl?$AAu?$AAa?$AAt?$AAe?$AAE?$AAv?$AAe?$AAn?$AAt?$AAF?$AAl?$AAa?$AAg?$AA?5?$AA?$CI?$AAe?$AAv?$AAe?$AAn?$AAt?$AAM?$AAa?$AAs?$AAk?$AA?5?$AA?$DN?$AA?5@ 100037d0     com_mdd2:mdd.obj
 0001:00002848       ??_C@_1EM@GAPNEPLB@?$AA?9?$AAC?$AAO?$AAM?$AA_?$AAI?$AAO?$AAC?$AAo?$AAn?$AAt?$AAr?$AAo?$AAl?$AA?5?$AA?$CF?$AAs?$AA?5?$AAE?$AAc?$AAo?$AAd?$AAe?$AA?$DN?$AA?$CF?$AAd?$AA?5?$AA?$CI?$AAl?$AAe?$AAn?$AA?$DN@ 10003848     com_mdd2:mdd.obj
 0001:00002894       ??_C@_1M@ILHOPKA@?$AAE?$AAr?$AAr?$AAo?$AAr?$AA?$AA@ 10003894     com_mdd2:mdd.obj
 0001:000028a0       ??_C@_1BA@JFDCMKFN@?$AAS?$AAu?$AAc?$AAc?$AAe?$AAs?$AAs?$AA?$AA@ 100038a0     com_mdd2:mdd.obj
 0001:000028b0       ??_C@_1CG@MLMOPDDN@?$AAI?$AAO?$AAC?$AAT?$AAL?$AA?5?$AAD?$AAi?$AAs?$AAa?$AAb?$AAl?$AAe?$AA?5?$AAI?$AAR?$AA?$AN?$AA?6?$AA?$AA@ 100038b0     com_mdd2:mdd.obj
 0001:000028d8       ??_C@_1CC@LGNHCIBI@?$AAI?$AAR?$AA?5?$AAm?$AAo?$AAd?$AAe?$AA?5?$AAf?$AAa?$AAi?$AAl?$AAe?$AAd?$AA?$AN?$AA?6?$AA?$AA@ 100038d8     com_mdd2:mdd.obj
 0001:000028fc       ??_C@_1CE@NOAPAGNI@?$AAI?$AAO?$AAC?$AAT?$AAL?$AA?5?$AAE?$AAn?$AAa?$AAb?$AAl?$AAe?$AA?5?$AAI?$AAR?$AA?$AN?$AA?6?$AA?$AA@ 100038fc     com_mdd2:mdd.obj
 0001:00002920       ??_C@_1CG@IAPBOCP@?$AA?5?$AAA?$AAp?$AAp?$AAl?$AAy?$AAD?$AAC?$AAB?$AA?5?$AAf?$AAa?$AAi?$AAl?$AAe?$AAd?$AA?$AN?$AA?6?$AA?$AA@ 10003920     com_mdd2:mdd.obj
 0001:00002948       ??_C@_1DA@GPICLALP@?$AA?5?$AAI?$AAO?$AAC?$AAT?$AAL?$AA_?$AAS?$AAE?$AAR?$AAI?$AAA?$AAL?$AA_?$AAS?$AAE?$AAT?$AA_?$AAD?$AAC?$AAB?$AA?$AN?$AA?6?$AA?$AA@ 10003948     com_mdd2:mdd.obj
 0001:00002978       ??_C@_1DA@MBKJPAMD@?$AA?5?$AAI?$AAO?$AAC?$AAT?$AAL?$AA_?$AAS?$AAE?$AAR?$AAI?$AAA?$AAL?$AA_?$AAG?$AAE?$AAT?$AA_?$AAD?$AAC?$AAB?$AA?$AN?$AA?6?$AA?$AA@ 10003978     com_mdd2:mdd.obj
 0001:000029a8       ??_C@_1EI@KIHCPENE@?$AA?5?$AAI?$AAO?$AAC?$AAT?$AAL?$AA_?$AAS?$AAE?$AAR?$AAI?$AAA?$AAL?$AA_?$AAI?$AAM?$AAM?$AAE?$AAD?$AAI?$AAA?$AAT?$AAE?$AA_?$AAC?$AAH?$AAA?$AAR?$AA?5?$AA0?$AAx?$AA?$CF@ 100039a8     com_mdd2:mdd.obj
 0001:000029f0       ??_C@_1FE@LCKDINPA@?$AA?5?$AAF?$AAl?$AAu?$AAs?$AAh?$AAi?$AAn?$AAg?$AA?5?$AA?$CF?$AAd?$AA?5?$AAb?$AAy?$AAt?$AAe?$AAs?$AA?5?$AAf?$AAr?$AAo?$AAm?$AA?5?$AAt?$AAh?$AAe?$AA?5?$AAr?$AAe?$AAa?$AAd@ 100039f0     com_mdd2:mdd.obj
 0001:00002a44       ??_C@_1DG@NONFKDMH@?$AA?5?$AAI?$AAO?$AAC?$AAT?$AAL?$AA_?$AAS?$AAE?$AAR?$AAI?$AAA?$AAL?$AA_?$AAP?$AAU?$AAR?$AAG?$AAE?$AA?5?$AA0?$AAx?$AA?$CF?$AAX?$AA?$AN?$AA?6?$AA?$AA@ 10003a44     com_mdd2:mdd.obj
 0001:00002a7c       ??_C@_1DK@FGFBKMCP@?$AA?5?$AAI?$AAO?$AAC?$AAT?$AAL?$AA_?$AAS?$AAE?$AAR?$AAI?$AAA?$AAL?$AA_?$AAG?$AAE?$AAT?$AA_?$AAT?$AAI?$AAM?$AAE?$AAO?$AAU?$AAT?$AAS?$AA?$AN?$AA?6?$AA?$AA@ 10003a7c     com_mdd2:mdd.obj
 0001:00002ab8       ??_C@_1GE@COCIEMAI@?$AA?5?$AAI?$AAO?$AAC?$AAT?$AAL?$AA_?$AAS?$AAE?$AAR?$AAI?$AAA?$AAL?$AA_?$AAS?$AAE?$AAT?$AA_?$AAC?$AAO?$AAM?$AAM?$AAT?$AAI?$AAM?$AAE?$AAO?$AAU?$AAT?$AAS?$AA?5?$AA?$CI@ 10003ab8     com_mdd2:mdd.obj
 0001:00002b1c       ??_C@_1DO@COBPCJBD@?$AA?5?$AAI?$AAO?$AAC?$AAT?$AAL?$AA_?$AAS?$AAE?$AAR?$AAI?$AAA?$AAL?$AA_?$AAG?$AAE?$AAT?$AA_?$AAP?$AAR?$AAO?$AAP?$AAE?$AAR?$AAT?$AAI?$AAE?$AAS?$AA?$AN?$AA?6?$AA?$AA@ 10003b1c     com_mdd2:mdd.obj
 0001:00002b60       ??_C@_1EA@IBDHDHLD@?$AA?5?$AAI?$AAO?$AAC?$AAT?$AAL?$AA_?$AAS?$AAE?$AAR?$AAI?$AAA?$AAL?$AA_?$AAG?$AAE?$AAT?$AA_?$AAM?$AAO?$AAD?$AAE?$AAM?$AAS?$AAT?$AAA?$AAT?$AAU?$AAS?$AA?$AN?$AA?6?$AA?$AA@ 10003b60     com_mdd2:mdd.obj
 0001:00002ba0       ??_C@_1DO@GPNOPFOC@?$AA?5?$AAI?$AAO?$AAC?$AAT?$AAL?$AA_?$AAS?$AAE?$AAR?$AAI?$AAA?$AAL?$AA_?$AAG?$AAE?$AAT?$AA_?$AAC?$AAO?$AAM?$AAM?$AAS?$AAT?$AAA?$AAT?$AAU?$AAS?$AA?$AN?$AA?6?$AA?$AA@ 10003ba0     com_mdd2:mdd.obj
 0001:00002be0       ??_C@_1FE@DCNACOPO@?$AA?5?$AAC?$AAO?$AAM?$AA_?$AAI?$AAO?$AAC?$AAo?$AAn?$AAt?$AAr?$AAo?$AAl?$AA?5?$AA?9?$AA?5?$AAE?$AAr?$AAr?$AAo?$AAr?$AA?5?$AAi?$AAn?$AA?5?$AAW?$AAa?$AAi?$AAt?$AAC?$AAo@ 10003be0     com_mdd2:mdd.obj
 0001:00002c34       ??_C@_1DK@MHHDNLMO@?$AA?5?$AAI?$AAO?$AAC?$AAT?$AAL?$AA_?$AAS?$AAE?$AAR?$AAI?$AAA?$AAL?$AA_?$AAW?$AAA?$AAI?$AAT?$AA_?$AAO?$AAN?$AA_?$AAM?$AAA?$AAS?$AAK?$AA?$AN?$AA?6?$AA?$AA@ 10003c34     com_mdd2:mdd.obj
 0001:00002c70       ??_C@_1FG@BOKINKK@?$AA?5?$AAS?$AAe?$AAt?$AAW?$AAa?$AAi?$AAt?$AAM?$AAa?$AAs?$AAk?$AA?5?$AA?9?$AA?5?$AAm?$AAa?$AAs?$AAk?$AA?5?$AAx?$AA?$CF?$AAX?$AA?0?$AA?5?$AAg?$AAl?$AAo?$AAb?$AAa?$AAl?$AA?5@ 10003c70     com_mdd2:mdd.obj
 0001:00002cc8       ??_C@_1EK@BIBFMIMA@?$AA?5?$AAS?$AAe?$AAt?$AAW?$AAa?$AAi?$AAt?$AAM?$AAa?$AAs?$AAk?$AA?5?$AA?9?$AA?5?$AAh?$AAa?$AAn?$AAd?$AAl?$AAe?$AA?5?$AAx?$AA?$CF?$AAX?$AA?5?$AAm?$AAa?$AAs?$AAk?$AA?5?$AAx@ 10003cc8     com_mdd2:mdd.obj
 0001:00002d18       ??_C@_1EG@JONHGGFH@?$AA?5?$AAI?$AAO?$AAC?$AAT?$AAL?$AA_?$AAS?$AAE?$AAR?$AAI?$AAA?$AAL?$AA_?$AAS?$AAE?$AAT?$AA_?$AAW?$AAA?$AAI?$AAT?$AA_?$AAM?$AAA?$AAS?$AAK?$AA?5?$AA0?$AAx?$AA?$CF?$AAX@ 10003d18     com_mdd2:mdd.obj
 0001:00002d60       ??_C@_1CK@EJMDEGNB@?$AA?5?$AAI?$AAn?$AAv?$AAa?$AAl?$AAi?$AAd?$AA?5?$AAp?$AAa?$AAr?$AAa?$AAm?$AAe?$AAt?$AAe?$AAr?$AA?$AN?$AA?6?$AA?$AA@ 10003d60     com_mdd2:mdd.obj
 0001:00002d8c       ??_C@_1DM@BJAAJCOJ@?$AA?5?$AAI?$AAO?$AAC?$AAT?$AAL?$AA_?$AAS?$AAE?$AAR?$AAI?$AAA?$AAL?$AA_?$AAG?$AAE?$AAT?$AA_?$AAW?$AAA?$AAI?$AAT?$AA_?$AAM?$AAA?$AAS?$AAK?$AA?$AN?$AA?6?$AA?$AA@ 10003d8c     com_mdd2:mdd.obj
 0001:00002dc8       ??_C@_1DA@CLADOFAD@?$AA?5?$AAI?$AAO?$AAC?$AAT?$AAL?$AA_?$AAS?$AAE?$AAR?$AAI?$AAA?$AAL?$AA_?$AAS?$AAE?$AAT?$AA_?$AAX?$AAO?$AAN?$AA?$AN?$AA?6?$AA?$AA@ 10003dc8     com_mdd2:mdd.obj
 0001:00002df8       ??_C@_1DC@OONFCAKE@?$AA?5?$AAI?$AAO?$AAC?$AAT?$AAL?$AA_?$AAS?$AAE?$AAR?$AAI?$AAA?$AAL?$AA_?$AAS?$AAE?$AAT?$AA_?$AAX?$AAO?$AAF?$AAF?$AA?$AN?$AA?6?$AA?$AA@ 10003df8     com_mdd2:mdd.obj
 0001:00002e2c       ??_C@_1DA@LCJAIJKL@?$AA?5?$AAI?$AAO?$AAC?$AAT?$AAL?$AA_?$AAS?$AAE?$AAR?$AAI?$AAA?$AAL?$AA_?$AAC?$AAL?$AAR?$AA_?$AAR?$AAT?$AAS?$AA?$AN?$AA?6?$AA?$AA@ 10003e2c     com_mdd2:mdd.obj
 0001:00002e5c       ??_C@_1DA@PJMEFDIH@?$AA?5?$AAI?$AAO?$AAC?$AAT?$AAL?$AA_?$AAS?$AAE?$AAR?$AAI?$AAA?$AAL?$AA_?$AAS?$AAE?$AAT?$AA_?$AAR?$AAT?$AAS?$AA?$AN?$AA?6?$AA?$AA@ 10003e5c     com_mdd2:mdd.obj
 0001:00002e8c       ??_C@_1DA@JNBPMBCJ@?$AA?5?$AAI?$AAO?$AAC?$AAT?$AAL?$AA_?$AAS?$AAE?$AAR?$AAI?$AAA?$AAL?$AA_?$AAC?$AAL?$AAR?$AA_?$AAD?$AAT?$AAR?$AA?$AN?$AA?6?$AA?$AA@ 10003e8c     com_mdd2:mdd.obj
 0001:00002ebc       ??_C@_1DA@NGELBLAF@?$AA?5?$AAI?$AAO?$AAC?$AAT?$AAL?$AA_?$AAS?$AAE?$AAR?$AAI?$AAA?$AAL?$AA_?$AAS?$AAE?$AAT?$AA_?$AAD?$AAT?$AAR?$AA?$AN?$AA?6?$AA?$AA@ 10003ebc     com_mdd2:mdd.obj
 0001:00002eec       ??_C@_1DM@GNACIDMB@?$AA?5?$AAI?$AAO?$AAC?$AAT?$AAL?$AA_?$AAS?$AAE?$AAR?$AAI?$AAA?$AAL?$AA_?$AAS?$AAE?$AAT?$AA_?$AAB?$AAR?$AAE?$AAA?$AAK?$AA_?$AAO?$AAF?$AAF?$AA?$AN?$AA?6?$AA?$AA@ 10003eec     com_mdd2:mdd.obj
 0001:00002f28       ??_C@_1DK@NGIHOHIF@?$AA?5?$AAI?$AAO?$AAC?$AAT?$AAL?$AA_?$AAS?$AAE?$AAR?$AAI?$AAA?$AAL?$AA_?$AAS?$AAE?$AAT?$AA_?$AAB?$AAR?$AAE?$AAA?$AAK?$AA_?$AAO?$AAN?$AA?$AN?$AA?6?$AA?$AA@ 10003f28     com_mdd2:mdd.obj
 0001:00002f68       ??_C@_1GI@OFPAKAHG@?$AAC?$AAO?$AAM?$AA_?$AAI?$AAo?$AAc?$AAt?$AAl?$AA?3?$AA?5?$AAI?$AAo?$AAc?$AAt?$AAl?$AA?5?$AA?$CF?$AAx?$AA?5?$AAa?$AAc?$AAc?$AAe?$AAs?$AAs?$AA?5?$AAp?$AAe?$AAr?$AAm?$AAi@ 10003f68     com_mdd2:mdd.obj
 0001:00002fd0       ??_C@_1CM@DKOMLJNL@?$AAP?$AAr?$AAo?$AAc?$AAe?$AAs?$AAs?$AA?5?$AAi?$AAs?$AA?5?$AAe?$AAx?$AAi?$AAt?$AAi?$AAn?$AAg?$AA?4?$AA?$AN?$AA?6?$AA?$AA@ 10003fd0     com_mdd2:mdd.obj
 0001:00003000       ??_C@_1EK@GAFFJFEI@?$AA?5?$AAC?$AAO?$AAM?$AA_?$AAI?$AAO?$AAC?$AAo?$AAn?$AAt?$AAr?$AAo?$AAl?$AA?5?$AA?9?$AA?5?$AAd?$AAe?$AAv?$AAi?$AAc?$AAe?$AA?5?$AAw?$AAa?$AAs?$AA?5?$AAc?$AAl?$AAo?$AAs@ 10004000     com_mdd2:mdd.obj
 0001:00003050       ??_C@_1GK@BPHGGHEJ@?$AA?$CL?$AAC?$AAO?$AAM?$AA_?$AAI?$AAO?$AAC?$AAo?$AAn?$AAt?$AAr?$AAo?$AAl?$AA?$CI?$AA0?$AAx?$AA?$CF?$AAX?$AA?0?$AA?5?$AA?$CF?$AAd?$AA?0?$AA?5?$AA0?$AAx?$AA?$CF?$AAX?$AA?0?$AA?5?$AA?$CF@ 10004050     com_mdd2:mdd.obj
 0001:000030bc       ??_C@_1CM@ENDIALIE@?$AA?5?$AAI?$AAn?$AAv?$AAa?$AAl?$AAi?$AAd?$AA?5?$AAi?$AAo?$AAc?$AAt?$AAl?$AA?5?$AA0?$AAx?$AA?$CF?$AAX?$AA?$AN?$AA?6?$AA?$AA@ 100040bc     com_mdd2:mdd.obj
 0001:000031a8       IoVTbl                     100041a8     serial_common_topaz_v1:serial.obj
 0001:00003220       IrVTbl                     10004220     serial_common_topaz_v1:serial.obj
 0001:00003298       ??_C@_1DC@CHKJNLCO@?$AAS?$AAe?$AAr?$AAi?$AAa?$AAl?$AA?3?$AA?3?$AAM?$AAa?$AAp?$AAD?$AAM?$AAA?$AAB?$AAu?$AAf?$AAf?$AAe?$AAr?$AAs?$AA?9?$AA?$AN?$AA?6?$AA?$AA@ 10004298     serial_common_topaz_v1:serial.obj
 0001:000032d0       ??_C@_1HK@IMKDHNPD@?$AAS?$AAe?$AAr?$AAi?$AAa?$AAl?$AA?3?$AAM?$AAa?$AAp?$AAD?$AAM?$AAA?$AAB?$AAu?$AAf?$AAf?$AAe?$AAr?$AAs?$AA?$CI?$AA?$CJ?$AA?5?$AA?9?$AA?5?$AAF?$AAa?$AAi?$AAl?$AAe?$AAd?$AA?5@ 100042d0     serial_common_topaz_v1:serial.obj
 0001:00003350       ??_C@_1HK@FHKOJLEH@?$AAS?$AAe?$AAr?$AAi?$AAa?$AAl?$AA?3?$AAM?$AAa?$AAp?$AAD?$AAM?$AAA?$AAB?$AAu?$AAf?$AAf?$AAe?$AAr?$AAs?$AA?$CI?$AA?$CJ?$AA?5?$AA?9?$AA?5?$AAF?$AAa?$AAi?$AAl?$AAe?$AAd?$AA?5@ 10004350     serial_common_topaz_v1:serial.obj
 0001:000033cc       ??_C@_1DC@OBMGNCKJ@?$AAS?$AAe?$AAr?$AAi?$AAa?$AAl?$AA?3?$AA?3?$AAM?$AAa?$AAp?$AAD?$AAM?$AAA?$AAB?$AAu?$AAf?$AAf?$AAe?$AAr?$AAs?$AA?$CL?$AA?$AN?$AA?6?$AA?$AA@ 100043cc     serial_common_topaz_v1:serial.obj
 0001:00003400       ??_C@_1DG@HIDCMBCI@?$AAS?$AAe?$AAr?$AAi?$AAa?$AAl?$AA?3?$AA?3?$AAU?$AAn?$AAm?$AAa?$AAp?$AAD?$AAM?$AAA?$AAB?$AAu?$AAf?$AAf?$AAe?$AAr?$AAs?$AA?$CL?$AA?$AN?$AA?6?$AA?$AA@ 10004400     serial_common_topaz_v1:serial.obj
 0001:00003438       ??_C@_1DE@ECNAKMCB@?$AAS?$AAe?$AAr?$AAi?$AAa?$AAl?$AA?3?$AA?3?$AAI?$AAn?$AAi?$AAt?$AAC?$AAh?$AAa?$AAn?$AAn?$AAe?$AAl?$AAD?$AAM?$AAA?$AA?9?$AA?$AN?$AA?6?$AA?$AA@ 10004438     serial_common_topaz_v1:serial.obj
 0001:00003470       ??_C@_1IA@FJHGBLNM@?$AAE?$AAR?$AAR?$AAO?$AAR?$AA?3?$AAI?$AAn?$AAi?$AAt?$AAC?$AAh?$AAa?$AAn?$AAn?$AAe?$AAl?$AAD?$AAM?$AAA?$AA?$CI?$AAT?$AAx?$AA?$CJ?$AA?3?$AA?5?$AAD?$AAD?$AAK?$AAS?$AAd?$AAm@ 10004470     serial_common_topaz_v1:serial.obj
 0001:000034f0       ??_C@_1HO@OIJBGMGH@?$AAE?$AAR?$AAR?$AAO?$AAR?$AA?3?$AAI?$AAn?$AAi?$AAt?$AAC?$AAh?$AAa?$AAn?$AAn?$AAe?$AAl?$AAD?$AAM?$AAA?$AA?$CI?$AAT?$AAx?$AA?$CJ?$AA?3?$AA?5?$AAS?$AAd?$AAm?$AAa?$AAO?$AAp@ 100044f0     serial_common_topaz_v1:serial.obj
 0001:00003570       ??_C@_1DK@MECGILIJ@?$AAC?$AAh?$AAa?$AAn?$AAn?$AAe?$AAl?$AA?5?$AAA?$AAl?$AAl?$AAo?$AAc?$AAa?$AAt?$AAe?$AAd?$AA?$CI?$AAT?$AAx?$AA?$CJ?$AA?5?$AA?3?$AA?5?$AA?$CF?$AAd?$AA?$AN?$AA?6?$AA?$AA@ 10004570     serial_common_topaz_v1:serial.obj
 0001:000035b0       ??_C@_1IA@LACMLKCC@?$AAE?$AAR?$AAR?$AAO?$AAR?$AA?3?$AAI?$AAn?$AAi?$AAt?$AAC?$AAh?$AAa?$AAn?$AAn?$AAe?$AAl?$AAD?$AAM?$AAA?$AA?$CI?$AAR?$AAx?$AA?$CJ?$AA?3?$AA?5?$AAD?$AAD?$AAK?$AAS?$AAd?$AAm@ 100045b0     serial_common_topaz_v1:serial.obj
 0001:00003630       ??_C@_1HG@FAMPPNKF@?$AAE?$AAR?$AAR?$AAO?$AAR?$AA?3?$AAI?$AAn?$AAi?$AAt?$AAC?$AAh?$AAa?$AAn?$AAn?$AAe?$AAl?$AAD?$AAM?$AAA?$AA?$CI?$AAR?$AAx?$AA?$CJ?$AA?3?$AA?5?$AAS?$AAd?$AAm?$AAa?$AAO?$AAp@ 10004630     serial_common_topaz_v1:serial.obj
 0001:000036a8       ??_C@_1DK@LGNHNBAJ@?$AAC?$AAh?$AAa?$AAn?$AAn?$AAe?$AAl?$AA?5?$AAA?$AAl?$AAl?$AAo?$AAc?$AAa?$AAt?$AAe?$AAd?$AA?$CI?$AAR?$AAx?$AA?$CJ?$AA?5?$AA?3?$AA?5?$AA?$CF?$AAd?$AA?$AN?$AA?6?$AA?$AA@ 100046a8     serial_common_topaz_v1:serial.obj
 0001:000036e4       ??_C@_1DE@IELPKFKG@?$AAS?$AAe?$AAr?$AAi?$AAa?$AAl?$AA?3?$AA?3?$AAI?$AAn?$AAi?$AAt?$AAC?$AAh?$AAa?$AAn?$AAn?$AAe?$AAl?$AAD?$AAM?$AAA?$AA?$CL?$AA?$AN?$AA?6?$AA?$AA@ 100046e4     serial_common_topaz_v1:serial.obj
 0001:00003718       ??_C@_1CG@EFDGJIGJ@?$AAS?$AAe?$AAr?$AAi?$AAa?$AAl?$AA?3?$AA?3?$AAI?$AAn?$AAi?$AAt?$AAD?$AAM?$AAA?$AA?9?$AA?$AN?$AA?6?$AA?$AA@ 10004718     serial_common_topaz_v1:serial.obj
 0001:00003740       ??_C@_1GM@FHBMJAOE@?$AAS?$AAe?$AAr?$AAi?$AAa?$AAl?$AA?3?$AAI?$AAn?$AAi?$AAt?$AAD?$AAM?$AAA?$AA?$CI?$AA?$CJ?$AA?5?$AA?9?$AA?5?$AAF?$AAa?$AAi?$AAl?$AAe?$AAd?$AA?5?$AAt?$AAo?$AA?5?$AAi?$AAn?$AAi@ 10004740     serial_common_topaz_v1:serial.obj
 0001:000037b0       ??_C@_1GA@JHBAKDBI@?$AAS?$AAe?$AAr?$AAi?$AAa?$AAl?$AA?3?$AAI?$AAn?$AAi?$AAt?$AAD?$AAM?$AAA?$AA?$CI?$AA?$CJ?$AA?5?$AA?9?$AA?5?$AAF?$AAa?$AAi?$AAl?$AAe?$AAd?$AA?5?$AAt?$AAo?$AA?5?$AAm?$AAa?$AAp@ 100047b0     serial_common_topaz_v1:serial.obj
 0001:00003810       ??_C@_1GA@KHDKMJHK@?$AAS?$AAe?$AAr?$AAi?$AAa?$AAl?$AA?3?$AAI?$AAn?$AAi?$AAt?$AAD?$AAM?$AAA?$AA?$CI?$AA?$CJ?$AA?5?$AA?9?$AA?5?$AAF?$AAa?$AAi?$AAl?$AAe?$AAd?$AA?5?$AAt?$AAo?$AA?5?$AAm?$AAa?$AAp@ 10004810     serial_common_topaz_v1:serial.obj
 0001:00003870       ??_C@_1CM@NCPBMLMN@?$AAC?$AAM?$AAX?$AA3?$AA1?$AAD?$AAi?$AAs?$AAk?$AA?3?$AA?3?$AAI?$AAn?$AAi?$AAt?$AAD?$AAM?$AAA?$AA?$CL?$AA?$AN?$AA?6?$AA?$AA@ 10004870     serial_common_topaz_v1:serial.obj
 0001:000038a0       ??_C@_1HC@HKDDJJBF@?$AAS?$AAe?$AAr?$AAi?$AAa?$AAl?$AA?3?$AAU?$AAn?$AAm?$AAa?$AAp?$AAD?$AAM?$AAA?$AAB?$AAu?$AAf?$AAf?$AAe?$AAr?$AAs?$AA?$CI?$AA?$CJ?$AA?5?$AA?9?$AA?5?$AAF?$AAa?$AAi?$AAl?$AAe@ 100048a0     serial_common_topaz_v1:serial.obj
 0001:00003918       ??_C@_1HE@LPLAFBPB@?$AAS?$AAe?$AAr?$AAi?$AAa?$AAl?$AA?3?$AAD?$AAe?$AAi?$AAn?$AAi?$AAt?$AAC?$AAh?$AAa?$AAn?$AAn?$AAe?$AAl?$AAD?$AAM?$AAA?$AA?$CI?$AA?$CJ?$AA?5?$AA?9?$AA?5?$AAF?$AAa?$AAi?$AAl@ 10004918     serial_common_topaz_v1:serial.obj
 0001:0000398c       ??_C@_1CC@GDJIGBB@?$AAS?$AAe?$AAr?$AAS?$AAe?$AAr?$AAi?$AAa?$AAl?$AAI?$AAn?$AAi?$AAt?$AA?$CL?$AA?$AN?$AA?6?$AA?$AA@ 1000498c     serial_common_topaz_v1:serial.obj
 0001:000039b0       ??_C@_1HI@GKOGACL@?$AAE?$AAR?$AAR?$AAO?$AAR?$AA?3?$AA?5?$AAF?$AAa?$AAi?$AAl?$AAe?$AAd?$AA?5?$AAt?$AAo?$AA?5?$AAo?$AAb?$AAt?$AAa?$AAi?$AAn?$AA?5?$AAs?$AAy?$AAs?$AAi?$AAn?$AAt?$AAr?$AA?5@ 100049b0     serial_common_topaz_v1:serial.obj
 0001:00003a28       ??_C@_1EO@NPLFPCN@?$AAE?$AAR?$AAR?$AAO?$AAR?$AA?3?$AA?5?$AAI?$AAn?$AAi?$AAt?$AAD?$AAM?$AAA?$AA?3?$AA?5?$AAS?$AAy?$AAs?$AAi?$AAn?$AAt?$AAr?$AA?5?$AAr?$AAe?$AAq?$AAu?$AAe?$AAs?$AAt?$AA?5@ 10004a28     serial_common_topaz_v1:serial.obj
 0001:00003a78       ??_C@_1DA@PBKEAGMP@?$AAE?$AAR?$AAR?$AAO?$AAR?$AA?3?$AA?5?$AAI?$AAn?$AAi?$AAt?$AAD?$AAM?$AAA?$AA?5?$AAf?$AAa?$AAi?$AAl?$AAe?$AAd?$AA?$AN?$AA?6?$AA?$AA@ 10004a78     serial_common_topaz_v1:serial.obj
 0001:00003aa8       ??_C@_1GE@LFJJNEHB@?$AAS?$AAe?$AAr?$AAI?$AAn?$AAi?$AAt?$AA?3?$AA?5?$AAD?$AAM?$AAA?$AA?5?$AAe?$AAn?$AAa?$AAb?$AAl?$AAe?$AAd?$AA?5?$AAf?$AAo?$AAr?$AA?5?$AAt?$AAh?$AAi?$AAs?$AA?5?$AAU?$AAA@ 10004aa8     serial_common_topaz_v1:serial.obj
 0001:00003b10       ??_C@_1EI@LKKKIHPA@?$AAS?$AAe?$AAr?$AAI?$AAn?$AAi?$AAt?$AA?5?$AA?9?$AA?5?$AAI?$AAn?$AAi?$AAt?$AAi?$AAa?$AAl?$AAi?$AAz?$AAa?$AAt?$AAi?$AAo?$AAn?$AA?5?$AAf?$AAa?$AAi?$AAl?$AAe?$AAd?$AA?$CB@ 10004b10     serial_common_topaz_v1:serial.obj
 0001:00003b58       ??_C@_1DE@MPEGKKCD@?$AAC?$AAa?$AAn?$AAn?$AAo?$AAt?$AA?5?$AAo?$AAb?$AAt?$AAa?$AAi?$AAn?$AA?5?$AAU?$AAA?$AAR?$AAT?$AA?5?$AAI?$AAR?$AAQ?$AA?$CB?$AA?$AN?$AA?6?$AA?$AA@ 10004b58     serial_common_topaz_v1:serial.obj
 0001:00003b8c       ??_C@_1CI@OHCJFJPM@?$AAE?$AAR?$AAR?$AAO?$AAR?$AA?3?$AA?5?$AA?$CF?$AAs?$AA?5?$AAl?$AAi?$AAn?$AAe?$AA?5?$AA?$CF?$AAd?$AA?3?$AA?5?$AA?$AA@ 10004b8c     serial_common_topaz_v1:serial.obj
 0001:00003bb8       ??_C@_1KK@CGFGHCOA@?$AAc?$AA?3?$AA?2?$AAw?$AAi?$AAn?$AAc?$AAe?$AAr?$AAo?$AAo?$AAt?$AAs?$AA?2?$AAt?$AAo?$AAp?$AAa?$AAz?$AA?2?$AAw?$AAi?$AAn?$AAc?$AAe?$AA7?$AA0?$AA0?$AA?2?$AAp?$AAl?$AAa@ 10004bb8     serial_common_topaz_v1:serial.obj
 0001:00003c68       ??_C@_1EK@CPGJFCEB@?$AAE?$AAR?$AAR?$AAO?$AAR?$AA?3?$AA?5?$AAF?$AAa?$AAi?$AAl?$AAe?$AAd?$AA?5?$AAt?$AAo?$AA?5?$AAo?$AAb?$AAt?$AAa?$AAi?$AAn?$AA?5?$AAu?$AAa?$AAr?$AAt?$AA?5?$AAi?$AAn?$AAf@ 10004c68     serial_common_topaz_v1:serial.obj
 0001:00003cb4       ??_C@_1BG@BBGKJFAK@?$AAS?$AAe?$AAr?$AAI?$AAn?$AAi?$AAt?$AA?5?$AA?$AN?$AA?6?$AA?$AA@ 10004cb4     serial_common_topaz_v1:serial.obj
 0001:00003cd0       ??_C@_1FG@GIOEEIKH@?$AAS?$AAe?$AAr?$AAI?$AAn?$AAi?$AAt?$AA?5?$AA?9?$AA?5?$AAU?$AAn?$AAa?$AAb?$AAl?$AAe?$AA?5?$AAt?$AAo?$AA?5?$AAr?$AAe?$AAa?$AAd?$AA?5?$AAr?$AAe?$AAg?$AAi?$AAs?$AAt?$AAr@ 10004cd0     serial_common_topaz_v1:serial.obj
 0001:00003d28       ??_C@_1BG@EMAAIJFM@?$AAS?$AAe?$AAr?$AAI?$AAn?$AAi?$AAt?$AA?$CL?$AA?$AN?$AA?6?$AA?$AA@ 10004d28     serial_common_topaz_v1:serial.obj
 0001:00003d40       ??_C@_1FE@JNJDHKCP@?$AAS?$AAe?$AAr?$AA_?$AAI?$AAn?$AAt?$AAe?$AAr?$AAn?$AAa?$AAl?$AAM?$AAa?$AAp?$AAR?$AAe?$AAg?$AAi?$AAs?$AAt?$AAe?$AAr?$AAA?$AAd?$AAd?$AAr?$AAe?$AAs?$AAs?$AAe?$AAs@ 10004d40     serial_common_topaz_v1:serial.obj
 0001:00003d94       ??_C@_1DO@NLGIPAAL@?$AAE?$AAr?$AAr?$AAo?$AAr?$AA?5?$AAt?$AAr?$AAa?$AAn?$AAs?$AAl?$AAa?$AAt?$AAi?$AAn?$AAg?$AA?5?$AAI?$AA?1?$AAO?$AA?5?$AAP?$AAo?$AAr?$AAt?$AAs?$AA?4?$AA?$AN?$AA?6?$AA?$AA@ 10004d94     serial_common_topaz_v1:serial.obj
 0001:00003dd4       ??_C@_1DE@LLPCMHLL@?$AAE?$AAr?$AAr?$AAo?$AAr?$AA?5?$AAm?$AAa?$AAp?$AAp?$AAi?$AAn?$AAg?$AA?5?$AAI?$AA?1?$AAO?$AA?5?$AAP?$AAo?$AAr?$AAt?$AAs?$AA?$AN?$AA?6?$AA?$AA@ 10004dd4     serial_common_topaz_v1:serial.obj
 0001:00003e08       ??_C@_1HI@DLIBJEEP@?$AAS?$AAe?$AAr?$AA_?$AAI?$AAn?$AAt?$AAe?$AAr?$AAn?$AAa?$AAl?$AAM?$AAa?$AAp?$AAR?$AAe?$AAg?$AAi?$AAs?$AAt?$AAe?$AAr?$AAA?$AAd?$AAd?$AAr?$AAe?$AAs?$AAs?$AAe?$AAs@ 10004e08     serial_common_topaz_v1:serial.obj
 0001:00003e80       ??_C@_1CO@MELJPONO@?$AAS?$AAe?$AAr?$AA_?$AAG?$AAe?$AAt?$AAR?$AAe?$AAg?$AAi?$AAs?$AAt?$AAr?$AAy?$AAD?$AAa?$AAt?$AAa?$AA?9?$AA?$AN?$AA?6?$AA?$AA@ 10004e80     serial_common_topaz_v1:serial.obj
 0001:00003eb0       ??_C@_1GG@DBBFFFPE@?$AAF?$AAa?$AAi?$AAl?$AAe?$AAd?$AA?5?$AAt?$AAo?$AA?5?$AAg?$AAe?$AAt?$AA?5?$AAs?$AAe?$AAr?$AAi?$AAa?$AAl?$AA?5?$AAr?$AAe?$AAg?$AAi?$AAs?$AAt?$AAr?$AAy?$AA?5?$AAv?$AAa@ 10004eb0     serial_common_topaz_v1:serial.obj
 0001:00003f18       ??_C@_1M@PEPOCCHH@?$AAI?$AAo?$AAL?$AAe?$AAn?$AA?$AA@ 10004f18     serial_common_topaz_v1:serial.obj
 0001:00003f24       ??_C@_1O@JMCNHCBG@?$AAI?$AAo?$AAB?$AAa?$AAs?$AAe?$AA?$AA@ 10004f24     serial_common_topaz_v1:serial.obj
 0001:00003f34       ??_C@_1DI@NMHDMNOM@?$AAF?$AAa?$AAi?$AAl?$AAe?$AAd?$AA?5?$AAt?$AAo?$AA?5?$AAo?$AAp?$AAe?$AAn?$AA?5?$AAd?$AAe?$AAv?$AAi?$AAc?$AAe?$AA?5?$AAk?$AAe?$AAy?$AA?$AN?$AA?6?$AA?$AA@ 10004f34     serial_common_topaz_v1:serial.obj
 0001:00003f70       ??_C@_1EM@GFJENPMG@?$AAS?$AAe?$AAr?$AA_?$AAG?$AAe?$AAt?$AAR?$AAe?$AAg?$AAi?$AAs?$AAt?$AAr?$AAy?$AAD?$AAa?$AAt?$AAa?$AA?$CL?$AA?3?$AAT?$AAr?$AAy?$AA?5?$AAt?$AAo?$AA?5?$AAo?$AAp?$AAe?$AAn@ 10004f70     serial_common_topaz_v1:serial.obj
 0001:00003fbc       ??_C@_1BK@OMAIILEJ@?$AAS?$AAe?$AAr?$AAI?$AAR?$AAI?$AAn?$AAi?$AAt?$AA?$CL?$AA?$AN?$AA?6?$AA?$AA@ 10004fbc     serial_common_topaz_v1:serial.obj
 0001:00003fd8       ??_C@_1BO@FBNPKIKO@?$AAS?$AAe?$AAr?$AAP?$AAo?$AAs?$AAt?$AAI?$AAn?$AAi?$AAt?$AA?9?$AA?$AN?$AA?6?$AA?$AA@ 10004fd8     serial_common_topaz_v1:serial.obj
 0001:00003ff8       ??_C@_1BO@JHLAKBCJ@?$AAS?$AAe?$AAr?$AAP?$AAo?$AAs?$AAt?$AAI?$AAn?$AAi?$AAt?$AA?$CL?$AA?$AN?$AA?6?$AA?$AA@ 10004ff8     serial_common_topaz_v1:serial.obj
 0001:00004018       ??_C@_1BG@EBFBNMHD@?$AAS?$AAe?$AAr?$AAO?$AAp?$AAe?$AAn?$AA?9?$AA?$AN?$AA?6?$AA?$AA@ 10005018     serial_common_topaz_v1:serial.obj
 0001:00004030       ??_C@_1BI@JGKCCCIH@?$AAS?$AAe?$AAr?$AAO?$AAp?$AAe?$AAn?$AA?$CL?$AA?5?$AA?$AN?$AA?6?$AA?$AA@ 10005030     serial_common_topaz_v1:serial.obj
 0001:00004048       ??_C@_1BI@JAKIKCJA@?$AAS?$AAe?$AAr?$AAC?$AAl?$AAo?$AAs?$AAe?$AA?9?$AA?$AN?$AA?6?$AA?$AA@ 10005048     serial_common_topaz_v1:serial.obj
 0001:00004060       ??_C@_1DI@CELLIILK@?$AAS?$AAe?$AAr?$AAC?$AAl?$AAo?$AAs?$AAe?$AA?0?$AA?5?$AAT?$AAX?$AA?5?$AAi?$AAn?$AA?5?$AAp?$AAr?$AAo?$AAg?$AAr?$AAe?$AAs?$AAs?$AA?4?$AA?$AN?$AA?6?$AA?$AA@ 10005060     serial_common_topaz_v1:serial.obj
 0001:00004098       ??_C@_1DI@BFALMAN@?$AAS?$AAe?$AAr?$AAC?$AAl?$AAo?$AAs?$AAe?$AA?5?$AA?9?$AA?5?$AAc?$AAl?$AAo?$AAs?$AAi?$AAn?$AAg?$AA?5?$AAd?$AAe?$AAv?$AAi?$AAc?$AAe?$AA?$AN?$AA?6?$AA?$AA@ 10005098     serial_common_topaz_v1:serial.obj
 0001:000040d0       ??_C@_1BK@FEEMAPGK@?$AAS?$AAe?$AAr?$AAC?$AAl?$AAo?$AAs?$AAe?$AA?$CL?$AA?5?$AA?$AN?$AA?6?$AA?$AA@ 100050d0     serial_common_topaz_v1:serial.obj
 0001:000040ec       ??_C@_1BK@BJMCBBFC@?$AAS?$AAe?$AAr?$AAD?$AAe?$AAi?$AAn?$AAi?$AAt?$AA?9?$AA?$AN?$AA?6?$AA?$AA@ 100050ec     serial_common_topaz_v1:serial.obj
 0001:00004108       ??_C@_1BK@NPKNBINF@?$AAS?$AAe?$AAr?$AAD?$AAe?$AAi?$AAn?$AAi?$AAt?$AA?$CL?$AA?$AN?$AA?6?$AA?$AA@ 10005108     serial_common_topaz_v1:serial.obj
 0001:00004124       ??_C@_1BO@HEKEJAFK@?$AAS?$AAe?$AAr?$AAP?$AAo?$AAw?$AAe?$AAr?$AAO?$AAf?$AAf?$AA?9?$AA?$AN?$AA?6?$AA?$AA@ 10005124     serial_common_topaz_v1:serial.obj
 0001:00004144       ??_C@_1BO@LCMLJJNN@?$AAS?$AAe?$AAr?$AAP?$AAo?$AAw?$AAe?$AAr?$AAO?$AAf?$AAf?$AA?$CL?$AA?$AN?$AA?6?$AA?$AA@ 10005144     serial_common_topaz_v1:serial.obj
 0001:00004164       ??_C@_1BM@JPFJIBBH@?$AAS?$AAe?$AAr?$AAP?$AAo?$AAw?$AAe?$AAr?$AAO?$AAn?$AA?9?$AA?$AN?$AA?6?$AA?$AA@ 10005164     serial_common_topaz_v1:serial.obj
 0001:00004180       ??_C@_1BM@FJDGIIJA@?$AAS?$AAe?$AAr?$AAP?$AAo?$AAw?$AAe?$AAr?$AAO?$AAn?$AA?$CL?$AA?$AN?$AA?6?$AA?$AA@ 10005180     serial_common_topaz_v1:serial.obj
 0001:0000419c       ??_C@_1BO@KDEEEAPG@?$AAS?$AAe?$AAr?$AAE?$AAn?$AAa?$AAb?$AAl?$AAe?$AAI?$AAR?$AA?9?$AA?$AN?$AA?6?$AA?$AA@ 1000519c     serial_common_topaz_v1:serial.obj
 0001:000041bc       ??_C@_1BO@GFCLEJHB@?$AAS?$AAe?$AAr?$AAE?$AAn?$AAa?$AAb?$AAl?$AAe?$AAI?$AAR?$AA?$CL?$AA?$AN?$AA?6?$AA?$AA@ 100051bc     serial_common_topaz_v1:serial.obj
 0001:000041dc       ??_C@_1CA@BIPACLML@?$AAS?$AAe?$AAr?$AAD?$AAi?$AAs?$AAa?$AAb?$AAl?$AAe?$AAI?$AAR?$AA?9?$AA?$AN?$AA?6?$AA?$AA@ 100051dc     serial_common_topaz_v1:serial.obj
 0001:000041fc       ??_C@_1CA@NOJPCCEM@?$AAS?$AAe?$AAr?$AAD?$AAi?$AAs?$AAa?$AAb?$AAl?$AAe?$AAI?$AAR?$AA?$CL?$AA?$AN?$AA?6?$AA?$AA@ 100051fc     serial_common_topaz_v1:serial.obj
 0001:0000421c       ??_C@_1DA@MBHIOAIP@?$AAS?$AAe?$AAr?$AAG?$AAe?$AAt?$AAC?$AAo?$AAm?$AAm?$AAP?$AAr?$AAo?$AAp?$AAe?$AAr?$AAt?$AAi?$AAe?$AAs?$AA?9?$AA?$AN?$AA?6?$AA?$AA@ 1000521c     serial_common_topaz_v1:serial.obj
 0001:0000424c       ??_C@_1DA@HBHOJAI@?$AAS?$AAe?$AAr?$AAG?$AAe?$AAt?$AAC?$AAo?$AAm?$AAm?$AAP?$AAr?$AAo?$AAp?$AAe?$AAr?$AAt?$AAi?$AAe?$AAs?$AA?$CL?$AA?$AN?$AA?6?$AA?$AA@ 1000524c     serial_common_topaz_v1:serial.obj
 0001:0000427c       ??_C@_1CC@GEOEGKIO@?$AAS?$AAe?$AAr?$AAI?$AAR?$AAC?$AAl?$AAe?$AAa?$AAr?$AAD?$AAT?$AAR?$AA?$CL?$AA?$AN?$AA?6?$AA?$AA@ 1000527c     serial_common_topaz_v1:serial.obj
 0001:000042a0       ??_C@_1BO@JMJINFLJ@?$AAS?$AAe?$AAr?$AAI?$AAR?$AAS?$AAe?$AAt?$AAD?$AAT?$AAR?$AA?$CL?$AA?$AN?$AA?6?$AA?$AA@ 100052a0     serial_common_topaz_v1:serial.obj
 0001:000042c0       ??_C@_1CC@BFFGHGGK@?$AAS?$AAe?$AAr?$AAI?$AAR?$AAC?$AAl?$AAe?$AAa?$AAr?$AAR?$AAT?$AAS?$AA?$CL?$AA?$AN?$AA?6?$AA?$AA@ 100052c0     serial_common_topaz_v1:serial.obj
 0001:000042e4       ??_C@_1BO@ONCKMJFN@?$AAS?$AAe?$AAr?$AAI?$AAR?$AAS?$AAe?$AAt?$AAR?$AAT?$AAS?$AA?$CL?$AA?$AN?$AA?6?$AA?$AA@ 100052e4     serial_common_topaz_v1:serial.obj
 0001:00004304       ??_C@_1CG@IJPJONEL@?$AAG?$AAe?$AAt?$AAS?$AAe?$AAr?$AAi?$AAa?$AAl?$AAO?$AAb?$AAj?$AAe?$AAc?$AAt?$AA?9?$AA?$AN?$AA?6?$AA?$AA@ 10005304     serial_common_topaz_v1:serial.obj
 0001:0000432c       ??_C@_1DA@BOMFGHCE@?$AAG?$AAe?$AAt?$AAS?$AAe?$AAr?$AAi?$AAa?$AAl?$AAO?$AAb?$AAj?$AAe?$AAc?$AAt?$AA?$CL?$AA?5?$AA0?$AAx?$AA?$CF?$AAx?$AA?$AN?$AA?6?$AA?$AA@ 1000532c     serial_common_topaz_v1:serial.obj
 0001:0000435c       ??_C@_1CM@OGMHCNHP@?$AAS?$AAL?$AA_?$AAR?$AAe?$AAa?$AAd?$AAM?$AAo?$AAd?$AAe?$AAm?$AAS?$AAt?$AAa?$AAt?$AAu?$AAs?$AA?9?$AA?$AN?$AA?6?$AA?$AA@ 1000535c     serial_common_topaz_v1:serialhw.obj
 0001:00004388       ??_C@_1BE@ONGCNMHP@?$AAE?$AAV?$AA_?$AAR?$AAL?$AAS?$AAD?$AA?$AN?$AA?6?$AA?$AA@ 10005388     serial_common_topaz_v1:serialhw.obj
 0001:0000439c       ??_C@_1BE@CJBOKGNE@?$AAE?$AAV?$AA_?$AAR?$AAI?$AAN?$AAG?$AA?$AN?$AA?6?$AA?$AA@ 1000539c     serial_common_topaz_v1:serialhw.obj
 0001:000043b0       ??_C@_1BC@IJKCEJBL@?$AAE?$AAV?$AA_?$AAD?$AAS?$AAR?$AA?$AN?$AA?6?$AA?$AA@ 100053b0     serial_common_topaz_v1:serialhw.obj
 0001:000043c4       ??_C@_1BC@NDEMLLHD@?$AAE?$AAV?$AA_?$AAC?$AAT?$AAS?$AA?$AN?$AA?6?$AA?$AA@ 100053c4     serial_common_topaz_v1:serialhw.obj
 0001:000043d8       ??_C@_1EO@BBNHNPIJ@?$AAS?$AAL?$AA_?$AAR?$AAe?$AAa?$AAd?$AAM?$AAo?$AAd?$AAe?$AAm?$AAS?$AAt?$AAa?$AAt?$AAu?$AAs?$AA?5?$AA?3?$AAE?$AAx?$AAc?$AAe?$AAp?$AAt?$AAi?$AAo?$AAn?$AA?5?$AAc?$AAa@ 100053d8     serial_common_topaz_v1:serialhw.obj
 0001:00004428       ??_C@_1CM@CAKICEPI@?$AAS?$AAL?$AA_?$AAR?$AAe?$AAa?$AAd?$AAM?$AAo?$AAd?$AAe?$AAm?$AAS?$AAt?$AAa?$AAt?$AAu?$AAs?$AA?$CL?$AA?$AN?$AA?6?$AA?$AA@ 10005428     serial_common_topaz_v1:serialhw.obj
 0001:00004454       ??_C@_1CK@CKBEJDG@?$AAS?$AAL?$AA_?$AAR?$AAe?$AAa?$AAd?$AAL?$AAi?$AAn?$AAe?$AAS?$AAt?$AAa?$AAt?$AAu?$AAs?$AA?9?$AA?$AN?$AA?6?$AA?$AA@ 10005454     serial_common_topaz_v1:serialhw.obj
 0001:00004480       ??_C@_1DA@NLGHEAKM@?$AAE?$AAr?$AAr?$AAo?$AAr?$AA?5?$AAB?$AAr?$AAe?$AAa?$AAk?$AA?5?$AAd?$AAe?$AAt?$AAe?$AAc?$AAt?$AA?$CB?$AA?$CB?$AA?$CB?$AA?$AN?$AA?6?$AA?$AA@ 10005480     serial_common_topaz_v1:serialhw.obj
 0001:000044b0       ??_C@_1CA@JJBJNOBC@?$AAE?$AAr?$AAr?$AAo?$AAr?$AA?5?$AAO?$AAv?$AAe?$AAr?$AAr?$AAu?$AAn?$AA?$AN?$AA?6?$AA?$AA@ 100054b0     serial_common_topaz_v1:serialhw.obj
 0001:000044d0       ??_C@_1BO@GIKMIKA@?$AAE?$AAr?$AAr?$AAo?$AAr?$AA?5?$AAp?$AAa?$AAr?$AAi?$AAt?$AAy?$AA?$AN?$AA?6?$AA?$AA@ 100054d0     serial_common_topaz_v1:serialhw.obj
 0001:000044f0       ??_C@_1BM@OEMJOLMO@?$AAE?$AAr?$AAr?$AAo?$AAr?$AA?5?$AAf?$AAr?$AAa?$AAm?$AAe?$AA?$AN?$AA?6?$AA?$AA@ 100054f0     serial_common_topaz_v1:serialhw.obj
 0001:00004510       ??_C@_1EM@BFKOKAEL@?$AAS?$AAL?$AA_?$AAR?$AAe?$AAa?$AAd?$AAL?$AAi?$AAn?$AAe?$AAS?$AAt?$AAa?$AAt?$AAu?$AAs?$AA?5?$AA?3?$AAE?$AAx?$AAc?$AAe?$AAp?$AAt?$AAi?$AAo?$AAn?$AA?5?$AAc?$AAa?$AAu@ 10005510     serial_common_topaz_v1:serialhw.obj
 0001:0000455c       ??_C@_1CK@MEMOEALB@?$AAS?$AAL?$AA_?$AAR?$AAe?$AAa?$AAd?$AAL?$AAi?$AAn?$AAe?$AAS?$AAt?$AAa?$AAt?$AAu?$AAs?$AA?$CL?$AA?$AN?$AA?6?$AA?$AA@ 1000555c     serial_common_topaz_v1:serialhw.obj
 0001:00004588       ??_C@_1EI@LNHFMLDH@?$AAS?$AAL?$AA_?$AAS?$AAe?$AAt?$AAO?$AAu?$AAt?$AAp?$AAu?$AAM?$AAo?$AAd?$AAe?$AA?5?$AA?3?$AAE?$AAx?$AAc?$AAe?$AAp?$AAt?$AAi?$AAo?$AAn?$AA?5?$AAc?$AAa?$AAu?$AAg?$AAh@ 10005588     serial_common_topaz_v1:serialhw.obj
 0001:000045d0       ??_C@_1CO@BBIHGLGD@?$AAS?$AAL?$AA_?$AAC?$AAl?$AAe?$AAa?$AAr?$AAP?$AAe?$AAn?$AAd?$AAi?$AAn?$AAg?$AAI?$AAn?$AAt?$AAs?$AA?9?$AA?$AN?$AA?6?$AA?$AA@ 100055d0     serial_common_topaz_v1:serialhw.obj
 0001:00004600       ??_C@_1FA@JLOCJEMH@?$AAS?$AAL?$AA_?$AAC?$AAl?$AAe?$AAa?$AAr?$AAP?$AAe?$AAn?$AAd?$AAi?$AAn?$AAg?$AAI?$AAn?$AAt?$AAs?$AA?5?$AA?3?$AAE?$AAx?$AAc?$AAe?$AAp?$AAt?$AAi?$AAo?$AAn?$AA?5?$AAc@ 10005600     serial_common_topaz_v1:serialhw.obj
 0001:00004650       ??_C@_1CO@NHOIGCOE@?$AAS?$AAL?$AA_?$AAC?$AAl?$AAe?$AAa?$AAr?$AAP?$AAe?$AAn?$AAd?$AAi?$AAn?$AAg?$AAI?$AAn?$AAt?$AAs?$AA?$CL?$AA?$AN?$AA?6?$AA?$AA@ 10005650     serial_common_topaz_v1:serialhw.obj
 0001:00004680       ??_C@_1CE@HMANGEPB@?$AAS?$AAL?$AA_?$AAS?$AAe?$AAt?$AAS?$AAt?$AAo?$AAp?$AAB?$AAi?$AAt?$AAs?$AA?9?$AA?$AN?$AA?6?$AA?$AA@ 10005680     serial_common_topaz_v1:serialhw.obj
 0001:000046a8       ??_C@_1EG@JGGAPAOG@?$AAS?$AAL?$AA_?$AAS?$AAe?$AAt?$AAS?$AAt?$AAo?$AAp?$AAB?$AAi?$AAt?$AAs?$AA?5?$AA?3?$AAE?$AAx?$AAc?$AAe?$AAp?$AAt?$AAi?$AAo?$AAn?$AA?5?$AAc?$AAa?$AAu?$AAg?$AAh?$AAt@ 100056a8     serial_common_topaz_v1:serialhw.obj
 0001:000046f0       ??_C@_1CO@PJPGKHFI@?$AAS?$AAL?$AA_?$AAS?$AAe?$AAt?$AAS?$AAt?$AAo?$AAp?$AAB?$AAi?$AAt?$AAs?$AA?$CL?$AA?5?$AA0?$AAx?$AA?$CF?$AAX?$AA?$AN?$AA?6?$AA?$AA@ 100056f0     serial_common_topaz_v1:serialhw.obj
 0001:00004720       ??_C@_1DG@PLGFEAGN@?$AAS?$AAL?$AA_?$AAS?$AAe?$AAt?$AAb?$AAa?$AAu?$AAd?$AAR?$AAa?$AAt?$AAe?$AA?9?$AA?5?$AAR?$AAe?$AAt?$AA?5?$AA?$DN?$AA?5?$AA?$CF?$AAd?$AA?$AN?$AA?6?$AA?$AA@ 10005720     serial_common_topaz_v1:serialhw.obj
 0001:00004758       ??_C@_1EG@KLCGBHHG@?$AAS?$AAL?$AA_?$AAS?$AAe?$AAt?$AAB?$AAa?$AAu?$AAd?$AAR?$AAa?$AAt?$AAe?$AA?5?$AA?3?$AAE?$AAx?$AAc?$AAe?$AAp?$AAt?$AAi?$AAo?$AAn?$AA?5?$AAc?$AAa?$AAu?$AAg?$AAh?$AAt@ 10005758     serial_common_topaz_v1:serialhw.obj
 0001:000047a0       ??_C@_1CG@IFGCBNHM@?$AAI?$AAR?$AA?5?$AAs?$AAp?$AAe?$AAc?$AAi?$AAa?$AAl?$AA?5?$AAc?$AAa?$AAs?$AAe?$AA?$CB?$AA?$AN?$AA?6?$AA?$AA@ 100057a0     serial_common_topaz_v1:serialhw.obj
 0001:000047c8       ??_C@_1CK@JGNKKOCJ@?$AAS?$AAL?$AA_?$AAS?$AAe?$AAt?$AAb?$AAa?$AAu?$AAd?$AAR?$AAa?$AAt?$AAe?$AA?$CL?$AA?5?$AA?$CF?$AAd?$AA?$AN?$AA?6?$AA?$AA@ 100057c8     serial_common_topaz_v1:serialhw.obj
 0001:000047f4       ??_C@_1DG@DNMHAIJE@?$AAS?$AAL?$AA_?$AAS?$AAe?$AAt?$AAB?$AAy?$AAt?$AAe?$AAS?$AAi?$AAz?$AAe?$AA?9?$AA?5?$AAR?$AAe?$AAt?$AA?5?$AA?$DN?$AA?5?$AA?$CF?$AAd?$AA?$AN?$AA?6?$AA?$AA@ 100057f4     serial_common_topaz_v1:serialhw.obj
 0001:00004830       ??_C@_1EG@MGCBBCF@?$AAS?$AAL?$AA_?$AAS?$AAe?$AAt?$AAB?$AAy?$AAt?$AAe?$AAS?$AAi?$AAz?$AAe?$AA?5?$AA?3?$AAE?$AAx?$AAc?$AAe?$AAp?$AAt?$AAi?$AAo?$AAn?$AA?5?$AAc?$AAa?$AAu?$AAg?$AAh?$AAt@ 10005830     serial_common_topaz_v1:serialhw.obj
 0001:00004878       ??_C@_1CO@GJJIKMCE@?$AAS?$AAL?$AA_?$AAS?$AAe?$AAt?$AAB?$AAy?$AAt?$AAe?$AAS?$AAi?$AAz?$AAe?$AA?$CL?$AA?5?$AA0?$AAx?$AA?$CF?$AAX?$AA?$AN?$AA?6?$AA?$AA@ 10005878     serial_common_topaz_v1:serialhw.obj
 0001:000048a8       ??_C@_1DC@IEEAPIAJ@?$AAS?$AAL?$AA_?$AAS?$AAe?$AAt?$AAP?$AAa?$AAr?$AAi?$AAt?$AAy?$AA?9?$AA?5?$AAR?$AAe?$AAt?$AA?5?$AA?$DN?$AA?5?$AA?$CF?$AAd?$AA?$AN?$AA?6?$AA?$AA@ 100058a8     serial_common_topaz_v1:serialhw.obj
 0001:000048e0       ??_C@_1EC@DBBBCNPD@?$AAS?$AAL?$AA_?$AAS?$AAe?$AAt?$AAP?$AAa?$AAr?$AAi?$AAt?$AAy?$AA?5?$AA?3?$AAE?$AAx?$AAc?$AAe?$AAp?$AAt?$AAi?$AAo?$AAn?$AA?5?$AAc?$AAa?$AAu?$AAg?$AAh?$AAt?$AA?5?$AA?6@ 100058e0     serial_common_topaz_v1:serialhw.obj
 0001:00004924       ??_C@_1CK@ONFIOLLG@?$AAS?$AAL?$AA_?$AAS?$AAe?$AAt?$AAP?$AAa?$AAr?$AAi?$AAt?$AAy?$AA?$CL?$AA?5?$AA0?$AAx?$AA?$CF?$AAX?$AA?$AN?$AA?6?$AA?$AA@ 10005924     serial_common_topaz_v1:serialhw.obj
 0001:00004950       ??_C@_1DM@DHBGBMJI@?$AAS?$AAL?$AA_?$AAS?$AAe?$AAt?$AAF?$AAl?$AAo?$AAw?$AAC?$AAo?$AAn?$AAt?$AAr?$AAo?$AAl?$AA?9?$AA?5?$AAR?$AAe?$AAt?$AA?5?$AA?$DN?$AA?5?$AA?$CF?$AAd?$AA?$AN?$AA?6?$AA?$AA@ 10005950     serial_common_topaz_v1:serialhw.obj
 0001:00004990       ??_C@_1EM@GGHGJLOO@?$AAS?$AAL?$AA_?$AAS?$AAe?$AAt?$AAF?$AAl?$AAo?$AAw?$AAC?$AAo?$AAn?$AAt?$AAr?$AAo?$AAl?$AA?5?$AA?3?$AAE?$AAx?$AAc?$AAe?$AAp?$AAt?$AAi?$AAo?$AAn?$AA?5?$AAc?$AAa?$AAu@ 10005990     serial_common_topaz_v1:serialhw.obj
 0001:000049dc       ??_C@_1CA@FOMOOPE@?$AAS?$AAe?$AAt?$AA?5?$AAI?$AAR?$AAT?$AAS?$AA?5?$AA0?$AAx?$AA?$CF?$AAX?$AA?$AN?$AA?6?$AA?$AA@ 100059dc     serial_common_topaz_v1:serialhw.obj
 0001:000049fc       ??_C@_1CE@LBCEPAJ@?$AAC?$AAl?$AAe?$AAa?$AAr?$AA?5?$AAI?$AAR?$AAT?$AAS?$AA?5?$AA0?$AAx?$AA?$CF?$AAX?$AA?$AN?$AA?6?$AA?$AA@ 100059fc     serial_common_topaz_v1:serialhw.obj
 0001:00004a20       ??_C@_1DE@OBFIKLE@?$AAS?$AAL?$AA_?$AAS?$AAe?$AAt?$AAF?$AAl?$AAo?$AAw?$AAC?$AAo?$AAn?$AAt?$AAr?$AAo?$AAl?$AA?$CL?$AA?5?$AA0?$AAx?$AA?$CF?$AAX?$AA?$AN?$AA?6?$AA?$AA@ 10005a20     serial_common_topaz_v1:serialhw.obj
 0001:00004a54       ??_C@_1BI@GBHFMPJJ@?$AAS?$AAL?$AA_?$AAR?$AAe?$AAs?$AAe?$AAt?$AA?9?$AA?$AN?$AA?6?$AA?$AA@ 10005a54     serial_common_topaz_v1:serialhw.obj
 0001:00004a6c       ??_C@_1DK@IOOMKFCH@?$AAS?$AAL?$AA_?$AAR?$AAe?$AAs?$AAe?$AAt?$AA?5?$AA?3?$AAE?$AAx?$AAc?$AAe?$AAp?$AAt?$AAi?$AAo?$AAn?$AA?5?$AAc?$AAa?$AAu?$AAg?$AAh?$AAt?$AA?5?$AA?6?$AA?$AA@ 10005a6c     serial_common_topaz_v1:serialhw.obj
 0001:00004aa8       ??_C@_1BI@KHBKMGBO@?$AAS?$AAL?$AA_?$AAR?$AAe?$AAs?$AAe?$AAt?$AA?$CL?$AA?$AN?$AA?6?$AA?$AA@ 10005aa8     serial_common_topaz_v1:serialhw.obj
 0001:00004ac0       ??_C@_1BG@FMMKOKAP@?$AAS?$AAL?$AA_?$AAI?$AAN?$AAI?$AAT?$AA?9?$AA?$AN?$AA?6?$AA?$AA@ 10005ac0     serial_common_topaz_v1:serialhw.obj
 0001:00004ad8       ??_C@_1BI@NKJCJMHP@?$AAS?$AAL?$AA_?$AAI?$AAN?$AAI?$AAT?$AA?$CL?$AA?5?$AA?$AN?$AA?6?$AA?$AA@ 10005ad8     serial_common_topaz_v1:serialhw.obj
 0001:00004af0       ??_C@_1BK@MOGJPFLC@?$AAS?$AAL?$AA_?$AAD?$AAe?$AAi?$AAn?$AAi?$AAt?$AA?9?$AA?$AN?$AA?6?$AA?$AA@ 10005af0     serial_common_topaz_v1:serialhw.obj
 0001:00004b10       ??_C@_1FE@CJELCOJJ@?$AAS?$AAL?$AA_?$AAD?$AAe?$AAi?$AAn?$AAi?$AAt?$AA?3?$AA?5?$AA?5?$AAB?$AAS?$AAP?$AAU?$AAa?$AAr?$AAt?$AAD?$AAi?$AAs?$AAa?$AAb?$AAl?$AAe?$AAC?$AAl?$AAo?$AAc?$AAk?$AA?5@ 10005b10     serial_common_topaz_v1:serialhw.obj
 0001:00004b68       ??_C@_1FC@MJPAJCJE@?$AAS?$AAL?$AA_?$AAD?$AAe?$AAi?$AAn?$AAi?$AAt?$AA?3?$AA?5?$AA?5?$AAB?$AAS?$AAP?$AAU?$AAa?$AAr?$AAt?$AAE?$AAn?$AAa?$AAb?$AAl?$AAe?$AAC?$AAl?$AAo?$AAc?$AAk?$AA?5?$AAf@ 10005b68     serial_common_topaz_v1:serialhw.obj
 0001:00004bbc       ??_C@_1BK@IAGPMDF@?$AAS?$AAL?$AA_?$AAD?$AAe?$AAi?$AAn?$AAi?$AAt?$AA?$CL?$AA?$AN?$AA?6?$AA?$AA@ 10005bbc     serial_common_topaz_v1:serialhw.obj
 0001:00004bd8       ??_C@_1BI@BBOFNEGF@?$AAS?$AAL?$AA_?$AAO?$AAp?$AAe?$AAn?$AA?9?$AA?5?$AA?$AN?$AA?6?$AA?$AA@ 10005bd8     serial_common_topaz_v1:serialhw.obj
 0001:00004bf0       ??_C@_1DI@FMFFPEGJ@?$AAS?$AAL?$AA_?$AAO?$AAp?$AAe?$AAn?$AA?5?$AA?3?$AAE?$AAx?$AAc?$AAe?$AAp?$AAt?$AAi?$AAo?$AAn?$AA?5?$AAc?$AAa?$AAu?$AAg?$AAh?$AAt?$AA?5?$AA?6?$AA?$AA@ 10005bf0     serial_common_topaz_v1:serialhw.obj
 0001:00004c28       ??_C@_1GK@JCGCHMOH@?$AAE?$AAR?$AAR?$AAO?$AAR?$AA?3?$AAI?$AAn?$AAi?$AAt?$AAC?$AAh?$AAa?$AAn?$AAn?$AAe?$AAl?$AAD?$AAM?$AAA?$AA?$CI?$AAT?$AAx?$AA?$CJ?$AA?3?$AA?5?$AAD?$AAD?$AAK?$AAS?$AAd?$AAm@ 10005c28     serial_common_topaz_v1:serialhw.obj
 0001:00004c98       ??_C@_1GK@GDOJNBL@?$AAE?$AAR?$AAR?$AAO?$AAR?$AA?3?$AAI?$AAn?$AAi?$AAt?$AAC?$AAh?$AAa?$AAn?$AAn?$AAe?$AAl?$AAD?$AAM?$AAA?$AA?$CI?$AAR?$AAx?$AA?$CJ?$AA?3?$AA?5?$AAD?$AAD?$AAK?$AAS?$AAd?$AAm@ 10005c98     serial_common_topaz_v1:serialhw.obj
 0001:00004d04       ??_C@_1DO@LHDKOKPM@?$AAB?$AAS?$AAP?$AAS?$AAe?$AAr?$AAA?$AAc?$AAq?$AAu?$AAi?$AAr?$AAe?$AAD?$AAM?$AAA?$AAR?$AAe?$AAq?$AAG?$AAp?$AAr?$AA?5?$AAf?$AAa?$AAi?$AAl?$AAe?$AAd?$AA?6?$AA?$AA@ 10005d04     serial_common_topaz_v1:serialhw.obj
 0001:00004d48       ??_C@_1EC@BKNDADN@?$AAS?$AAL?$AA_?$AAO?$AAp?$AAe?$AAn?$AA?5?$AAS?$AAe?$AAt?$AAt?$AAi?$AAn?$AAg?$AA?5?$AAD?$AAC?$AAB?$AA?5?$AAp?$AAa?$AAr?$AAa?$AAm?$AAe?$AAt?$AAe?$AAr?$AAs?$AA?$AN?$AA?6@ 10005d48     serial_common_topaz_v1:serialhw.obj
 0001:00004d90       ??_C@_1EO@FGICAOGJ@?$AAS?$AAL?$AA_?$AAO?$AAp?$AAe?$AAn?$AA?3?$AA?5?$AA?5?$AAB?$AAS?$AAP?$AAU?$AAa?$AAr?$AAt?$AAE?$AAn?$AAa?$AAb?$AAl?$AAe?$AAC?$AAl?$AAo?$AAc?$AAk?$AA?5?$AAf?$AAa?$AAi@ 10005d90     serial_common_topaz_v1:serialhw.obj
 0001:00004de0       ??_C@_1BI@BMPLKECC@?$AAS?$AAL?$AA_?$AAO?$AAp?$AAe?$AAn?$AA?$CL?$AA?5?$AA?$AN?$AA?6?$AA?$AA@ 10005de0     serial_common_topaz_v1:serialhw.obj
 0001:00004df8       ??_C@_1BK@IOPJJLMN@?$AAS?$AAL?$AA_?$AAC?$AAl?$AAo?$AAs?$AAe?$AA?9?$AA?5?$AA?$AN?$AA?6?$AA?$AA@ 10005df8     serial_common_topaz_v1:serialhw.obj
 0001:00004e18       ??_C@_1FC@OLBDKHOM@?$AAS?$AAL?$AA_?$AAC?$AAl?$AAo?$AAs?$AAe?$AA?3?$AA?5?$AA?5?$AAB?$AAS?$AAP?$AAU?$AAa?$AAr?$AAt?$AAD?$AAi?$AAs?$AAa?$AAb?$AAl?$AAe?$AAC?$AAl?$AAo?$AAc?$AAk?$AA?5?$AAf@ 10005e18     serial_common_topaz_v1:serialhw.obj
 0001:00004e6c       ??_C@_1DK@LBKBBMEN@?$AAS?$AAL?$AA_?$AAC?$AAl?$AAo?$AAs?$AAe?$AA?5?$AA?3?$AAE?$AAx?$AAc?$AAe?$AAp?$AAt?$AAi?$AAo?$AAn?$AA?5?$AAc?$AAa?$AAu?$AAg?$AAh?$AAt?$AA?5?$AA?6?$AA?$AA@ 10005e6c     serial_common_topaz_v1:serialhw.obj
 0001:00004ea8       ??_C@_1BK@IDOHOLIK@?$AAS?$AAL?$AA_?$AAC?$AAl?$AAo?$AAs?$AAe?$AA?$CL?$AA?5?$AA?$AN?$AA?6?$AA?$AA@ 10005ea8     serial_common_topaz_v1:serialhw.obj
 0001:00004ec4       ??_C@_1CA@HJCMDCEJ@?$AAS?$AAL?$AA_?$AAP?$AAo?$AAw?$AAe?$AAr?$AAO?$AAf?$AAf?$AA?9?$AA?5?$AA?$AN?$AA?6?$AA?$AA@ 10005ec4     serial_common_topaz_v1:serialhw.obj
 0001:00004ee4       ??_C@_1CA@HEDCECAO@?$AAS?$AAL?$AA_?$AAP?$AAo?$AAw?$AAe?$AAr?$AAO?$AAf?$AAf?$AA?$CL?$AA?5?$AA?$AN?$AA?6?$AA?$AA@ 10005ee4     serial_common_topaz_v1:serialhw.obj
 0001:00004f04       ??_C@_1BO@KCCHBEDD@?$AAS?$AAL?$AA_?$AAP?$AAo?$AAw?$AAe?$AAr?$AAO?$AAn?$AA?9?$AA?5?$AA?$AN?$AA?6?$AA?$AA@ 10005f04     serial_common_topaz_v1:serialhw.obj
 0001:00004f24       ??_C@_1BO@KPDJGEHE@?$AAS?$AAL?$AA_?$AAP?$AAo?$AAw?$AAe?$AAr?$AAO?$AAn?$AA?$CL?$AA?5?$AA?$AN?$AA?6?$AA?$AA@ 10005f24     serial_common_topaz_v1:serialhw.obj
 0001:00004f44       ??_C@_1CO@FLEGJJEP@?$AAS?$AAL?$AA_?$AAG?$AAe?$AAt?$AAI?$AAn?$AAt?$AAr?$AAT?$AAy?$AAp?$AAe?$AA?9?$AA?5?$AA0?$AAx?$AA?$CF?$AAX?$AA?$AN?$AA?6?$AA?$AA@ 10005f44     serial_common_topaz_v1:serialhw.obj
 0001:00004f78       ??_C@_1EI@EIMDHOFB@?$AAU?$AAA?$AAR?$AAT?$AA_?$AAU?$AAS?$AAR?$AA1?$AA?3?$AA?5?$AA0?$AAx?$AA?$CF?$AAx?$AA?5?$AA?$HM?$AA?5?$AAU?$AAA?$AAR?$AAT?$AA_?$AAU?$AAS?$AAR?$AA2?$AA?3?$AA?5?$AA0?$AAx?$AA?$CF@ 10005f78     serial_common_topaz_v1:serialhw.obj
 0001:00004fc0       ??_C@_1EE@FHJHLHHJ@?$AAS?$AAL?$AA_?$AAG?$AAe?$AAt?$AAI?$AAn?$AAt?$AAr?$AAT?$AAy?$AAp?$AAe?$AA?5?$AA?9?$AA?5?$AAA?$AAd?$AAd?$AAT?$AAX?$AAI?$AAn?$AAt?$AAr?$AA?5?$AA0?$AAx?$AA?$CF?$AAx?$AA?$AN@ 10005fc0     serial_common_topaz_v1:serialhw.obj
 0001:00005008       ??_C@_1EG@GJLKDFIJ@?$AAS?$AAL?$AA_?$AAG?$AAe?$AAt?$AAI?$AAn?$AAt?$AAr?$AAT?$AAy?$AAp?$AAe?$AA?5?$AA?3?$AAE?$AAx?$AAc?$AAe?$AAp?$AAt?$AAi?$AAo?$AAn?$AA?5?$AAc?$AAa?$AAu?$AAg?$AAh?$AAt@ 10006008     serial_common_topaz_v1:serialhw.obj
 0001:00005050       ??_C@_1DM@IJJAMJCH@?$AAG?$AAe?$AAt?$AAI?$AAn?$AAt?$AAr?$AA?3?$AA?5?$AAT?$AAX?$AA?5?$AAS?$AAD?$AAM?$AAA?$AA?5?$AAc?$AAo?$AAm?$AAp?$AAl?$AAe?$AAt?$AAi?$AAo?$AAn?$AA?$AN?$AA?6?$AA?$AA@ 10006050     serial_common_topaz_v1:serialhw.obj
 0001:0000508c       ??_C@_1DA@GAHNMNED@?$AAG?$AAe?$AAt?$AAI?$AAn?$AAt?$AAr?$AA?3?$AA?5?$AAS?$AAt?$AAa?$AAt?$AAu?$AAs?$AA?3?$AA?5?$AA0?$AAx?$AA?$CF?$AAx?$AA?$AN?$AA?6?$AA?$AA@ 1000608c     serial_common_topaz_v1:serialhw.obj
 0001:000050c0       ??_C@_1FM@MJAAPNGB@?$AAG?$AAe?$AAt?$AAI?$AAn?$AAt?$AAr?$AA?3?$AA?5?$AAp?$AAS?$AAe?$AAr?$AAH?$AAe?$AAa?$AAd?$AA?9?$AA?$DO?$AAa?$AAw?$AAa?$AAi?$AAt?$AAi?$AAn?$AAg?$AAT?$AAx?$AAD?$AAM?$AAA@ 100060c0     serial_common_topaz_v1:serialhw.obj
 0001:0000511c       ??_C@_1DM@PJOHNPMB@?$AAG?$AAe?$AAt?$AAI?$AAn?$AAt?$AAr?$AA?3?$AA?5?$AAR?$AAX?$AA?5?$AAS?$AAD?$AAM?$AAA?$AA?5?$AAc?$AAo?$AAm?$AAp?$AAl?$AAe?$AAt?$AAi?$AAo?$AAn?$AA?$AN?$AA?6?$AA?$AA@ 1000611c     serial_common_topaz_v1:serialhw.obj
 0001:00005158       ??_C@_1DO@NBICOIBA@?$AAD?$AAM?$AAA?$AA?5?$AAt?$AAx?$AA?5?$AAB?$AAu?$AAf?$AA?5?$AA0?$AA?5?$AAs?$AAt?$AAa?$AAt?$AAu?$AAs?$AA?5?$AA?$DN?$AA?5?$AA0?$AAx?$AA?$CF?$AA0?$AA8?$AAX?$AA?$AN?$AA?6?$AA?$AA@ 10006158     serial_common_topaz_v1:serialhw.obj
 0001:00005198       ??_C@_1EA@DLJIPCBP@?$AAD?$AAM?$AAA?$AA?5?$AAr?$AAx?$AA?5?$AAB?$AAu?$AAf?$AA?5?$AA?$CF?$AAd?$AA?5?$AAs?$AAt?$AAa?$AAt?$AAu?$AAs?$AA?5?$AA?$DN?$AA?5?$AA0?$AAx?$AA?$CF?$AA0?$AA8?$AAX?$AA?$AN?$AA?6?$AA?$AA@ 10006198     serial_common_topaz_v1:serialhw.obj
 0001:000051d8       ??_C@_1CG@HHGBLGMB@?$AAS?$AAL?$AA_?$AAG?$AAe?$AAt?$AAI?$AAn?$AAt?$AAr?$AAT?$AAy?$AAp?$AAe?$AA?$CL?$AA?5?$AA?$AN?$AA?6?$AA?$AA@ 100061d8     serial_common_topaz_v1:serialhw.obj
 0001:00005200       ??_C@_1FG@CAFGHEKE@?$AAS?$AAL?$AA_?$AAR?$AAx?$AAI?$AAn?$AAt?$AAr?$AAH?$AAa?$AAn?$AAd?$AAl?$AAe?$AAr?$AA?5?$AA?9?$AA?5?$AAr?$AAx?$AA?8?$AAe?$AAd?$AA?5?$AA?$CF?$AAd?$AA?0?$AA?5?$AAd?$AAr?$AAo@ 10006200     serial_common_topaz_v1:serialhw.obj
 0001:00005258       ??_C@_1BM@DPONJIOF@?$AAR?$AAx?$AA?5?$AAd?$AAr?$AAo?$AAp?$AA?5?$AA?$CF?$AAd?$AA?4?$AA?$AN?$AA?6?$AA?$AA@ 10006258     serial_common_topaz_v1:serialhw.obj
 0001:00005274       ??_C@_1CI@CDCGLEDP@?$AAE?$AAV?$AA_?$AAR?$AAX?$AAF?$AAL?$AAA?$AAG?$AA?5?$AAn?$AAo?$AAt?$AA?5?$AAs?$AAe?$AAt?$AA?$AN?$AA?6?$AA?$AA@ 10006274     serial_common_topaz_v1:serialhw.obj
 0001:0000529c       ??_C@_1CA@PHDPGJKI@?$AAE?$AAV?$AA_?$AAR?$AAX?$AAF?$AAL?$AAA?$AAG?$AA?5?$AAs?$AAe?$AAt?$AA?$AN?$AA?6?$AA?$AA@ 1000629c     serial_common_topaz_v1:serialhw.obj
 0001:000052c0       ??_C@_1EK@FPMGLCLK@?$AAS?$AAL?$AA_?$AAR?$AAx?$AAI?$AAn?$AAt?$AAr?$AAH?$AAa?$AAn?$AAd?$AAl?$AAe?$AAr?$AA?5?$AA?3?$AAE?$AAx?$AAc?$AAe?$AAp?$AAt?$AAi?$AAo?$AAn?$AA?5?$AAc?$AAa?$AAu?$AAg@ 100062c0     serial_common_topaz_v1:serialhw.obj
 0001:0000530c       ??_C@_1BA@MBMDFCIG@?$AAR?$AA?$CF?$AA0?$AA2?$AAx?$AA?$AN?$AA?6?$AA?$AA@ 1000630c     serial_common_topaz_v1:serialhw.obj
 0001:0000531c       ??_C@_1BO@KBJDPJCB@?$AAE?$AAv?$AAt?$AA?5?$AAC?$AAh?$AAa?$AAr?$AA?5?$AAx?$AA?$CF?$AAx?$AA?$AN?$AA?6?$AA?$AA@ 1000631c     serial_common_topaz_v1:serialhw.obj
 0001:00005340       ??_C@_1EE@OFPCFJOL@?$AAD?$AAr?$AAo?$AAp?$AAp?$AAi?$AAn?$AAg?$AA?5?$AAN?$AAU?$AAL?$AAL?$AA?5?$AAb?$AAy?$AAt?$AAe?$AA?5?$AAd?$AAu?$AAe?$AA?5?$AAt?$AAo?$AA?5?$AAf?$AAN?$AAu?$AAl?$AAl?$AA?$AN@ 10006340     serial_common_topaz_v1:serialhw.obj
 0001:00005388       ??_C@_1EI@BBLKKMFK@?$AAD?$AAr?$AAo?$AAp?$AAp?$AAi?$AAn?$AAg?$AA?5?$AAb?$AAy?$AAt?$AAe?$AA?5?$AAb?$AAe?$AAc?$AAa?$AAu?$AAs?$AAe?$AA?5?$AAD?$AAS?$AAR?$AA?5?$AAi?$AAs?$AA?5?$AAh?$AAi?$AAg@ 10006388     serial_common_topaz_v1:serialhw.obj
 0001:000053d0       ??_C@_1BG@BBJIEPHD@?$AAR?$AAe?$AAa?$AAd?$AA?5?$AAx?$AA?$CF?$AAx?$AA?$AN?$AA?6?$AA?$AA@ 100063d0     serial_common_topaz_v1:serialhw.obj
 0001:000053e8       ??_C@_1CK@EHCEHIML@?$AAR?$AAE?$AAA?$AAD?$AA?5?$AAE?$AAR?$AAR?$AAO?$AAR?$AA?$CB?$AA?$CB?$AA?$CB?$AA?5?$AA?5?$AAx?$AA?$CF?$AAx?$AA?$AN?$AA?6?$AA?$AA@ 100063e8     serial_common_topaz_v1:serialhw.obj
 0001:00005418       ??_C@_1FG@ECHEIFPL@?$AAS?$AAL?$AA_?$AAR?$AAx?$AAI?$AAn?$AAt?$AAr?$AAH?$AAa?$AAn?$AAd?$AAl?$AAe?$AAr?$AA?$CL?$AA?5?$AA?3?$AA?5?$AAl?$AAe?$AAn?$AA?5?$AA?$CF?$AAd?$AA?4?$AA?5?$AAE?$AAv?$AAt?$AAC@ 10006418     serial_common_topaz_v1:serialhw.obj
 0001:00005470       ??_C@_1DK@FCFONANF@?$AAS?$AAL?$AA_?$AAT?$AAx?$AAI?$AAn?$AAt?$AAr?$AAH?$AAa?$AAn?$AAd?$AAl?$AAe?$AAr?$AA?9?$AA?5?$AAs?$AAe?$AAn?$AAt?$AA?5?$AA?$CF?$AAd?$AA?4?$AA?$AN?$AA?6?$AA?$AA@ 10006470     serial_common_topaz_v1:serialhw.obj
 0001:000054b0       ??_C@_1EI@DKJLIMCK@?$AAS?$AAL?$AA_?$AAT?$AAx?$AAI?$AAn?$AAt?$AAr?$AAH?$AAa?$AAn?$AAd?$AAl?$AAe?$AAr?$AA?3?$AA?5?$AAE?$AAn?$AAa?$AAb?$AAl?$AAe?$AA?5?$AAI?$AAN?$AAT?$AAR?$AA_?$AAT?$AAX@ 100064b0     serial_common_topaz_v1:serialhw.obj
 0001:000054f8       ??_C@_1FC@HKJLDPOK@?$AAS?$AAL?$AA_?$AAT?$AAx?$AAI?$AAn?$AAt?$AAr?$AAH?$AAa?$AAn?$AAd?$AAl?$AAe?$AAr?$AA?3?$AA?5?$AAN?$AAu?$AAm?$AAb?$AAe?$AAr?$AAO?$AAf?$AAB?$AAy?$AAt?$AAe?$AAs?$AA?5@ 100064f8     serial_common_topaz_v1:serialhw.obj
 0001:00005550       ??_C@_1FI@EJOAIGOC@?$AAS?$AAL?$AA_?$AAT?$AAx?$AAI?$AAn?$AAt?$AAr?$AAH?$AAa?$AAn?$AAd?$AAl?$AAe?$AAr?$AA?3?$AA?5?$AAS?$AAt?$AAa?$AAt?$AAu?$AAs?$AA?5?$AAb?$AAe?$AAf?$AAo?$AAr?$AAe?$AA?5@ 10006550     serial_common_topaz_v1:serialhw.obj
 0001:000055a8       ??_C@_1BI@ENEHIFAK@?$AAW?$AAr?$AAi?$AAt?$AAe?$AA?5?$AAx?$AA?$CF?$AAx?$AA?$AN?$AA?6?$AA?$AA@ 100065a8     serial_common_topaz_v1:serialhw.obj
 0001:000055c0       ??_C@_1GG@PEMDFIJB@?$AAS?$AAL?$AA_?$AAT?$AAx?$AAI?$AAn?$AAt?$AAr?$AAH?$AAa?$AAn?$AAd?$AAl?$AAe?$AAr?$AA?5?$AA?9?$AA?5?$AAW?$AAr?$AAi?$AAt?$AAe?$AA?5?$AAm?$AAa?$AAx?$AA?5?$AAo?$AAf?$AA?5@ 100065c0     serial_common_topaz_v1:serialhw.obj
 0001:00005628       ??_C@_1EK@NKDKOEDH@?$AAS?$AAL?$AA_?$AAT?$AAx?$AAI?$AAn?$AAt?$AAr?$AAH?$AAa?$AAn?$AAd?$AAl?$AAe?$AAr?$AA?5?$AA?3?$AAE?$AAx?$AAc?$AAe?$AAp?$AAt?$AAi?$AAo?$AAn?$AA?5?$AAc?$AAa?$AAu?$AAg@ 10006628     serial_common_topaz_v1:serialhw.obj
 0001:00005678       ??_C@_1EO@FBFLNOIJ@?$AAS?$AAL?$AA_?$AAT?$AAx?$AAI?$AAn?$AAt?$AAr?$AAH?$AAa?$AAn?$AAd?$AAl?$AAe?$AAr?$AA?5?$AA?9?$AA?5?$AAf?$AAO?$AAu?$AAt?$AAx?$AAD?$AAs?$AAr?$AAF?$AAl?$AAo?$AAw?$AA?5@ 10006678     serial_common_topaz_v1:serialhw.obj
 0001:000056c8       ??_C@_1EM@JOFDPOIO@?$AAS?$AAL?$AA_?$AAT?$AAx?$AAI?$AAn?$AAt?$AAr?$AAH?$AAa?$AAn?$AAd?$AAl?$AAe?$AAr?$AA?0?$AA?5?$AAf?$AAl?$AAo?$AAw?$AAe?$AAd?$AA?5?$AAo?$AAf?$AAf?$AA?5?$AAv?$AAi?$AAa@ 100066c8     serial_common_topaz_v1:serialhw.obj
 0001:00005718       ??_C@_1GE@GHMPINNH@?$AAS?$AAL?$AA_?$AAT?$AAx?$AAI?$AAn?$AAt?$AAr?$AAH?$AAa?$AAn?$AAd?$AAl?$AAe?$AAr?$AA?5?$AA?9?$AA?5?$AAf?$AAO?$AAu?$AAt?$AAx?$AAC?$AAt?$AAs?$AAF?$AAl?$AAo?$AAw?$AA?5@ 10006718     serial_common_topaz_v1:serialhw.obj
 0001:00005780       ??_C@_1EO@HGNCCHF@?$AAS?$AAL?$AA_?$AAT?$AAx?$AAI?$AAn?$AAt?$AAr?$AAH?$AAa?$AAn?$AAd?$AAl?$AAe?$AAr?$AA?5?$AA?9?$AA?5?$AAf?$AAO?$AAu?$AAt?$AAx?$AAC?$AAt?$AAs?$AAF?$AAl?$AAo?$AAw?$AA?5@ 10006780     serial_common_topaz_v1:serialhw.obj
 0001:000057d0       ??_C@_1EM@NLBBMEKN@?$AAS?$AAL?$AA_?$AAT?$AAx?$AAI?$AAn?$AAt?$AAr?$AAH?$AAa?$AAn?$AAd?$AAl?$AAe?$AAr?$AA?5?$AA?9?$AA?5?$AAD?$AAi?$AAs?$AAa?$AAb?$AAl?$AAe?$AA?5?$AAI?$AAN?$AAT?$AAR?$AA_@ 100067d0     serial_common_topaz_v1:serialhw.obj
 0001:0000581c       ??_C@_1DM@FCGGJKNG@?$AAT?$AAr?$AAa?$AAn?$AAs?$AAm?$AAi?$AAt?$AA?5?$AAE?$AAv?$AAe?$AAn?$AAt?$AA?5?$AA0?$AAx?$AA?$CF?$AAX?$AA?0?$AA?5?$AAL?$AAe?$AAn?$AA?5?$AA?$CF?$AAd?$AA?$AN?$AA?6?$AA?$AA@ 1000681c     serial_common_topaz_v1:serialhw.obj
 0001:00005858       ??_C@_1CI@NHMBGMLE@?$AAS?$AAL?$AA_?$AAT?$AAx?$AAI?$AAn?$AAt?$AAr?$AAH?$AAa?$AAn?$AAd?$AAl?$AAe?$AAr?$AA?$CL?$AA?$AN?$AA?6?$AA?$AA@ 10006858     serial_common_topaz_v1:serialhw.obj
 0001:00005880       ??_C@_1CO@PAGHMEGH@?$AAS?$AAL?$AA_?$AAM?$AAo?$AAd?$AAe?$AAm?$AAI?$AAn?$AAt?$AAr?$AAH?$AAa?$AAn?$AAd?$AAl?$AAe?$AAr?$AA?9?$AA?$AN?$AA?6?$AA?$AA@ 10006880     serial_common_topaz_v1:serialhw.obj
 0001:000058b0       ??_C@_1FA@EIIGAMCH@?$AAS?$AAL?$AA_?$AAM?$AAo?$AAd?$AAe?$AAm?$AAI?$AAn?$AAt?$AAr?$AAH?$AAa?$AAn?$AAd?$AAl?$AAe?$AAr?$AA?5?$AA?3?$AAE?$AAx?$AAc?$AAe?$AAp?$AAt?$AAi?$AAo?$AAn?$AA?5?$AAc@ 100068b0     serial_common_topaz_v1:serialhw.obj
 0001:00005900       ??_C@_1EG@IFDJOLIL@?$AAR?$AAS?$AA2?$AA3?$AA2?$AA?5?$AAd?$AAi?$AAs?$AAc?$AAo?$AAn?$AAn?$AAe?$AAc?$AAt?$AA?5?$AAn?$AAo?$AAt?$AAi?$AAf?$AAi?$AAc?$AAa?$AAt?$AAi?$AAo?$AAn?$AA?$CB?$AA?$CB?$AA?$CB@ 10006900     serial_common_topaz_v1:serialhw.obj
 0001:00005948       ??_C@_1FM@IMBGGKMM@?$AAS?$AAL?$AA_?$AAM?$AAo?$AAd?$AAe?$AAm?$AAI?$AAn?$AAt?$AAr?$AAH?$AAa?$AAn?$AAd?$AAl?$AAe?$AAr?$AA?5?$AA?9?$AA?5?$AAC?$AAT?$AAS?$AAF?$AAl?$AAo?$AAw?$AAO?$AAf?$AAf@ 10006948     serial_common_topaz_v1:serialhw.obj
 0001:000059a4       ??_C@_1DK@ENFMPLIO@?$AAP?$AAu?$AAt?$AAB?$AAy?$AAt?$AAe?$AAs?$AA?0?$AA?5?$AAf?$AAl?$AAo?$AAw?$AAe?$AAd?$AA?5?$AAo?$AAn?$AA?5?$AAv?$AAi?$AAa?$AA?5?$AAD?$AAS?$AAR?$AA?6?$AA?$AA@ 100069a4     serial_common_topaz_v1:serialhw.obj
 0001:000059e0       ??_C@_1CO@DGAIMNOA@?$AAS?$AAL?$AA_?$AAM?$AAo?$AAd?$AAe?$AAm?$AAI?$AAn?$AAt?$AAr?$AAH?$AAa?$AAn?$AAd?$AAl?$AAe?$AAr?$AA?$CL?$AA?$AN?$AA?6?$AA?$AA@ 100069e0     serial_common_topaz_v1:serialhw.obj
 0001:00005a10       ??_C@_1CO@MEPOPIOP@?$AAS?$AAL?$AA_?$AAL?$AAi?$AAn?$AAe?$AAI?$AAn?$AAt?$AAr?$AAH?$AAa?$AAn?$AAd?$AAl?$AAe?$AAr?$AA?9?$AA?5?$AA?$AN?$AA?6?$AA?$AA@ 10006a10     serial_common_topaz_v1:serialhw.obj
 0001:00005a40       ??_C@_1CO@MJOAIIKI@?$AAS?$AAL?$AA_?$AAL?$AAi?$AAn?$AAe?$AAI?$AAn?$AAt?$AAr?$AAH?$AAa?$AAn?$AAd?$AAl?$AAe?$AAr?$AA?$CL?$AA?5?$AA?$AN?$AA?6?$AA?$AA@ 10006a40     serial_common_topaz_v1:serialhw.obj
 0001:00005a70       ??_C@_1BO@LAOLELIF@?$AAS?$AAL?$AA_?$AAC?$AAl?$AAe?$AAa?$AAr?$AAD?$AAT?$AAR?$AA?9?$AA?$AN?$AA?6?$AA?$AA@ 10006a70     serial_common_topaz_v1:serialhw.obj
 0001:00005a90       ??_C@_1EA@MJGPCAPJ@?$AAS?$AAL?$AA_?$AAC?$AAl?$AAe?$AAa?$AAr?$AAD?$AAT?$AAR?$AA?5?$AA?3?$AAE?$AAx?$AAc?$AAe?$AAp?$AAt?$AAi?$AAo?$AAn?$AA?5?$AAc?$AAa?$AAu?$AAg?$AAh?$AAt?$AA?5?$AA?6?$AA?$AA@ 10006a90     serial_common_topaz_v1:serialhw.obj
 0001:00005ad0       ??_C@_1BO@HGIEECAC@?$AAS?$AAL?$AA_?$AAC?$AAl?$AAe?$AAa?$AAr?$AAD?$AAT?$AAR?$AA?$CL?$AA?$AN?$AA?6?$AA?$AA@ 10006ad0     serial_common_topaz_v1:serialhw.obj
 0001:00005af0       ??_C@_1BK@PHBAGCPN@?$AAS?$AAL?$AA_?$AAS?$AAe?$AAt?$AAD?$AAT?$AAR?$AA?9?$AA?$AN?$AA?6?$AA?$AA@ 10006af0     serial_common_topaz_v1:serialhw.obj
 0001:00005b0c       ??_C@_1DM@EJBPBCKH@?$AAS?$AAL?$AA_?$AAS?$AAe?$AAt?$AAD?$AAT?$AAR?$AA?5?$AA?3?$AAE?$AAx?$AAc?$AAe?$AAp?$AAt?$AAi?$AAo?$AAn?$AA?5?$AAc?$AAa?$AAu?$AAg?$AAh?$AAt?$AA?5?$AA?6?$AA?$AA@ 10006b0c     serial_common_topaz_v1:serialhw.obj
 0001:00005b48       ??_C@_1BK@DBHPGLHK@?$AAS?$AAL?$AA_?$AAS?$AAe?$AAt?$AAD?$AAT?$AAR?$AA?$CL?$AA?$AN?$AA?6?$AA?$AA@ 10006b48     serial_common_topaz_v1:serialhw.obj
 0001:00005b64       ??_C@_1CA@IBKBMKHP@?$AA?9?$AAS?$AAL?$AA_?$AAC?$AAl?$AAe?$AAa?$AAr?$AAR?$AAT?$AAS?$AA?9?$AA?$AN?$AA?6?$AA?$AA@ 10006b64     serial_common_topaz_v1:serialhw.obj
 0001:00005b88       ??_C@_1EA@DBPLDBB@?$AAS?$AAL?$AA_?$AAC?$AAl?$AAe?$AAa?$AAr?$AAR?$AAT?$AAS?$AA?5?$AA?3?$AAE?$AAx?$AAc?$AAe?$AAp?$AAt?$AAi?$AAo?$AAn?$AA?5?$AAc?$AAa?$AAu?$AAg?$AAh?$AAt?$AA?5?$AA?6?$AA?$AA@ 10006b88     serial_common_topaz_v1:serialhw.obj
 0001:00005bc8       ??_C@_1BO@HDGFOOG@?$AAS?$AAL?$AA_?$AAC?$AAl?$AAe?$AAa?$AAr?$AAR?$AAT?$AAS?$AA?$CL?$AA?$AN?$AA?6?$AA?$AA@ 10006bc8     serial_common_topaz_v1:serialhw.obj
 0001:00005be8       ??_C@_1BK@IGKCHOBJ@?$AAS?$AAL?$AA_?$AAS?$AAe?$AAt?$AAR?$AAT?$AAS?$AA?9?$AA?$AN?$AA?6?$AA?$AA@ 10006be8     serial_common_topaz_v1:serialhw.obj
 0001:00005c04       ??_C@_1DM@IDGPIBEP@?$AAS?$AAL?$AA_?$AAS?$AAe?$AAt?$AAR?$AAT?$AAS?$AA?5?$AA?3?$AAE?$AAx?$AAc?$AAe?$AAp?$AAt?$AAi?$AAo?$AAn?$AA?5?$AAc?$AAa?$AAu?$AAg?$AAh?$AAt?$AA?5?$AA?6?$AA?$AA@ 10006c04     serial_common_topaz_v1:serialhw.obj
 0001:00005c40       ??_C@_1BK@EAMNHHJO@?$AAS?$AAL?$AA_?$AAS?$AAe?$AAt?$AAR?$AAT?$AAS?$AA?$CL?$AA?$AN?$AA?6?$AA?$AA@ 10006c40     serial_common_topaz_v1:serialhw.obj
 0001:00005c5c       ??_C@_1CC@JNGKOLFI@?$AAS?$AAL?$AA_?$AAC?$AAl?$AAe?$AAa?$AAr?$AAB?$AAr?$AAe?$AAa?$AAk?$AA?9?$AA?$AN?$AA?6?$AA?$AA@ 10006c5c     serial_common_topaz_v1:serialhw.obj
 0001:00005c80       ??_C@_1EE@ILPIGOPO@?$AAS?$AAL?$AA_?$AAC?$AAl?$AAe?$AAa?$AAr?$AAB?$AAr?$AAe?$AAa?$AAk?$AA?5?$AA?3?$AAE?$AAx?$AAc?$AAe?$AAp?$AAt?$AAi?$AAo?$AAn?$AA?5?$AAc?$AAa?$AAu?$AAg?$AAh?$AAt?$AA?5@ 10006c80     serial_common_topaz_v1:serialhw.obj
 0001:00005cc4       ??_C@_1CC@FLAFOCNP@?$AAS?$AAL?$AA_?$AAC?$AAl?$AAe?$AAa?$AAr?$AAB?$AAr?$AAe?$AAa?$AAk?$AA?$CL?$AA?$AN?$AA?6?$AA?$AA@ 10006cc4     serial_common_topaz_v1:serialhw.obj
 0001:00005ce8       ??_C@_1BO@BLINPCAB@?$AAS?$AAL?$AA_?$AAS?$AAe?$AAt?$AAB?$AAr?$AAe?$AAa?$AAk?$AA?9?$AA?$AN?$AA?6?$AA?$AA@ 10006ce8     serial_common_topaz_v1:serialhw.obj
 0001:00005d08       ??_C@_1EA@EFECNNEH@?$AAS?$AAL?$AA_?$AAS?$AAe?$AAt?$AAB?$AAr?$AAe?$AAa?$AAk?$AA?5?$AA?3?$AAE?$AAx?$AAc?$AAe?$AAp?$AAt?$AAi?$AAo?$AAn?$AA?5?$AAc?$AAa?$AAu?$AAg?$AAh?$AAt?$AA?5?$AA?6?$AA?$AA@ 10006d08     serial_common_topaz_v1:serialhw.obj
 0001:00005d48       ??_C@_1BO@NNOCPLIG@?$AAS?$AAL?$AA_?$AAS?$AAe?$AAt?$AAB?$AAr?$AAe?$AAa?$AAk?$AA?$CL?$AA?$AN?$AA?6?$AA?$AA@ 10006d48     serial_common_topaz_v1:serialhw.obj
 0001:00005d68       ??_C@_1CE@CBOOMMIE@?$AAS?$AAL?$AA_?$AAX?$AAm?$AAi?$AAt?$AAC?$AAo?$AAm?$AAC?$AAh?$AAa?$AAr?$AA?9?$AA?$AN?$AA?6?$AA?$AA@ 10006d68     serial_common_topaz_v1:serialhw.obj
 0001:00005d90       ??_C@_1EG@GLCEIKAG@?$AAS?$AAL?$AA_?$AAX?$AAm?$AAi?$AAt?$AAC?$AAo?$AAm?$AAC?$AAh?$AAa?$AAr?$AA?5?$AA?3?$AAE?$AAx?$AAc?$AAe?$AAp?$AAt?$AAi?$AAo?$AAn?$AA?5?$AAc?$AAa?$AAu?$AAg?$AAh?$AAt@ 10006d90     serial_common_topaz_v1:serialhw.obj
 0001:00005dd8       ??_C@_1CC@FKNGPPMN@?$AAS?$AAL?$AA_?$AAX?$AAm?$AAi?$AAt?$AAC?$AAo?$AAm?$AAC?$AAh?$AAa?$AAr?$AA?9?$AA?6?$AA?$AA@ 10006dd8     serial_common_topaz_v1:serialhw.obj
 0001:00005dfc       ??_C@_1CA@LOKJHMKJ@?$AAS?$AAL?$AA_?$AAG?$AAe?$AAt?$AAS?$AAt?$AAa?$AAt?$AAu?$AAs?$AA?9?$AA?$AN?$AA?6?$AA?$AA@ 10006dfc     serial_common_topaz_v1:serialhw.obj
 0001:00005e20       ??_C@_1EC@MCFHKKAH@?$AAS?$AAL?$AA_?$AAG?$AAe?$AAt?$AAS?$AAt?$AAa?$AAt?$AAu?$AAs?$AA?5?$AA?3?$AAE?$AAx?$AAc?$AAe?$AAp?$AAt?$AAi?$AAo?$AAn?$AA?5?$AAc?$AAa?$AAu?$AAg?$AAh?$AAt?$AA?5?$AA?6@ 10006e20     serial_common_topaz_v1:serialhw.obj
 0001:00005e64       ??_C@_1CA@HIMGHFCO@?$AAS?$AAL?$AA_?$AAG?$AAe?$AAt?$AAS?$AAt?$AAa?$AAt?$AAu?$AAs?$AA?$CL?$AA?$AN?$AA?6?$AA?$AA@ 10006e64     serial_common_topaz_v1:serialhw.obj
 0001:00005e88       ??_C@_1EC@DJGKKHLM@?$AAS?$AAL?$AA_?$AAG?$AAe?$AAt?$AAM?$AAo?$AAd?$AAe?$AAm?$AAS?$AAt?$AAa?$AAt?$AAu?$AAs?$AA?9?$AA?$CI?$AAs?$AAt?$AAa?$AAt?$AA?5?$AA0?$AAx?$AA?$CF?$AAX?$AA?$CJ?$AA?5?$AA?$AN?$AA?6@ 10006e88     serial_common_topaz_v1:serialhw.obj
 0001:00005ecc       ??_C@_1BK@LHPJEBK@?$AAM?$AAS?$AA_?$AAR?$AAI?$AAN?$AAG?$AA_?$AAO?$AAN?$AA?$AN?$AA?6?$AA?$AA@ 10006ecc     serial_common_topaz_v1:serialhw.obj
 0001:00005ee8       ??_C@_1BK@HMIJKMOB@?$AAM?$AAS?$AA_?$AAR?$AAL?$AAS?$AAD?$AA_?$AAO?$AAN?$AA?$AN?$AA?6?$AA?$AA@ 10006ee8     serial_common_topaz_v1:serialhw.obj
 0001:00005f04       ??_C@_1BI@OLBHNJIN@?$AAM?$AAS?$AA_?$AAD?$AAS?$AAR?$AA_?$AAO?$AAN?$AA?$AN?$AA?6?$AA?$AA@ 10006f04     serial_common_topaz_v1:serialhw.obj
 0001:00005f1c       ??_C@_1BI@GKMPMKOK@?$AAM?$AAS?$AA_?$AAC?$AAT?$AAS?$AA_?$AAO?$AAN?$AA?$AN?$AA?6?$AA?$AA@ 10006f1c     serial_common_topaz_v1:serialhw.obj
 0001:00005f34       ??_C@_1CK@GPPJFAGP@?$AAS?$AAL?$AA_?$AAG?$AAe?$AAt?$AAM?$AAo?$AAd?$AAe?$AAm?$AAS?$AAt?$AAa?$AAt?$AAu?$AAs?$AA?$CL?$AA?$AN?$AA?6?$AA?$AA@ 10006f34     serial_common_topaz_v1:serialhw.obj
 0001:00005f60       ??_C@_1CC@JPEAAJCH@?$AAS?$AAL?$AA_?$AAP?$AAu?$AAr?$AAg?$AAe?$AAC?$AAo?$AAm?$AAm?$AA?9?$AA?5?$AA?$AN?$AA?6?$AA?$AA@ 10006f60     serial_common_topaz_v1:serialhw.obj
 0001:00005f88       ??_C@_1EC@GDIDBILI@?$AAS?$AAL?$AA_?$AAP?$AAu?$AAr?$AAg?$AAe?$AAC?$AAo?$AAm?$AAm?$AA?5?$AA?3?$AAE?$AAx?$AAc?$AAe?$AAp?$AAt?$AAi?$AAo?$AAn?$AA?5?$AAc?$AAa?$AAu?$AAg?$AAh?$AAt?$AA?5?$AA?6@ 10006f88     serial_common_topaz_v1:serialhw.obj
 0001:00005fcc       ??_C@_1CA@NOGEKKLI@?$AAP?$AAU?$AAR?$AAG?$AAE?$AA_?$AAR?$AAX?$AAC?$AAL?$AAE?$AAA?$AAR?$AA?$AN?$AA?6?$AA?$AA@ 10006fcc     serial_common_topaz_v1:serialhw.obj
 0001:00005fec       ??_C@_1CA@FKEHDHGN@?$AAP?$AAU?$AAR?$AAG?$AAE?$AA_?$AAT?$AAX?$AAC?$AAL?$AAE?$AAA?$AAR?$AA?$AN?$AA?6?$AA?$AA@ 10006fec     serial_common_topaz_v1:serialhw.obj
 0001:0000600c       ??_C@_1CA@PIINPJIF@?$AAS?$AAL?$AA_?$AAP?$AAu?$AAr?$AAg?$AAe?$AAC?$AAo?$AAm?$AAm?$AA?$CL?$AA?$AN?$AA?6?$AA?$AA@ 1000700c     serial_common_topaz_v1:serialhw.obj
 0001:0000602c       ??_C@_1CM@DNIFDBOB@?$AAS?$AAL?$AA_?$AAS?$AAe?$AAt?$AAD?$AAC?$AAB?$AA?9?$AA?5?$AAR?$AAe?$AAt?$AA?5?$AA?$DN?$AA?5?$AA?$CF?$AAd?$AA?$AN?$AA?6?$AA?$AA@ 1000702c     serial_common_topaz_v1:serialhw.obj
 0001:00006058       ??_C@_1BK@BOMJNNAN@?$AAS?$AAL?$AA_?$AAS?$AAe?$AAt?$AAD?$AAC?$AA?$CL?$AA?5?$AA?$AN?$AA?6?$AA?$AA@ 10007058     serial_common_topaz_v1:serialhw.obj
 0001:00006074       ??_C@_1CK@EKGBFFFP@?$AAS?$AAL?$AA_?$AAS?$AAe?$AAt?$AAC?$AAo?$AAm?$AAm?$AAT?$AAi?$AAm?$AAe?$AAo?$AAu?$AAt?$AA?9?$AA?$AN?$AA?6?$AA?$AA@ 10007074     serial_common_topaz_v1:serialhw.obj
 0001:000060a0       ??_C@_1CM@DLPHHJJN@?$AAS?$AAL?$AA_?$AAS?$AAe?$AAt?$AAC?$AAo?$AAm?$AAm?$AAT?$AAi?$AAm?$AAe?$AAo?$AAu?$AAt?$AA?$CL?$AA?5?$AA?$AN?$AA?6?$AA?$AA@ 100070a0     serial_common_topaz_v1:serialhw.obj
 0001:000060d0       ??_C@_1FC@EMENGKEI@?$AAS?$AAl?$AA_?$AAI?$AAO?$AAC?$AAo?$AAn?$AAt?$AAr?$AAo?$AAl?$AA?3?$AAU?$AAn?$AAs?$AAu?$AAp?$AAp?$AAo?$AAr?$AAt?$AAe?$AAd?$AA?5?$AAI?$AAO?$AAC?$AAT?$AAL?$AA?5?$AAc@ 100070d0     serial_common_topaz_v1:serialhw.obj
 0001:00006124       ??_C@_1CK@NJIGBENJ@?$AAS?$AAL?$AA_?$AAI?$AAO?$AAC?$AAT?$AAL?$AA_?$AAP?$AAO?$AAW?$AAE?$AAR?$AA_?$AAG?$AAE?$AAT?$AA?$AN?$AA?6?$AA?$AA@ 10007124     serial_common_topaz_v1:serialhw.obj
 0001:00006150       ??_C@_1BK@HEFCAJFH@?$AAC?$AAu?$AAr?$AAD?$AAx?$AA?5?$AA?$DN?$AA?5?$AA?$CF?$AAd?$AA?$AN?$AA?6?$AA?$AA@ 10007150     serial_common_topaz_v1:serialhw.obj
 0001:0000616c       ??_C@_1BK@MINAOBBM@?$AAS?$AAE?$AAR?$AAI?$AAA?$AAL?$AA?5?$AAO?$AAf?$AAf?$AA?$AN?$AA?6?$AA?$AA@ 1000716c     serial_common_topaz_v1:serialhw.obj
 0001:00006188       ??_C@_1BK@HOPLIAJK@?$AAS?$AAE?$AAR?$AAI?$AAA?$AAL?$AA?5?$AAO?$AAF?$AAF?$AA?$AN?$AA?6?$AA?$AA@ 10007188     serial_common_topaz_v1:serialhw.obj
 0001:000061a4       ??_C@_1CK@NGJIMCFK@?$AAS?$AAL?$AA_?$AAI?$AAO?$AAC?$AAT?$AAL?$AA_?$AAP?$AAO?$AAW?$AAE?$AAR?$AA_?$AAS?$AAE?$AAT?$AA?$AN?$AA?6?$AA?$AA@ 100071a4     serial_common_topaz_v1:serialhw.obj
 0001:000061d0       ??_C@_1DK@EDBLHBKN@?$AAS?$AAL?$AA_?$AAI?$AAO?$AAC?$AAT?$AAL?$AA_?$AAP?$AAO?$AAW?$AAE?$AAR?$AA_?$AAQ?$AAU?$AAE?$AAR?$AAY?$AA?5?$AA?$CF?$AAu?$AA?5?$AA?$CF?$AAs?$AA?$AN?$AA?6?$AA?$AA@ 100071d0     serial_common_topaz_v1:serialhw.obj
 0001:0000620c       ??_C@_1O@KPGHAGDD@?$AAf?$AAa?$AAi?$AAl?$AAe?$AAd?$AA?$AA@ 1000720c     serial_common_topaz_v1:serialhw.obj
 0001:0000621c       ??_C@_1BE@GCAFJAHI@?$AAs?$AAu?$AAc?$AAc?$AAe?$AAe?$AAd?$AAe?$AAd?$AA?$AA@ 1000721c     serial_common_topaz_v1:serialhw.obj
 0001:00006230       ??_C@_1BK@NIBAJMFP@?$AAN?$AAe?$AAw?$AAD?$AAx?$AA?5?$AA?$DN?$AA?5?$AA?$CF?$AAd?$AA?$AN?$AA?6?$AA?$AA@ 10007230     serial_common_topaz_v1:serialhw.obj
 0001:0000624c       ??_C@_1CO@NGIJLINN@?$AAS?$AAL?$AA_?$AAI?$AAO?$AAC?$AAT?$AAL?$AA_?$AAP?$AAO?$AAW?$AAE?$AAR?$AA_?$AAQ?$AAU?$AAE?$AAR?$AAY?$AA?$AN?$AA?6?$AA?$AA@ 1000724c     serial_common_topaz_v1:serialhw.obj
 0001:0000627c       ??_C@_1DM@FHEEOGHJ@?$AAS?$AAL?$AA_?$AAI?$AAO?$AAC?$AAT?$AAL?$AA_?$AAP?$AAO?$AAW?$AAE?$AAR?$AA_?$AAC?$AAA?$AAP?$AAA?$AAB?$AAI?$AAL?$AAI?$AAT?$AAI?$AAE?$AAS?$AA?$AN?$AA?6?$AA?$AA@ 1000727c     serial_common_topaz_v1:serialhw.obj
 0001:000062e0       BSPUartCalRFDIV            100072e0 f   bspserial.obj
 0001:000063c4       BSPUartGetType             100073c4 f   bspserial.obj
 0001:000064e8       BSPUartEnableClock         100074e8 f   bspserial.obj
 0001:00006624       BSPUartConfigTranceiver    10007624 f   bspserial.obj
 0001:00006634       BSPUartConfigureGPIO       10007634 f   bspserial.obj
 0001:00006890       BSPSerGetChannelPriority   10007890 f   bspserial.obj
 0001:000068a8       BSPSerGetDMAIsEnabled      100078a8 f   bspserial.obj
 0001:00006994       BSPSerGetDMARequest        10007994 f   bspserial.obj
 0001:00006ad8       BSPSerAcquireDMAReqGpr     10007ad8 f   bspserial.obj
 0001:00006b04       BSPSerRestoreDMAReqGpr     10007b04 f   bspserial.obj
 0001:00006b30       GetSdmaChannelIRQ          10007b30 f   bspserial.obj
 0001:00006b58       BSPGetDMABuffSize          10007b58 f   bspserial.obj
 0001:00006b80       DllEntry                   10007b80 f   com_mdd2:mdd.obj
 0001:00006c34       DoTxData                   10007c34 f   com_mdd2:mdd.obj
 0001:00007130       SerialEventHandler         10008130 f   com_mdd2:mdd.obj
 0001:00007c4c       StartDispatchThread        10008c4c f   com_mdd2:mdd.obj
 0001:00008064       StopDispatchThread         10009064 f   com_mdd2:mdd.obj
 0001:00008248       ApplyDCB                   10009248 f   com_mdd2:mdd.obj
 0001:00008828       COM_Init                   10009828 f   com_mdd2:mdd.obj
 0001:0000915c       COM_Open                   1000a15c f   com_mdd2:mdd.obj
 0001:00009c8c       COM_PreClose               1000ac8c f   com_mdd2:mdd.obj
 0001:00009f30       COM_Close                  1000af30 f   com_mdd2:mdd.obj
 0001:0000a380       ProcessExiting             1000b380 f   com_mdd2:mdd.obj
 0001:0000a490       COM_PreDeinit              1000b490 f   com_mdd2:mdd.obj
 0001:0000a720       COM_Deinit                 1000b720 f   com_mdd2:mdd.obj
 0001:0000aad8       COM_Read                   1000bad8 f   com_mdd2:mdd.obj
 0001:0000b618       COM_Write                  1000c618 f   com_mdd2:mdd.obj
 0001:0000bf08       COM_Seek                   1000cf08 f   com_mdd2:mdd.obj
 0001:0000bf2c       COM_PowerUp                1000cf2c f   com_mdd2:mdd.obj
 0001:0000bfb4       COM_PowerDown              1000cfb4 f   com_mdd2:mdd.obj
 0001:0000c03c       SerialGetDroppedByteNumber 1000d03c f   com_mdd2:mdd.obj
 0001:0000c0a0       WaitCommEvent_mdd          1000d0a0 f   com_mdd2:mdd.obj
 0001:0000c4b0       EvaluateEventFlag          1000d4b0 f   com_mdd2:mdd.obj
 0001:0000c6c4       COM_IOControl              1000d6c4 f   com_mdd2:mdd.obj
 0001:0000e330       SetEvent                   1000f330 f i com_mdd2:mdd.obj
 0001:0000e364       RxBytesAvail               1000f364 f i com_mdd2:mdd.obj
 0001:0000e3ec       GetCurrentThread           1000f3ec f i com_mdd2:mdd.obj
 0001:0000e404       InitializeListHead         1000f404 f i com_mdd2:mdd.obj
 0001:0000e444       RemoveEntryList            1000f444 f i com_mdd2:mdd.obj
 0001:0000e4b8       CheckListEntry             1000f4b8 f i com_mdd2:mdd.obj
 0001:0000e660       InsertHeadList             1000f660 f i com_mdd2:mdd.obj
 0001:0000e684       InsertEntryList            1000f684 f i com_mdd2:mdd.obj
 0001:0000e714       ResetEvent                 1000f714 f i com_mdd2:mdd.obj
 0001:0000e748       PulseEvent                 1000f748 f i com_mdd2:mdd.obj
 0001:0000e77c       DisableThreadLibraryCalls  1000f77c f   coredll:COREDLL.dll
 0001:0000e78c       NKDbgPrintfW               1000f78c f   coredll:COREDLL.dll
 0001:0000e79c       RegisterDbgZones           1000f79c f   coredll:COREDLL.dll
 0001:0000e7ac       LeaveCriticalSection       1000f7ac f   coredll:COREDLL.dll
 0001:0000e7bc       EnterCriticalSection       1000f7bc f   coredll:COREDLL.dll
 0001:0000e7cc       EventModify                1000f7cc f   coredll:COREDLL.dll
 0001:0000e7dc       InterlockedDecrement       1000f7dc f   coredll:COREDLL.dll
 0001:0000e7ec       InterlockedCompareExchange 1000f7ec f   coredll:COREDLL.dll
 0001:0000e7fc       InterlockedIncrement       1000f7fc f   coredll:COREDLL.dll
 0001:0000e80c       ExitThread                 1000f80c f   coredll:COREDLL.dll
 0001:0000e81c       GetLastError               1000f81c f   coredll:COREDLL.dll
 0001:0000e82c       CreateThread               1000f82c f   coredll:COREDLL.dll
 0001:0000e83c       InterruptDone              1000f83c f   coredll:COREDLL.dll
 0001:0000e84c       InterruptInitialize        1000f84c f   coredll:COREDLL.dll
 0001:0000e85c       WaitForSingleObject        1000f85c f   coredll:COREDLL.dll
 0001:0000e86c       Sleep                      1000f86c f   coredll:COREDLL.dll
 0001:0000e87c       InterruptDisable           1000f87c f   coredll:COREDLL.dll
 0001:0000e88c       CloseHandle                1000f88c f   coredll:COREDLL.dll
 0001:0000e89c       CeSetThreadPriority        1000f89c f   coredll:COREDLL.dll
 0001:0000e8ac       CeGetThreadPriority        1000f8ac f   coredll:COREDLL.dll
 0001:0000e8bc       RegCloseKey                1000f8bc f   coredll:COREDLL.dll
 0001:0000e8cc       RegQueryValueExW           1000f8cc f   coredll:COREDLL.dll
 0001:0000e8dc       OpenDeviceKey              1000f8dc f   coredll:COREDLL.dll
 0001:0000e8ec       CreateEventW               1000f8ec f   coredll:COREDLL.dll
 0001:0000e8fc       InitializeCriticalSection  1000f8fc f   coredll:COREDLL.dll
 0001:0000e90c       LocalAlloc                 1000f90c f   coredll:COREDLL.dll
 0001:0000e91c       LocalFree                  1000f91c f   coredll:COREDLL.dll
 0001:0000e92c       DeleteCriticalSection      1000f92c f   coredll:COREDLL.dll
 0001:0000e93c       SetLastError               1000f93c f   coredll:COREDLL.dll
 0001:0000e94c       SetThreadPriority          1000f94c f   coredll:COREDLL.dll
 0001:0000e95c       GetTickCount               1000f95c f   coredll:COREDLL.dll
 0001:0000e96c       CeSafeCopyMemory           1000f96c f   coredll:COREDLL.dll
 0001:0000e97c       CeFreeAsynchronousBuffer   1000f97c f   coredll:COREDLL.dll
 0001:0000e98c       CeAllocAsynchronousBuffer  1000f98c f   coredll:COREDLL.dll
 0001:0000e99c       InterlockedExchange        1000f99c f   coredll:COREDLL.dll
 0001:0000e9ac       DDKClockGetFreq            1000f9ac f   cspddk:CSPDDK.dll
 0001:0000e9bc       DDKClockSetGatingMode      1000f9bc f   cspddk:CSPDDK.dll
 0001:0000e9cc       DDKIomuxSelectInput        1000f9cc f   cspddk:CSPDDK.dll
 0001:0000e9dc       DDKIomuxSetPinMux          1000f9dc f   cspddk:CSPDDK.dll
 0001:0000e9ec       _DllEntryCRTStartup        1000f9ec f   corelib0:pegdentry.obj
 0001:0000ea58       __security_init_cookie     1000fa58 f   corelib0:seccinit.obj
 0001:0000eaf0       __GSHandlerCheck           1000faf0 f   corelib0:gshandler.obj
 0001:0000eb34       __GSHandlerCheckCommon     1000fb34 f   corelib0:gshandler.obj
 0001:0000ebd8       __security_check_cookie    1000fbd8 f   corelib0:armsecgs.obj
 0001:0000ebe8       __gsfailure                1000fbe8     corelib0:armsecgs.obj
 0001:0000ec2c       exit                       1000fc2c f   corelib0:cexit.obj
 0001:0000ed50       _exit                      1000fd50 f   corelib0:cexit.obj
 0001:0000ed70       _cexit                     1000fd70 f   corelib0:cexit.obj
 0001:0000ed88       _c_exit                    1000fd88 f   corelib0:cexit.obj
 0001:0000eda0       _initterm                  1000fda0 f   corelib0:crt0dat.obj
 0001:0000edec       _cinit                     1000fdec f   corelib0:crt0dat.obj
 0001:0000ee1c       __crt_ExitProcess          1000fe1c f   corelib0:exitproc_proxy.obj
 0001:0000ee48       GetCurrentProcess          1000fe48 f i corelib0:exitproc_proxy.obj
 0001:0000ee60       _onexit                    1000fe60 f   corelib0:onexit.obj
 0001:0000f03c       atexit                     1001003c f   corelib0:onexit.obj
 0001:0000f08c       __rt_udiv                  1001008c f   corelib1:COREDLL.dll
 0001:0000f09c       memmove                    1001009c f   corelib1:COREDLL.dll
 0001:0000f0ac       memcpy                     100100ac f   corelib1:COREDLL.dll
 0001:0000f0bc       memset                     100100bc f   corelib1:COREDLL.dll
 0001:0000f0cc       __C_specific_handler       100100cc f   corelib1:COREDLL.dll
 0001:0000f0dc       __security_gen_cookie2     100100dc f   corelib1:COREDLL.dll
 0001:0000f0ec       __report_gsfailure         100100ec f   corelib1:COREDLL.dll
 0001:0000f0fc       free                       100100fc f   corelib1:COREDLL.dll
 0001:0000f10c       realloc                    1001010c f   corelib1:COREDLL.dll
 0001:0000f11c       malloc                     1001011c f   corelib1:COREDLL.dll
 0001:0000f12c       _msize                     1001012c f   corelib1:COREDLL.dll
 0001:0000f13c       MapDMABuffers              1001013c f   serial_common_topaz_v1:serial.obj
 0001:0000f344       UnmapDMABuffers            10010344 f   serial_common_topaz_v1:serial.obj
 0001:0000f47c       DeinitChannelDMA           1001047c f   serial_common_topaz_v1:serial.obj
 0001:0000f514       InitChannelDMA             10010514 f   serial_common_topaz_v1:serial.obj
 0001:0000f7f0       InitDMA                    100107f0 f   serial_common_topaz_v1:serial.obj
 0001:0000f9bc       DeInitDMA                  100109bc f   serial_common_topaz_v1:serial.obj
 0001:00010eb8       SerIRClearDTR              10011eb8 f   serial_common_topaz_v1:serial.obj
 0001:00010f04       SerIRSetDTR                10011f04 f   serial_common_topaz_v1:serial.obj
 0001:00010f50       SerIRClearRTS              10011f50 f   serial_common_topaz_v1:serial.obj
 0001:00010f9c       SerIRSetRTS                10011f9c f   serial_common_topaz_v1:serial.obj
 0001:00010fe8       GetSerialObject            10011fe8 f   serial_common_topaz_v1:serial.obj
 0001:000110f8       SerialSetMux               100120f8 f   serial_common_topaz_v1:serialhw.obj
 0001:0001112c       SL_CalculateRFDIV          1001212c f   serial_common_topaz_v1:serialhw.obj
 0001:0001119c       SL_ReadModemStatus         1001219c f   serial_common_topaz_v1:serialhw.obj
 0001:00011514       SL_ReadLineStatus          10012514 f   serial_common_topaz_v1:serialhw.obj
 0001:000118c4       SL_SetOutputMode           100128c4 f   serial_common_topaz_v1:serialhw.obj
 0001:000119c0       SL_ClearPendingInts        100129c0 f   serial_common_topaz_v1:serialhw.obj
 0001:00011b14       SL_SetStopBits             10012b14 f   serial_common_topaz_v1:serialhw.obj
 0001:00011da0       SL_SetBaudRate             10012da0 f   serial_common_topaz_v1:serialhw.obj
 0001:00012070       SL_SetByteSize             10013070 f   serial_common_topaz_v1:serialhw.obj
 0001:000122e8       SL_SetParity               100132e8 f   serial_common_topaz_v1:serialhw.obj
 0001:00012608       SL_SetFlowControl          10013608 f   serial_common_topaz_v1:serialhw.obj
 0001:000128dc       SL_Reset                   100138dc f   serial_common_topaz_v1:serialhw.obj
 0001:00012ba4       SL_Init                    10013ba4 f   serial_common_topaz_v1:serialhw.obj
 0001:00012d0c       SL_Deinit                  10013d0c f   serial_common_topaz_v1:serialhw.obj
 0001:00012f7c       SL_Open                    10013f7c f   serial_common_topaz_v1:serialhw.obj
 0001:00013884       SL_Close                   10014884 f   serial_common_topaz_v1:serialhw.obj
 0001:00013d1c       SL_PowerOff                10014d1c f   serial_common_topaz_v1:serialhw.obj
 0001:00013dc8       SL_PowerOn                 10014dc8 f   serial_common_topaz_v1:serialhw.obj
 0001:00013e90       SL_GetIntrType             10014e90 f   serial_common_topaz_v1:serialhw.obj
 0001:000145fc       SL_RxIntrHandler           100155fc f   serial_common_topaz_v1:serialhw.obj
 0001:00015174       SL_TxIntrHandler           10016174 f   serial_common_topaz_v1:serialhw.obj
 0001:00015b60       SL_ModemIntrHandler        10016b60 f   serial_common_topaz_v1:serialhw.obj
 0001:00015ec4       SL_LineIntrHandler         10016ec4 f   serial_common_topaz_v1:serialhw.obj
 0001:00015f48       SL_GetRxBufferSize         10016f48 f   serial_common_topaz_v1:serialhw.obj
 0001:00015f74       SL_ClearDTR                10016f74 f   serial_common_topaz_v1:serialhw.obj
 0001:000160c0       SL_SetDTR                  100170c0 f   serial_common_topaz_v1:serialhw.obj
 0001:00016210       SL_ClearRTS                10017210 f   serial_common_topaz_v1:serialhw.obj
 0001:000163b0       SL_SetRTS                  100173b0 f   serial_common_topaz_v1:serialhw.obj
 0001:0001658c       SL_ClearBreak              1001758c f   serial_common_topaz_v1:serialhw.obj
 0001:000166d8       SL_SetBreak                100176d8 f   serial_common_topaz_v1:serialhw.obj
 0001:00016828       SL_XmitComChar             10017828 f   serial_common_topaz_v1:serialhw.obj
 0001:00016a30       SL_GetStatus               10017a30 f   serial_common_topaz_v1:serialhw.obj
 0001:00016c5c       SL_GetModemStatus          10017c5c f   serial_common_topaz_v1:serialhw.obj
 0001:00016e60       SL_PurgeComm               10017e60 f   serial_common_topaz_v1:serialhw.obj
 0001:00016ff4       SL_SetDCB                  10017ff4 f   serial_common_topaz_v1:serialhw.obj
 0001:0001735c       SL_SetCommTimeouts         1001835c f   serial_common_topaz_v1:serialhw.obj
 0001:00017408       SL_Ioctl                   10018408 f   serial_common_topaz_v1:serialhw.obj
 0001:000179d0       HalAllocateCommonBuffer    100189d0 f   ceddk:CEDDK.dll
 0001:000179e0       HalFreeCommonBuffer        100189e0 f   ceddk:CEDDK.dll
 0001:000179f0       MmUnmapIoSpace             100189f0 f   ceddk:CEDDK.dll
 0001:00017a00       MmMapIoSpace               10018a00 f   ceddk:CEDDK.dll
 0001:00017a10       HalTranslateBusAddress     10018a10 f   ceddk:CEDDK.dll
 0001:00017a20       TerminateProcess           10018a20 f   coredll:COREDLL.dll
 0001:00017a30       KernelIoControl            10018a30 f   coredll:COREDLL.dll
 0001:00017a40       CeEventHasOccurred         10018a40 f   coredll:COREDLL.dll
 0001:00017a50       IsAPIReady                 10018a50 f   coredll:COREDLL.dll
 0001:00017a60       DDKSdmaCloseChan           10018a60 f   cspddk:CSPDDK.dll
 0001:00017a70       DDKSdmaAllocChain          10018a70 f   cspddk:CSPDDK.dll
 0001:00017a80       DDKSdmaOpenChan            10018a80 f   cspddk:CSPDDK.dll
 0001:00017a90       DDKSdmaStartChan           10018a90 f   cspddk:CSPDDK.dll
 0001:00017aa0       DDKSdmaSetBufDesc          10018aa0 f   cspddk:CSPDDK.dll
 0001:00017ab0       DDKSdmaClearChainStatus    10018ab0 f   cspddk:CSPDDK.dll
 0001:00017ac0       DDKSdmaInitChain           10018ac0 f   cspddk:CSPDDK.dll
 0001:00017ad0       DDKSdmaStopChan            10018ad0 f   cspddk:CSPDDK.dll
 0001:00017ae0       DDKSdmaGetBufDescStatus    10018ae0 f   cspddk:CSPDDK.dll
 0001:00017af0       DDKSdmaClearBufDescStatus  10018af0 f   cspddk:CSPDDK.dll
 0001:00017b00       __rt_udiv64by64            10018b00 f   corelib1:COREDLL.dll
 0001:00017b10       __rt_sdiv                  10018b10 f   corelib1:COREDLL.dll
 0001:00017d40       __IMPORT_DESCRIPTOR_COREDLL 10018d40     coredll:COREDLL.dll
 0001:00017d54       __IMPORT_DESCRIPTOR_CSPDDK 10018d54     cspddk:CSPDDK.dll
 0001:00017d68       __IMPORT_DESCRIPTOR_CEDDK  10018d68     ceddk:CEDDK.dll
 0001:00017d7c       __NULL_IMPORT_DESCRIPTOR   10018d7c     coredll:COREDLL.dll
 0002:00000000       __imp_MmMapIoSpace         1001a000     ceddk:CEDDK.dll
 0002:00000004       __imp_MmUnmapIoSpace       1001a004     ceddk:CEDDK.dll
 0002:00000008       __imp_HalFreeCommonBuffer  1001a008     ceddk:CEDDK.dll
 0002:0000000c       __imp_HalAllocateCommonBuffer 1001a00c     ceddk:CEDDK.dll
 0002:00000010       __imp_HalTranslateBusAddress 1001a010     ceddk:CEDDK.dll
 0002:00000014       \177CEDDK_NULL_THUNK_DATA  1001a014     ceddk:CEDDK.dll
 0002:00000018       __imp_InterlockedDecrement 1001a018     coredll:COREDLL.dll
 0002:0000001c       __imp_InterlockedCompareExchange 1001a01c     coredll:COREDLL.dll
 0002:00000020       __imp_InterlockedIncrement 1001a020     coredll:COREDLL.dll
 0002:00000024       __imp_ExitThread           1001a024     coredll:COREDLL.dll
 0002:00000028       __imp_GetLastError         1001a028     coredll:COREDLL.dll
 0002:0000002c       __imp_CreateThread         1001a02c     coredll:COREDLL.dll
 0002:00000030       __imp_InterruptDone        1001a030     coredll:COREDLL.dll
 0002:00000034       __imp_InterruptInitialize  1001a034     coredll:COREDLL.dll
 0002:00000038       __imp_WaitForSingleObject  1001a038     coredll:COREDLL.dll
 0002:0000003c       __imp_Sleep                1001a03c     coredll:COREDLL.dll
 0002:00000040       __imp_InterruptDisable     1001a040     coredll:COREDLL.dll
 0002:00000044       __imp_CloseHandle          1001a044     coredll:COREDLL.dll
 0002:00000048       __imp_CeSetThreadPriority  1001a048     coredll:COREDLL.dll
 0002:0000004c       __imp_CeGetThreadPriority  1001a04c     coredll:COREDLL.dll
 0002:00000050       __imp_RegCloseKey          1001a050     coredll:COREDLL.dll
 0002:00000054       __imp_RegQueryValueExW     1001a054     coredll:COREDLL.dll
 0002:00000058       __imp_OpenDeviceKey        1001a058     coredll:COREDLL.dll
 0002:0000005c       __imp_CreateEventW         1001a05c     coredll:COREDLL.dll
 0002:00000060       __imp_InitializeCriticalSection 1001a060     coredll:COREDLL.dll
 0002:00000064       __imp_LocalAlloc           1001a064     coredll:COREDLL.dll
 0002:00000068       __imp_LocalFree            1001a068     coredll:COREDLL.dll
 0002:0000006c       __imp_DeleteCriticalSection 1001a06c     coredll:COREDLL.dll
 0002:00000070       __imp_EventModify          1001a070     coredll:COREDLL.dll
 0002:00000074       __imp_SetThreadPriority    1001a074     coredll:COREDLL.dll
 0002:00000078       __imp_GetTickCount         1001a078     coredll:COREDLL.dll
 0002:0000007c       __imp_CeSafeCopyMemory     1001a07c     coredll:COREDLL.dll
 0002:00000080       __imp_CeFreeAsynchronousBuffer 1001a080     coredll:COREDLL.dll
 0002:00000084       __imp_CeAllocAsynchronousBuffer 1001a084     coredll:COREDLL.dll
 0002:00000088       __imp_InterlockedExchange  1001a088     coredll:COREDLL.dll
 0002:0000008c       __imp___rt_udiv64by64      1001a08c     corelib1:COREDLL.dll
 0002:00000090       __imp___rt_sdiv            1001a090     corelib1:COREDLL.dll
 0002:00000094       __imp_IsAPIReady           1001a094     coredll:COREDLL.dll
 0002:00000098       __imp_CeEventHasOccurred   1001a098     coredll:COREDLL.dll
 0002:0000009c       __imp_KernelIoControl      1001a09c     coredll:COREDLL.dll
 0002:000000a0       __imp___rt_udiv            1001a0a0     corelib1:COREDLL.dll
 0002:000000a4       __imp_memmove              1001a0a4     corelib1:COREDLL.dll
 0002:000000a8       __imp_memcpy               1001a0a8     corelib1:COREDLL.dll
 0002:000000ac       __imp_memset               1001a0ac     corelib1:COREDLL.dll
 0002:000000b0       __imp___C_specific_handler 1001a0b0     corelib1:COREDLL.dll
 0002:000000b4       __imp___security_gen_cookie2 1001a0b4     corelib1:COREDLL.dll
 0002:000000b8       __imp___report_gsfailure   1001a0b8     corelib1:COREDLL.dll
 0002:000000bc       __imp_free                 1001a0bc     corelib1:COREDLL.dll
 0002:000000c0       __imp_realloc              1001a0c0     corelib1:COREDLL.dll
 0002:000000c4       __imp_malloc               1001a0c4     corelib1:COREDLL.dll
 0002:000000c8       __imp__msize               1001a0c8     corelib1:COREDLL.dll
 0002:000000cc       __imp_EnterCriticalSection 1001a0cc     coredll:COREDLL.dll
 0002:000000d0       __imp_LeaveCriticalSection 1001a0d0     coredll:COREDLL.dll
 0002:000000d4       __imp_RegisterDbgZones     1001a0d4     coredll:COREDLL.dll
 0002:000000d8       __imp_NKDbgPrintfW         1001a0d8     coredll:COREDLL.dll
 0002:000000dc       __imp_SetLastError         1001a0dc     coredll:COREDLL.dll
 0002:000000e0       __imp_DisableThreadLibraryCalls 1001a0e0     coredll:COREDLL.dll
 0002:000000e4       __imp_TerminateProcess     1001a0e4     coredll:COREDLL.dll
 0002:000000e8       \177COREDLL_NULL_THUNK_DATA 1001a0e8     coredll:COREDLL.dll
 0002:000000ec       __imp_DDKIomuxSetPinMux    1001a0ec     cspddk:CSPDDK.dll
 0002:000000f0       __imp_DDKIomuxSelectInput  1001a0f0     cspddk:CSPDDK.dll
 0002:000000f4       __imp_DDKSdmaCloseChan     1001a0f4     cspddk:CSPDDK.dll
 0002:000000f8       __imp_DDKSdmaAllocChain    1001a0f8     cspddk:CSPDDK.dll
 0002:000000fc       __imp_DDKSdmaOpenChan      1001a0fc     cspddk:CSPDDK.dll
 0002:00000100       __imp_DDKSdmaStartChan     1001a100     cspddk:CSPDDK.dll
 0002:00000104       __imp_DDKSdmaSetBufDesc    1001a104     cspddk:CSPDDK.dll
 0002:00000108       __imp_DDKSdmaClearChainStatus 1001a108     cspddk:CSPDDK.dll
 0002:0000010c       __imp_DDKSdmaInitChain     1001a10c     cspddk:CSPDDK.dll
 0002:00000110       __imp_DDKSdmaStopChan      1001a110     cspddk:CSPDDK.dll
 0002:00000114       __imp_DDKSdmaGetBufDescStatus 1001a114     cspddk:CSPDDK.dll
 0002:00000118       __imp_DDKSdmaClearBufDescStatus 1001a118     cspddk:CSPDDK.dll
 0002:0000011c       __imp_DDKClockGetFreq      1001a11c     cspddk:CSPDDK.dll
 0002:00000120       __imp_DDKClockSetGatingMode 1001a120     cspddk:CSPDDK.dll
 0002:00000124       \177CSPDDK_NULL_THUNK_DATA 1001a124     cspddk:CSPDDK.dll
 0002:00000128       dpCurSettings              1001a128     com_mdd2:mdd.obj
 0002:0000056c       __security_cookie          1001a56c     corelib0:seccinit.obj
 0002:00000570       __security_cookie_complement 1001a570     corelib0:seccinit.obj
 0002:00000578       _exitflag                  1001a578     corelib0:cexit.obj
 0002:00000584       __onexitend                1001a584     <common>
 0002:00000588       __onexitbegin              1001a588     <common>

 entry point at        0001:0000e9ec

 Static symbols

 0001:00007eac       SerialDispatchThread       10008eac f   com_mdd2:mdd.obj
 0001:0000ec4c       doexit                     1000fc4c f   corelib0:cexit.obj
 0001:0000faac       SerSerialInit              10010aac f   serial_common_topaz_v1:serial.obj
 0001:0000fb1c       SerInit                    10010b1c f   serial_common_topaz_v1:serial.obj
 0001:00010214       Ser_InternalMapRegisterAddresses 10011214 f   serial_common_topaz_v1:serial.obj
 0001:000103b4       Ser_GetRegistryData        100113b4 f   serial_common_topaz_v1:serial.obj
 0001:000105c8       SerIRInit                  100115c8 f   serial_common_topaz_v1:serial.obj
 0001:00010638       SerPostInit                10011638 f   serial_common_topaz_v1:serial.obj
 0001:000106c8       SerOpen                    100116c8 f   serial_common_topaz_v1:serial.obj
 0001:000107e8       SerClose                   100117e8 f   serial_common_topaz_v1:serial.obj
 0001:00010958       SerDeinit                  10011958 f   serial_common_topaz_v1:serial.obj
 0001:00010ae8       SerPowerOff                10011ae8 f   serial_common_topaz_v1:serial.obj
 0001:00010b88       SerPowerOn                 10011b88 f   serial_common_topaz_v1:serial.obj
 0001:00010c60       SerEnableIR                10011c60 f   serial_common_topaz_v1:serial.obj
 0001:00010d40       SerDisableIR               10011d40 f   serial_common_topaz_v1:serial.obj
 0001:00010e20       SerGetCommProperties       10011e20 f   serial_common_topaz_v1:serial.obj
